:020000040800F2
:1000000000200010CD4903083D020208C962000823
:10001000390202083502020831020208000000001D
:100020000000000000000000000000002D02020897
:10003000290202080000000025020208057C0008D1
:10004000354A0308354A0308354A0308354A030888
:10005000354A0308354A03089D0E0108C90F0108F7
:100060008D0F0108510F0108150F01081931000803
:1000700009310008F9300008E9300008D9300008DB
:10008000C5300008B1300008354A0308354A030876
:10009000590C0208354A0308354A0308D90E0108ED
:1000A0003573000885730008354A0308AD730008EE
:1000B0007573000865730008354A0308354A03085C
:1000C000354A0308354A0308354A0308354A030808
:1000D000354A0308C5FC00080D7D0008917C000826
:1000E000610E0108354A030815020208354A030863
:1000F00045730008354A030855730008354A03085C
:10010000000000000000000000000000354A030865
:10011000354A0308354A0308E1300208C5300208B1
:100120009D300008893000087530000861300008F3
:100130004D300008354A03080000000000000000B0
:10014000354A0308354A0308354A03080000000011
:10015000000000000000000000000000000000009F
:100160000000000000000000354A0308354A03087B
:10017000354A0308000000000000000000000000F5
:0801800000000000354A0308ED
:10018800002870B51EDB0928044620DD012303EB97
:1001980083035B00B0FBF3F2092AF8D87BB10E4E5B
:1001A800B4FBF3F00928CCBF57223022A6FB03E5A5
:1001B800024403FB1044EB0801F8012BF0D10023A3
:1001C8000B7070BD2D230B7040420131DBE73030DE
:1001D80001F8010BF3E700BFCDCCCCCC884230B49A
:1001E8004FF001042ED301FB04F4B0FBF4F58D426B
:1001F800F9D284B1AAB901E0B0FBF4F5092DCCBF5E
:10020800572230222A4404FB150003F8012BB4FBC3
:10021800F1F4002CF0D100221A7030BC7047B0FB0A
:10022800F4F5092DCCBF372230222A4404FB1500EF
:1002380003F8012BB4FBF1F4002CF0D100221A7062
:1002480030BC70470546002AEBD1D7E72DE9F047C7
:1002580014461D46064600234FF47A722046294666
:1002680034F0DCF9DFF840814B4A4C4F88FB003111
:100278000144C31782FB002EC3EB611188FB0128E0
:1002880087FB00278644464AC3EBEE2EC1EB011CD0
:1002980082FB0E29A0EB8C0C0744424A86F806C064
:1002A800C3EB27474FEAEE7C08EB010ACCEBA90C1D
:1002B80082FB07824FEAE1780CEB4C0CC8EB6A181A
:1002C800AEEBCC0EC8EB0818DFF8E0C086F804E007
:1002D800A1EB880171718CFB0010F917C1EBE212D8
:1002E80040F2B55101FB1272C3EBE050B2F5896FD1
:1002F8004FEA80073CDA40F2DA239A4242DCB2F550
:10030800B77FB4BF4FF0000C4FF0010C4FEA4C0917
:10031800DFF89C8009EB0C0308EBC3031FFA8CFE83
:10032800D88A09EB0C0108EBC10116310B2301E057
:1003380031F8020D824218DA013BF9D1CC4401238D
:1003480038F83C00B37007F2B2770132121ABE4493
:10035800F270A6F800E0204629464FF47A7200238E
:1003680034F05CF93281BDE8F0870133DBB2E9E7AC
:100378004FF0030EF44640F29650DFF834804FF009
:100388000609CEE74FF0020EDFF82480F44640F26B
:1003980029404FF00409C4E7C5B3A29107452EC20E
:1003A800ABAAAA2A73B06D1689888888792D03119B
:1003B800C85F030803685A1C02601970704700BFC1
:1003C8002DE9F047089C2578002B804689460CBF0C
:1003D8004FF0200A4FF0300A661C35B3002A29DD99
:1003E800334601E0024698B113F8011B501E00295C
:1003F800F8D1971E60B13D46013D51464046C84779
:100408006B1C002BF8DC257827EAE770013055B122
:10041800041B29464046C847301916F8015B002DD1
:10042800F7D1BDE8F087BDE8F087002A04DC28464C
:10043800BDE8F0870020EBE7571EDCE783684268D9
:10044800D0ED037A00EB83010133934281ED040A76
:10045800836004BF0023836000EB830393ED047A79
:10046800036870EE277A9A42C0ED037A77EEC77A6E
:10047800C0ED037A0CDA013307EE103AF8EEC76ADA
:10048800B7EE007A87EEA60A036030EE070A7047D7
:1004980007EE102AB8EEC77A87EE870A704700BFC2
:1004A80090ED057A90ED004AD0ED066AD0ED014A4C
:1004B800D0ED047A90ED035AD0ED025AA4EE007AFA
:1004C800B0EE406AB0EE470AB0EE667AA6EE247A3D
:1004D80067EEC07AA0EE457AE6EE257A80ED057AD9
:1004E800C0ED067A704700BFD0ED057A90ED013A6D
:1004F800D0ED003AD0ED064A90ED024A90ED077A29
:1005080090ED035A90ED086AD0ED045AC0ED067AD2
:10051800F0EE406A27EE830AC0ED056AA3EEA60A4C
:1005280080ED087AA4EE240AA5EE470AA5EEC60ACD
:1005380080ED070A704700BFD0ED007A90ED017A90
:1005480030EE670AE7EE007AB0EE670AC0ED007A8F
:10055800704700BF704700BF0A44914214D030B4BE
:100568000139551E41F2210211F8014F082380EA92
:10057800042004044CBF82EA40004000013B80B2E2
:10058800F7D18D42F0D130BC70474378007840EA0B
:10059800032010FB01F04FF4807190FBF1F000F3A1
:1005A8000F0000B270472DE9F74F6A4CDFF8A8E159
:1005B80023880091DEF80010B4F90480C3EB2112FF
:1005C8005B00C3EBE103B4F9021052435943131320
:1005D80008FB03F84FEAA83808EBE12101EB810298
:1005E800B1F5FA3802F180024FEAE1794FEA2223A5
:1005F80049F1FF39B4F908200193A8FB08AB08FBBF
:1006080009F30BEB430BA161D31702FB09F108FBBC
:100618000311A2FB08230B441F03160347EA1257D2
:10062800B4F90A2002FB0BF1D3170AFB03130546A2
:10063800A2FB0A011944020A42EA016292194FEA2E
:100648002123E6887B41003243F50043A2FB0601E3
:1006580006FB03114A10CB1752EA03016FD0B4F915
:100668001060B4F90E00F71706FB0BF10AFB07112F
:10067800A6FB0AAB8B4400FB09F6C11708FB016116
:10068800A0FB08898944DEF804104FEA4846C1F502
:10069800801E4FEA494747EAD8371AEB060AB4F9E9
:1006A8000C8076464BEB070BF71700264FEACE7007
:1006B800F90716EB0A064FEAC80741EA5E0147EB5D
:1006C8000B0740F6354E861B61EB0707A6FB0E01AC
:1006D8000EFB071133F0A2FFB4F916204E13470B97
:1006E80047EAC14702FB06FED31707FB03EEA2FB4E
:1006F80007237344564307FB0366A2FB07233344CF
:10070800560E46EAC3163218B4F914604FEA636706
:1007180047EB01037143F71700FB0717A6FB00011E
:100728003944C60C46EA413692194FEAE147B4F912
:1007380012607B41100A40EA0360320112180DB1C1
:10074800120A2A60009B13B11A46019B136003B07A
:10075800BDE8F08F5C3D0020481E002070477047C0
:1007680010B5064C237A0BB9002010BD07F002F92A
:10077800E368C01AD0F5FA50F6D410BD481E002020
:100788004FF40063838270474FF40063838270479D
:10079800012380F84530704707B5F7216A462FF0E6
:1007A8004BFD9DF801309DF800100C4A1B0143EAEF
:1007B80001339DF8021043EA111353609DF8043089
:1007C8009DF803101B0143EA01339DF8051043EA25
:1007D8001113136003B05DF804FB00BF481E00202E
:1007E80038B504460D46FFF7BBFF246808B107F08B
:1007F8000DF9054B00221A7249215B7A2A462046D8
:1008080010F07CFC012038BD481E002070B404683C
:10081800037B2268022101FA03F31A4213D04269CA
:100828000A495C2000FB02124FF6FE765068528996
:10083800C5680068296831402960C168D24392B20E
:100848000A40C260636070BC704700BF405200201D
:1008580030B40A4B1D7875B1094B002003EBC50570
:100868001A6899885062D4682143D160083323F804
:10087800040CAB42F4D130BC704700BF20550020B7
:100888002455002010B40268047B11680223A34099
:10089800194209D00649406800240C7001684FF6D7
:1008A800FE742140016053605DF8044B704700BF3F
:1008B800C3480020014B18680FF0AABAEC1E0020AC
:1008C8003122F42110F02CBDF0B5836983B00546C0
:1008D80013B11A689B8813856869264F8389C324D6
:1008E8004FF47A734FF0060E6E464FF6FF710137DC
:1008F80003E0013B9BB28B421DD002899207F8D5D9
:1009080004734FF47A7302E0A3B28B4213D00289C6
:10091800D20703F1FF34F7D5027BD2B20EB13270A1
:100928000136BEF1000F08D00EF1FF3EFF24002F64
:10093800E3D03C78DBE710F0C5FBAB6913B11A686C
:100948009B8893619DF805009DF801609DF8021051
:100958009DF803409DF804209DF8063041EA0621E1
:1009680043EA002342EA0422012029876A87AB87E9
:1009780003B0F0BD286003082DE9F04F89B090F866
:1009880055300390002B40F07985039BBF4CC04D38
:10099800DFF804931033184680226B21029310F07D
:1009A800BFFCBC48DFF8F4E24FF0640A4FF0100CCB
:1009B8004FF47A76D9F80430C3F30803002B40F0DB
:1009C8005B84EFF31183002B40F056842168826822
:1009D80000BF23689942F9D12F6806FB07F39B1AD9
:1009E800B3FBF7F306FB013101270191D9F8043075
:1009F800C3F30803002B40F00584EFF31183002BA9
:100A080040F000842368816800BF22689342F9D1CE
:100A1800D5F800B006FB0BF2521AB2FBFBF206FB4C
:100A28000323019A9B1AB3F57A7FDFD3BAF1010A3F
:100A3800C0D1072268210298DFF85C92954E10F029
:100A48006FFCDFF858C24FF0640A4FF010084FF4FB
:100A58007A77D9F80430C3F30803002B40F0F08309
:100A6800EFF31183002B40F0EB832168B26800BFDD
:100A780023689942F9D1286807FB00F39B1AB3FB56
:100A8800F0F307FB013101200191D9F80430C3F3D9
:100A98000803002B40F09983EFF31183002B40F0FB
:100AA80094832368B16800BF22689342F9D1D5F8CE
:100AB80000B007FB0BF2521AB2FBFBF207FB032351
:100AC800019A9B1AB3F57A7FDFD3BAF1010AC0D134
:100AD80052466B210298DFF8C09110F021FC6D4856
:100AE800DFF8B8E14FF0640A4FF0100C4FF47A7653
:100AF800D9F80430C3F30803002B40F06984EFF3FE
:100B08001183002B40F064842168826800BF236849
:100B18009942F9D12F6806FB07F39B1AB3FBF7F349
:100B280006FB013101270191D9F80430C3F308030A
:100B3800002B40F02D83EFF31183002B40F0288326
:100B48002368816800BF22689342F9D1D5F800B0C4
:100B580006FB0BF2521AB2FBFBF206FB0323019AC7
:100B68009B1AB3F57A7FDFD3BAF1010AC0D101220B
:100B78006B210298DFF8209110F0D2FB4548DFF88E
:100B88001CE14FF00F0A4FF0100C4FF47A76D9F8A9
:100B98000430C3F30803002B40F0FD83EFF3118307
:100BA800002B40F0F8832168826800BF23689942CF
:100BB800F9D12F6806FB07F39B1AB3FBF7F306FB83
:100BC800013101270191D9F80430C3F30803002B40
:100BD80040F0C182EFF31183002B40F0BC82236800
:100BE800816800BF22689342F9D1D5F800B006FBAE
:100BF8000BF2521AB2FBFBF206FB0323019A9B1A73
:100C0800B3F57A7FDFD3BAF1010AC0D1039B02980A
:100C180093F84F30DFF88090042B34BF18221A2243
:100C28001B2110F07DFB1B48DFF870E04FF00F0A26
:100C38004FF0100C4FF47A76D9F80430C3F3080358
:100C4800002B40F0FE83EFF31183002B40F0F98373
:100C58002168826800BF23689942F9D12F6806FB92
:100C680007F39B1AB3FBF7F306FB01310127019148
:100C7800D9F80430C3F30803002B40F04F82EFF398
:100C88001183002B40F04A820AE000BFC0760020A2
:100C9800C476002010E000E000ED00E0BC76002003
:100CA8002368816800BF22689342F9D1D5F800B063
:100CB80006FB0BF2521AB2FBFBF206FB0323019A66
:100CC8009B1AB3F57A7FD3D3BAF1010AB4D11822AB
:100CD8001C210298DFF8E89210F022FBB648DFF8F2
:100CE800DCE24FF00F0A4FF0100C4FF47A76D9F887
:100CF8000430C3F30803002B40F08783EFF311831C
:100D0800002B40F082832168826800BF23689942E3
:100D1800F9D12F6806FB07F39B1AB3FBF7F306FB21
:100D2800013101270191D9F80430C3F30803002BDE
:100D380040F0D781EFF31183002B40F0D281236874
:100D4800816800BF22689342F9D1D5F800B006FB4C
:100D58000BF2521AB2FBFBF206FB0323019A9B1A11
:100D6800B3F57A7FDFD3BAF1010AC0D1039B0298A9
:100D780093F84E20DFF848921A2110F0D1FA8E48E5
:100D8800DFF838E24FF00F0A4FF0100C4FF47A7684
:100D9800D9F80430C3F30803002B40F0A682EFF320
:100DA8001183002B40F0A1822168826800BF23686C
:100DB8009942F9D12F6806FB07F39B1AB3FBF7F3A7
:100DC80006FB013101270191D9F80430C3F3080368
:100DD800002B40F06981EFF31183002B40F0648110
:100DE8002368816800BF22689342F9D1D5F800B022
:100DF80006FB0BF2521AB2FBFBF206FB0323019A25
:100E08009B1AB3F57A7FDFD3BAF1010AC0D1039BED
:100E1800029893F85020DFF8A891192110F080FA71
:100E28006548DFF898E14FF0640A4FF0100C4FF472
:100E38007A76D9F80430C3F30803002B40F03982DE
:100E4800EFF31183002B40F034822168826800BFE1
:100E580023689942F9D12F6806FB07F39B1AB3FB65
:100E6800F7F306FB013101270191D9F80430C3F3E8
:100E78000803002B40F0FB80EFF31183002B40F0B8
:100E8800F6802368816800BF22689342F9D1D5F8BB
:100E980000B006FB0BF2521AB2FBFBF206FB03236F
:100EA800019A9B1AB3F57A7FDFD3BAF1010AC0D150
:100EB800102237210298DFF8089110F031FA3E48E5
:100EC800DFF8F8E04FF00F0A4FF0100C4FF47A7685
:100ED800D9F80430C3F30803002B40F04082EFF345
:100EE8001183002B40F03B822168826800BF236891
:100EF8009942F9D12F6806FB07F39B1AB3FBF7F366
:100F080006FB013101270191D9F80430C3F3080326
:100F1800002B40F08F80EFF31183002B40F08A8084
:100F28002368816800BF22689342F9D1D5F800B0E0
:100F380006FB0BF2521AB2FBFBF206FB0323019AE3
:100F48009B1AB3F57A7FDFD3BAF1010AC0D13821F1
:100F58000298DFF86C80194F012210F0E1F9164968
:100F68004FF00F094FF0100E4FF47A70D8F8043094
:100F7800C3F30803002B40F0D481EFF31183002B57
:100F880040F0CF8122688E6800BF23689A42F9D169
:100F9800D5F800C000FB0CF39B1BB3FBFCF300FB74
:100FA800023301930126D8F80430C3F308032BBB9E
:100FB800EFF3118313BB05E010E000E0BC760020DE
:100FC80000ED00E02368D1F808A000BF2268934232
:100FD800F8D1D5F800B000FB0BFCACEB0A0CBCFB5D
:100FE800FBFC00FB03C3019A9B1AB3F57A7FDAD3A3
:100FF800B9F10109BAD109B0BDE8F08FEFF3118A50
:101008008EF312888A680B68DB0344BF3E608A68E7
:101018002368D7F800C05FFA8AFA8AF31188D5F8EE
:1010280000A09C4400FB0AF39B1AB3FBFAF300FBF5
:101038000C33D8E7EFF311888CF3128881680368C2
:10104800DB0344BFCEF8007081682368DEF8002017
:101058005FFA88F888F31188D5F800801A4406FBEF
:1010680008F35B1AB3FBF8F306FB023367E7EFF309
:1010780011888CF3128881680368DB0344BFCEF8BB
:10108800007081682368DEF800205FFA88F888F32A
:101098001188D5F800801A4406FB08F35B1AB3FBE5
:1010A800F8F306FB0233FBE6EFF311888CF31288A2
:1010B80081680368DB0344BFCEF800708168236849
:1010C800DEF800205FFA88F888F31188D5F80080E8
:1010D8001A4406FB08F35B1AB3FBF8F306FB02336A
:1010E8008DE6EFF311888CF3128881680368DB03BF
:1010F80044BFCEF8007081682368DEF800205FFAEC
:1011080088F888F31188D5F800801A4406FB08F39C
:101118005B1AB3FBF8F306FB02331FE6EFF3118803
:101128008CF3128881680368DB0344BFCEF8007033
:1011380081682368DEF800205FFA88F888F3118850
:10114800D5F800801A4406FB08F35B1AB3FBF8F3E2
:1011580006FB0233B3E5EFF311888CF3128881683C
:101168000368DB0344BFCEF8007081682368DEF8AB
:1011780000205FFA88F888F31188D5F800801A44AF
:1011880006FB08F35B1AB3FBF8F306FB023335E5FD
:10119800EFF311888CF3128881680368DB0344BF7E
:1011A800CEF8007081682368DEF800205FFA88F8BE
:1011B80088F31188D5F800801A4406FB08F35B1AF7
:1011C800B3FBF8F306FB0233C9E4EFF3118E88F39F
:1011D8001288B1683368DB0344BFCCF80000B168FB
:1011E8002368DCF800205FFA8EFE8EF31188D5F8AC
:1011F80000E01A4407FB0EF35B1AB3FBFEF307FB90
:1012080002335DE4EFF311888CF312888168036878
:10121800DB0344BFCEF8007081682368DEF8002045
:101228005FFA88F888F31188D5F800801A4406FB1D
:1012380008F35B1AB3FBF8F306FB0233FFF7F1BBC5
:10124800EFF3118288F31288B0683368D90303D5A5
:101258000123CCF80030B0682368DCF80010D2B263
:1012680082F311882A68194407FB02F31B1AB3FB9F
:10127800F2F307FB013106E4EFF311828CF31288D5
:1012880087680368D90303D50123CEF8003087683F
:101298002368DEF80010D2B282F311882A68194454
:1012A80006FB02F3DB1BB3FBF2F306FB0131FFF78E
:1012B8009BBBEFF311828CF3128887680368D9030C
:1012C80003D50123CEF8003087682368DEF80010C4
:1012D800D2B282F311882A68194406FB02F3DB1B99
:1012E800B3FBF2F306FB0131BDE5EFF311828CF39A
:1012F800128887680368D90303D50123CEF8003024
:1013080087682368DEF80010D2B282F311882A6851
:10131800194406FB02F3DB1BB3FBF2F306FB0131B6
:1013280050E5EFF311868EF31288D1F808C00B68E8
:10133800DA0303D501233B60D1F808C023683A6873
:10134800F6B286F311882E681A4400FB06F3A3EB65
:101358000C03B3FBF6F300FB0233019322E6EFF331
:1013680011828CF3128887680368D90303D5012397
:10137800CEF8003087682368DEF80010D2B282F316
:1013880011882A68194406FB02F3DB1BB3FBF2F34E
:1013980006FB0131B6E5EFF311828CF312888768FA
:1013A8000368D90303D50123CEF800308768236882
:1013B800DEF80010D2B282F311882A68194406FBBD
:1013C80002F3DB1BB3FBF2F306FB0131FFF7F9BBBA
:1013D800EFF311828CF3128887680368D90303D569
:1013E8000123CEF8003087682368DEF80010D2B2F7
:1013F80082F311882A68194406FB02F3DB1BB3FB4E
:10140800F2F306FB0131FFF78DBBEFF311828CF38A
:10141800128887680368D90303D50123CEF8003002
:1014280087682368DEF80010D2B282F311882A6830
:10143800194406FB02F3DB1BB3FBF2F306FB013195
:101448006FE4EFF311828CF3128887680368D9037D
:1014580003D50123CEF8003087682368DEF8001032
:10146800D2B282F311882A68194406FB02F3DB1B07
:10147800B3FBF2F306FB0131FFF7F8BB1C09013C93
:10148800052C03F00F0300F293805C4A32F8140035
:1014980040FA03F2D50740F18B80012505FA03F3E2
:1014A800013B184033F00AF9554B564F1E5D064470
:1014B80017EBC6047CD057F83600B4F804E0038A6A
:1014C8001EEA03037FF461AA00F13842920A4E49EA
:1014D800E3718B5C03F01F025B092021022B05FAE4
:1014E80002F2A17100F08580032B7DD0012B64D01E
:1014F80006A90025CDF818E0079528F053FBA38826
:101508000398424AC260B3FA83F2C2F11F02511C27
:101518003ED0D1B201F0FC0303F1804303F58033E0
:1015280001F00301D3F808E04FEA81084FF00F0CEF
:1015380057F83610364F0CFA08F62EEA060600F170
:101548000C0E47F822E09E60D3F808E0314E324F87
:10155800C1F3872101FA08F141EA0E014FF00108B1
:10156800996008FA02FEB118C7F800E0082306A837
:10157800069291F868708DF81D308DF81E808DF8F0
:101588001C502EF0CBFE254AD35DF02B1ADCA38825
:10159800B3FA83F3C3F11F03581C3FF4F6A90122E1
:1015A80002FA03F31E490A6813430B60FFF7EDB90B
:1015B800039A164BD3600123F4E71A494B691A437F
:1015C8004A6195E7F319F02193F878308DF81430D3
:1015D80005A803238DF816508DF81780D1558DF87E
:1015E800153028F0A9FAD2E70E49CB691A43CA6127
:1015F8007EE70C498B691A438A6179E748880308B2
:1016080054880308F87E00205C88030899070008BE
:1016180034220020C85F030814040140742200200B
:1016280000040140001002402DE9F04F4269B24C1D
:101638001388DFF8D082B14E23F040031B041B0C43
:10164800138013889BB223F0380343F030031380D0
:1016580013889BB283B043F040031380019006F0D7
:1016680089F9DFF8A4E2A649844610274FF47A7571
:101678000120DEF80430C3F30803002B40F01D817D
:10168800EFF31183002B40F018812368D1F80890FC
:1016980000BF22689342F8D1D8F800A005FB0AF2EF
:1016A800A2EB0902B2FBFAF205FB03239C45E0D04A
:1016B800019D2846FFF760F9AB6913B11A689B884A
:1016C8001385019B586940F2E93302E0002B00F0D2
:1016D80038810289013B12F0020F9BB2F6D06A23CF
:1016E800037340F2E93302E0002B00F02A810289FB
:1016F800013B12F0010F9BB2F6D0037B019B5869A6
:1017080040F2E93302E0002B00F01E810289013B20
:1017180012F0020F9BB2F6D01023037340F2E933A4
:1017280002E0002B00F010810289013B12F0010F4A
:101738009BB2F6D0037B019B9B6913B11A689B8807
:101748009361DFF8C4916E486C4F4FF0640A4FF014
:10175800100E4FF47A75D9F80430C3F30803002B40
:1017680040F0D480EFF31183002B40F0CF80216844
:10177800826800BF23689942F9D1D8F8006005FB58
:1017880006F39B1AB3FBF6F305FB01310126009122
:10179800D9F80430C3F30803002B56D1EFF31183B3
:1017A800002B52D12368816800BF22689342F9D187
:1017B800D8F800B005FB0BF2521AB2FBFBF205FB9E
:1017C8000323009A9B1AB3F57A7FE1D3BAF1010A91
:1017D800C1D1019B4A4D5A69484F138823F04003F1
:1017E8001B041B0C1380138823F038031B041B0CE9
:1017F800138013889BB243F04003138006F0BAF8B5
:10180800DFF804C181464FF0100E4FF47A760120BC
:10181800DCF80430C3F30803002B31D1EFF3118354
:1018280073BB2368A96800BF22689342F9D1D8F82E
:1018380000A006FB0AF2521AB2FBFAF206FB0323D7
:101848009945E5D003B0BDE8F08FEFF3118C8EF326
:10185800128881680368DA0344BF3E6081682368A0
:101868003A685FFA8CFC8CF31188D8F800C01A44E7
:1018780005FB0CF35B1AB3FBFCF305FB0233A0E793
:10188800EFF311818EF31288D5F808A02B68DB03DB
:1018980044BF3860D5F808A023683A68C9B281F314
:1018A8001188D8F800101A4406FB01F3A3EB0A03C9
:1018B800B3FBF1F306FB0233C2E7EFF3118987F3B9
:1018C8001288D1F808A00B68DB0344BF3060D1F858
:1018D80008A0236832685FFA89F989F31188D8F873
:1018E80000901A4405FB09F3A3EB0A03B3FBF9F3D1
:1018F80005FB0233DAE600BFC0760020BC76002084
:1019080010E000E0C476002000ED00E0EFF3118263
:101918008EF3128886680368D90302D501233B60D9
:10192800866823683968D2B282F31188D8F8002013
:10193800194405FB02F39B1BB3FBF2F305FB0131D2
:1019480024E70FF0BFFBD9E60FF0BCFBF3E600BFBE
:1019580010B490E80600047B40690223A3404B6062
:1019680013685DF8044B4FF6FE710B4013600EF0E0
:10197800E3B9F8B5174D2B78A52B28D16B78BE2B7A
:1019880025D1022229464FF6FF70FEF7E5FD124FDA
:10199800AC1C22884AB1A618BE4218D2052A16D90C
:1019A8002146FEF7D9FD3446F3E721460222FEF729
:1019B800D3FD0222A118FEF7CFFD0634074B641BA6
:1019C8001C8041F60F53C31A58425841F8BD0020F5
:1019D800F8BD00BF00F0030800000408162D002021
:1019E8002DE9F04FDFF848914C4F8BB00326A7EB59
:1019F80009071822002104A834F073FA484BCDF8DF
:101A0800109005971A69120604D5464A5A6002F1E1
:101A180088325A6001228DF824203422DA60424B41
:101A2800424C1B88ADF800300222694604A80FF02A
:101A380013FE022269464FF6FF70FEF78DFDDFF8B0
:101A4800F4A080464FF0000B544536D30AAC00256D
:101A580024F8245D0222214604A80FF0FDFD02228D
:101A680021464046FEF778FD40BAC043ADF808006D
:101A7800022202A904A80FF0EFFD079860B106AB97
:101A8800C0F104022946184434F02BFA069904A838
:101A98000FF088FD079508909DF82430089A23B127
:101AA8001F490B6943F080030B61013E2DD0002ACA
:101AB8009FD1FFF75EFF50B32CE065888DF80DB01D
:101AC800C5F30B05AB1DADF808302388C3F30B0233
:101AD800ADF80A201B0B062202A904A88DF80C30C9
:101AE8000FF0BAFD062202A94046FEF735FD6168EF
:101AF80080462A4604A80FF0AFFD616840462A4692
:101B0800FEF72AFD143480469EE7002AD1D005202E
:101B180004F03EFC0BB0BDE8F08F00BF00000408E5
:101B2800002002402301674547600308C0C103083D
:101B380000F0030834C603080378202B024600F19E
:101B48000100F9D0092BF7D02D2B2CD02B2B03BF5C
:101B58005378B7EE000A0246B7EE000AA3F1300147
:101B6800C8B209289FED467A10D8F2EE046A07EE4B
:101B7800901AF8EEE77A12F8013FE7EE267AA3F119
:101B88003001C8B20928B0EE677AF0D92E2B4CD0B4
:101B980003F0DF03452B0BD0F7EE007A67EE276AD8
:101BA80020EE260A70475378BFEE000A0246D5E7B2
:101BB80010B451782D2959D02B290ABF9178501C7F
:101BC800901C0024A1F13003092B53D8002303EB08
:101BD800830301EB430310F8011FA1F13002092A26
:101BE800A3F13003F3D9B3F59A7F28BF4FF49A7362
:101BF800072B42D9DFED236A1A46F7EE007A083A36
:101C0800072A67EEA67AFAD803F007032BB1F2EE9B
:101C1800046A013B67EEA67AFBD124B3C7EE276AB4
:101C28005DF8044B20EE260A70475378A3F1300183
:101C3800C8B2092802F10102AAD8F2EE046AF0EE4D
:101C4800665A07EE901AF8EEE77A12F8013F87EE27
:101C5800A66AA3F13001C8B2092866EEA56A37EE74
:101C6800067AEED994E767EE276AD9E7901C91784F
:101C78000124A7E7F7EE007ACFE7F7EE007AC5E789
:101C88000000000020BCBE4CB5EEC00ADFED317A82
:101C9800F1EE10FACCBF30EE270A30EE670ADFED1E
:101CA8002E7A20EE270A30B5FDEEC07A87B017EEFF
:101CB800904A054684EAE470002303A9A0EBE47087
:101CC80001930093029328F0D1FE002CACBF20238F
:101CD8002D2303A88DF8003031F0D6FF012803A981
:101CE80024D002282DD0032805BF30236846684633
:101CF8008DF8013034F0FDF8684631F0C5FF03383F
:101D0800C4B222466946284634F02AF900232B55E6
:101D1800284631F0B9FF2E22431C2A540DEB04014A
:101D2800E81834F003F9284607B030BD3023684678
:101D38008DF801308DF802308DF8033034F0D9F881
:101D4800DAE7302368468DF801308DF8023034F038
:101D5800D0F8D1E76F12033A00007A442DE9F04138
:101D6800064615460846B6FBF2F43CB905FB146472
:101D7800124B1B5D00F8013BBDE8F081B4FBF2F7A4
:101D880067B90E4B05FB174705FB1464DA5D00F8CD
:101D9800012B1B5D00F8013BBDE8F081B7FBF2F8B1
:101DA800B8F1000F02D04046FFF7D8FF05FB1878BE
:101DB800024B13F8082000F8012BE3E7E88A030830
:101DC800104B2DE93048D3E9004554EA05020BD100
:101DD8000346012200201871587198719A70DA70C0
:101DE80018801881BDE83088074B1A6814EB020B7D
:101DF80045F1000C5A466346FEF728FA0120BDE873
:101E0800308800BFA01E0020C0760020F0B40288F1
:101E18008578154FC37804794179A2F2B27202F03D
:101E2800030606EB4606013D05EB8605013B37F840
:101E380015608579008940F2B557920807FB023290
:101E4800931903EB430304EBC303C3EB031301EB45
:101E58008303C3EB031305EB830300214FF47A726A
:101E6800C2FB0301F0BC7047C85F0308FAB170B445
:101E78008E18044603E0101A14D1B14214D014F895
:101E8800012BA2F14103192B11F8013BA3F14105E4
:101E980098BF2032192D03F12000ECD9D01A01D1B6
:101EA800002BEAD170BC7047002070BC7047104608
:101EB800704700BF4FF0FF32FFF7D8BFA0F16103B2
:101EC800192B98BF20387047A0F14103192B98BFF0
:101ED80020307047202805D0093804288CBF0020FE
:101EE8000120704701207047613819288CBF0020F5
:101EF80001207047413819288CBF00200120704705
:101F0800303809288CBF002001207047A0F1300329
:101F1800092B07D920F02000413819288CBF002050
:101F2800012070470120704730B402681146531CE5
:101F3800036011F8024B0160D31C51780360937859
:101F4800151D05601B0443EA0123D078234343EAA7
:101F5800006030BC704700BF0368591C1A46016016
:101F680012F8021B0260587841EA0020704700BF4F
:101F780003685A1C02601878704700BF38B50446D9
:101F88000068154632F01CFE22682A44226038BDDB
:101F9800036810B40A0A5C1C04601A7003685A1CAF
:101FA800026019705DF8044B704700BF03685A1C43
:101FB800026010B4197003680A0A5C1C04601A7085
:101FC80003680A0C5C1C04601A700368090E5A1C2A
:101FD800026019705DF8044B704700BF03685A1C13
:101FE800026019700368090A5A1C02601970704768
:101FF8002DE9F047002488B080460F461E46A146CA
:1020080005AD531C0393117839B3252933D1931C9B
:10201800CDF810900393507830284ED04FF0000A36
:10202800A0F13003DBB2092B42D96C2819D06428FF
:1020380000F0938024D825281CD063D9582876D05E
:1020480063281BD131784046B847039A531C039341
:102058001178043601340029D7D1204608B0BDE8EC
:10206800F087039B5A1C03921B78642B7CD02AD8D8
:10207800252B54D1252140460134B847039AC0E79F
:10208800732833D044D975284FD106F1040E30682F
:102098002B4600220A217646FEF7A0F8049A0095FE
:1020A800534639464046FEF78BF9039A0444A8E79D
:1020B80004AA03A92EF06AFFB7E7D31C039390780C
:1020C8004FF0010AACE7732B10D05BD9752B3AD0CF
:1020D800782B96D1A3F15802B2FA82F230685209ED
:1020E8002B4610210436FEF779F8D7E73368049AAF
:1020F8000093394600234046FEF762F9043604444B
:10210800039A7EE70028B9D1204608B0BDE8F087D9
:102118006E28B3D1039A336804361C6071E72AD954
:10212800582BD7D0632B8DD06BE77828A6D1A0F198
:102138005802B2FA82F2306852092B461021FEF793
:102148004DF80436AAE706F1040E30682B46002243
:102158000A217646FEF742F8A0E7331D3068294683
:102168001E46FEF70DF899E7331D306829461E46CE
:10217800FEF706F892E7002B7FF443AF204608B03D
:10218800BDE8F0876E2BC6D03BE700BF0EB400B5A4
:1021980084B005AB019053F8042B0649039301A8BA
:1021A800FFF726FF019B00221A7004B05DF804EBCC
:1021B80003B07047BD0300082DE9F04707468CB00F
:1021C8001E469246002A6AD1154614460A8840F2ED
:1021D800B1739A423AD98B78581E0B2836D891F8A1
:1021E80003E00EF1FF301E2830D891F804C0BCF18E
:1021F800170F2BD891F80590B9F13B0F26D888799D
:102208003B2823D8B1F80880B8F57A7F1ED24FF062
:102218000108002E34D109890491002CB4BF2D2166
:102228002B21002CB8BF6442039005910795CDF887
:102238000890CDF804C0CDF800E0384606942F4940
:10224800FFF7A4FF40460CB0BDE8F087002301214A
:1022580018468E46ADF824308DF828308DF8293090
:102268008DF82A30ADF82C3099469C461A46984687
:102278008DF826108DF827100B4609A9002ECAD014
:102288000390CDF80890CDF804C0CDF800E03846AA
:102298001B49FFF77BFF40460CB0BDE8F087194C9F
:1022A80084FB0234A318D417C4EB6314C4EB0415DD
:1022B800A2EB85052DB2002D0846B8BF6D42FFF789
:1022C800A5FD4FF47A7200238046894632F0A6F9BC
:1022D8003C230AFB030A4FF47A720023404649461E
:1022E80032F09CF94FF47A7192B20023C1FB0A23B1
:1022F80009A8FDF7ABFF24B209A967E7308B0308EB
:10230800108B0308898888880FB430B583B006AB72
:102318000B490C4853F8042B096800680193FFF730
:1023280067FE094C0546206803685B6998470028E2
:10233800F9D0284603B0BDE8304004B0704700BF6C
:10234800E82A0020EC2A0020EC1E0020DFED2B7A82
:10235800B4EEE70AF1EE10FA4ADDDFED296A9FEDE7
:10236800297A01E0B0EE670AB4EEC70AF1EE10FA76
:1023780070EE667AF6DC9FED247AF4EEC77AF1EE19
:1023880010FA38D5DFED1E6A9FED207A01E0F0EEF5
:10239800407AF4EEC77AF1EE10FA37EEA60AF6D4D0
:1023A800DFED1B7AB4EEE70AF1EE10FA14DDDFED8B
:1023B800137A37EEC00A60EE006A9FED166A9FED49
:1023C800167ADFED167AA6EE867A20EE266AE6EE13
:1023D800877AA6EE270A7047DFED117AB4EEE70A8E
:1023E800F1EE10FA44BFDFED087A37EEC00AE2E7F3
:1023F800F0EE407ABFE7B0EE670AD1E7DB0F49405D
:10240800DB0FC940E4CB1641DB0F49C0E4CB16C152
:10241800DB0FC93F92E741B99730083C15A82ABE9F
:10242800DB0FC9BF09B909E0194690FBF1F301FBBD
:1024380013030846002BF7D1084670470146FBE70F
:1024480007EE901AF8EE677A9FED837A27EE800AF6
:1024580020EE070AFDEEC07A17EE903A2033402BA3
:1024680000F28C80DFED7D7AB4EEE70AF1EE10FA27
:1024780040F3E880B0EE407A9FED796ADFED796A43
:1024880001E0B0EE677AB4EEE67AF1EE10FA77EE94
:10249800467AF6DC9FED747AF4EEC77AF1EE10FA1C
:1024A80040F1CD809FED6E6ADFED706A01E0F0EEDD
:1024B800477AF4EEE67AF1EE10FA37EE867AF6D439
:1024C800DFED6B7AB4EEE77AF1EE10FA51DCDFED6E
:1024D800697AB4EEE77AF1EE10FA44BFDFED627A7A
:1024E80037EEC77A27EE076ADFED635ADFED637AC6
:1024F800DFED636A9FED635AE6EE257A67EE065ACA
:10250800E6EE276AF7EE007AA5EEA67AF0EE675AAD
:10251800E7EE055AE7EE457A87EEA55ADFED547ADD
:1025280030EE277AFDEEC76A16EE903A2033402B3C
:1025380029D99FED557AF6EE006AB7EE006AF7EEF4
:10254800004AC4EEA57A0023836143610362C36134
:1025580080ED045A67EEA66A27EE866A27EE877A28
:10256800C0ED006AC0ED026A80ED016A80ED037A71
:102578007047DFED3A7A37EEC77AB3E7B7EE005A1D
:10258800F0EE455ACAE7B4EEE70AF1EE10FA5FDD5D
:102598009FED336ADFED336A01E0B0EE677AB4EE9F
:1025A800E67AF1EE10FA77EE467AF6DC9FED2E7AAF
:1025B800F4EEC77AF1EE10FA47D59FED296ADFED00
:1025C8002B6A01E0F0EE477AF4EEE67AF1EE10FAC3
:1025D80037EE867AF6D4DFED267AB4EEE77AF1EEB6
:1025E80010FA27DCDFED237AB4EEE77AF1EE10FA81
:1025F80044BFDFED1D7A37EEC77A27EE076ADFEDB5
:102608001E4ADFED1E6ADFED1E7AE6EE246A67EEEB
:10261800064AE6EE267AB7EE006AA4EEA77AF6EE48
:10262800006A36EE476AF8EE007A27EE277A66EEF9
:10263800266A84E7DFED097A37EEC77ADDE7B0EE80
:10264800677A3DE7F0EE407A24E7B0EE677AC2E7B2
:10265800F0EE477AAAE700BF27D4D236DB0F49400D
:10266800DB0FC940E4CB1641DB0F49C0E4CB16C1F0
:10267800DB0FC93FDB0FC9BF92E741B99730083C70
:1026880015A82ABEF304353F0000008070B4066820
:102698008E4217D90139751E002311F8014F0822FF
:1026A800634013F0800F4FEA430318BF83F0D5034C
:1026B800013ADBB2F5D18D42EFD1721C0260337062
:1026C80070BC70470023F8E710B44C09012250F899
:1026D800243001F01F0102FA01F10B4340F82430C5
:1026E8005DF8044B704700BF4B0901F01F0150F81B
:1026F8002320012303FA01F1114214BF18460020D8
:10270800704700BF0C480D4A0D4B10B44FF4FA4106
:1027180000240470118003F1EA045A202C213C2281
:10272800187059709A70D87019715A714E33A34243
:10273800F6D15DF8044B7047402B0020185200205A
:102748000A81002008B50EF033FD0A2005F05EF975
:10275800012008BDF8B50F4D46686A721446027A22
:102768000F4642F0800225213046FFF7EBFF3A463C
:1027780026213046FFF7E6FF04F00F0242F0800200
:1027880027213046FFF7DEFF05F0F4F8E860012066
:102798002872F8BD481E002070B50478032C0E4638
:1027A800154603D0BDE870400EF0BABD4468027A01
:1027B80025212046FFF7C6FF324626212046FFF78F
:1027C800C1FF2A4663212046FFF7BCFF812227214B
:1027D8002046FFF7B7FF012070BD2DE9F0410478CE
:1027E800032C884617461E4621D14468027A2521C3
:1027F80042F080022046FFF7A5FF424626212046E8
:10280800FFF7A0FF06F00F0242F0800227212046C2
:10281800FFF798FF042005F053F972B649213346B3
:102828003A4620460EF06AFC62B6BDE8F081BDE883
:10283800F0410EF001BD37B500F10C040546002249
:102848000A212046FFF7A8FF0F220A212046FFF79A
:10285800A3FF01AA032310212046FFF7BEFF9DF81E
:10286800043080336B839DF805308033AB839DF84B
:1028780006308033EB8300220A212046FFF78CFFC5
:102888000DF10302012302212046FFF7A6FF0123D1
:102898000DF1030209212046FFF79FFF11220A21AB
:1028A8002046FFF779FF012003B030BD2DE9FF472F
:1028B800037B0546884600F10C061BB1022B06D99E
:1028C800032B3DD00024204604B0BDE8F087012347
:1028D8000DF1070202213046FFF77FFF0028F1D0F3
:1028E8009DF80730D907EDD5072302AA0321304602
:1028F800FFF773FF0446002CE4D09DF80E701122F8
:102908000A213046FFF748FF3B07DBD4B5F91A1018
:1029180002A8FDF73AFE4042A8F80000B5F91C10DD
:102928000DF10A00FDF731FE4042A8F80200B5F9A2
:102938001E1003A8FDF729FE4042A8F80400C2E7CC
:10294800224F4FF0010A0024B9463B7C012B1BD0D3
:102958000FD3022BCFD1FDF703FF81460028B1D159
:1029680002A905F11000FDF73BFF87F81090044617
:10297800C1E73B7A23B9012202213046FFF7EAFE7C
:10298800012389F810309DE7FDF7EAFE002899D168
:1029980002A905F11000FDF723FF9DF80830044651
:1029A80008B1DA0707D4002389F81030BAF1000F0C
:1029B80088D09A46C9E73B7A23B9072203213046D3
:1029C800FFF7C8FE022389F810307BE7481E002075
:1029D800028822F040021204120C0280028822F0BF
:1029E80038031B041B0C59B141F48071002991FA7A
:1029F800A1F2B2FA82F108BF4FF0FF310139C900E4
:102A08000B439BB2038003889BB243F040030380CF
:102A1800704700BF08B540F2E93300E09BB1028976
:102A2800013B12F0020F9BB2F8D0017340F2E93378
:102A380000E043B10289013B12F0010F9BB2F8D0CC
:102A4800007BC0B208BD0EF03DFBC0B208BD00BFA0
:102A5800F8B584894FF6FF764FF47A742BB311B327
:102A68000F78013101E0B44217D00589013CAD0768
:102A7800A4B2F8D507734FF47A7402E0BCB2B4423A
:102A88000BD00589ED0704F1FF37F7D5057BEDB2CB
:102A98000AB115700132013BE0E70EF013FB00307C
:102AA80018BF0120F8BDFF27DFE70120F8BD00BFF0
:102AB800F0B55B4B5B4A97B01968914200AF00F0E4
:102AC800A3805949594A00234FF47000C1F888007F
:102AD8003B607B60136843F48033136003E03B681A
:102AE800B3F5A04F09D0136803F400337B603B684B
:102AF80001333B607B68002BF1D04C4B1B6813F40F
:102B0800003318BF01237B607B68012B52D0464CF1
:102B1800464B474AE260474A596A11605A6A42F08E
:102B280080725A625A6942F4FC025A6100250322F3
:102B380007F10801012341F6FF764FF09040FD6050
:102B4800BE603A73BB7327F02DF84FF6FF7307F199
:102B580008013948BB6027F025F807F10801374814
:102B6800374E27F01FF807F10801364827F01AF802
:102B780007F10801344827F015F807F10801334830
:102B880027F010F807F1080027F066F8BB6830490D
:102B9800304AA1FB031330499B0CF0204FF0070E7D
:102BA8005C370B60566084F823009560C2F800E03B
:102BB800BD46F0BD294A1D4B122111605A685A6062
:102BC8005A685A605A6842F480625A605A6822F415
:102BD8007C125A605A6842F4E8125A601A6842F045
:102BE80080721A601A689201FCD559680F4A21F060
:102BF80003015960596841F002015960536803F0B4
:102C08000C03082BFAD182E700221A6062B6144B33
:102C18001B6883F30888134B1B689847FEE700BFBF
:102C2800FC9F0020EFBEADDE00ED00E0001002408A
:102C38000005FA058C5500200004004800080048EB
:102C48003F190100000C004800100048001400481B
:102C580083DE1B4310E000E0C47600200020024021
:102C680000D8FF1F04D8FF1F064A0023516881427D
:102C780002F11C0204D001330C2BF7D1002070475D
:102C8800D8B270474C00002070B50F4C0F4DC0EB08
:102C9800C00004EB8004686926693043686182B02B
:102CA8009209667BA1600025012101A863618DF866
:102CB80004608DF805208DF806508DF8071026F071
:102CC8003BFF02B070BD00BF4C0000200010024066
:102CD800074BC0EBC00030B403EB8000054C05691E
:102CE80063692B4363610176427630BC704700BF4D
:102CF8004C000020001002402DE9F04F554C54F8CC
:102D0800204083B0002C60D0A56D1F469046524BE2
:102D18006A682265A160236004F15E014FF4807344
:102D280004F5AF726161A261E36023610646287E03
:102D380029F0A4FEE86858B1FFF796FF721CD2B2DA
:102D48000C21FFF7C5FF236DEA6862632433E3644F
:102D5800A86890B1FFF788FF721C8146D2B20B2198
:102D6800FFF7B6FF2346EA7E3C494846FFF78CFF4B
:102D7800236DAA68A2632833A36494F85D000DF05C
:102D8800DFFB814694F85C000DF0DAFB3A078246D7
:102D980095F819B01DD5B9F1000F1AD017F0110F19
:102DA8004FF00B0306F1010614BF4E213E2189F8AE
:102DB800063089F807605A4648460DF085FCFB073F
:102DC80043D5636B6BB3A36B5BB3204603B0BDE81D
:102DD800F08F17F0010F0CBF2E274E2718F0020FA7
:102DE8000DD0B9F1000F0AD00B22731C89F8062008
:102DF80089F8073048465A4639460DF065FC18F000
:102E0800010FDED0BAF1000FDBD001360C238AF8AF
:102E180007605A4639468AF8063050460DF054FC89
:102E2800CFE72B7FAA7E8DF804209B090021012281
:102E380001A88DF805308DF806108DF8072026F0CA
:102E48007BFE204603B0BDE8F08F48460DF0CAFF70
:102E5800B7E700BFF42A00204C600308591900089E
:102E680000B97047F0B595B005462AF08BF86C4E5E
:102E7800C368026832600446002B00F0C38028460D
:102E88000DF05EFB674B586118B12922002382714F
:102E9800C371227A644D2E210DF016FC306804F0BF
:102EA800F9FB29F0EBFD3068604A038823F0010341
:102EB8001B041B0C038014A91E232B8001270F233E
:102EC8000025138021F84C7D2D230293ADF80C507A
:102ED800ADF80650ADF80E502AF002F8E379ADF8D7
:102EE800145060229907ADF816500695ADF81C509D
:102EF800ADF81E50ADF82050ADF82250049200F104
:102F0800838013F0010F0CBF002202224FF480735C
:102F1800ADF81470ADF81C20ADF82030002304AAD9
:102F280061793068069304F007F861793068404F9A
:102F380029F0B6FF33685A6C42F400425A641A8882
:102F480092B242F080021A80E2796079196A920797
:102F58004CBF04220122824021EA02011962196A47
:102F68000A431A621A8892B242F001021A80207C3F
:102F780000222921FFF7ACFE2E49207C0023602285
:102F8800FFF782FEE068386026F042FD3868036883
:102F98004FF6FE721340036026F03AFD09A826F0AA
:102FA80009FD33686279244938680A913433134437
:102FB800099380221023002509A940F22A3E0E9287
:102FC8000B934FF400724FF400530D951095139521
:102FD80011950F921293ADF830E026F0F9FC627962
:102FE80033680C2A98BF1549D86898BF31F8125031
:102FF8003A6813490543DD601368012043F0020372
:103008001360087015B0F0BD13F0010F0CBF2A460D
:1030180008220423ADF81E20ADF816307EE700BF65
:103028008C820020481E002082820020808200209E
:10303800888200208D0800081C490020E87F0308CA
:10304800848200200348D0F83C3113B100F59A700F
:10305800184770474C0000200348D0F8203113B1BE
:1030680000F58C70184770474C0000200348D0F8D2
:1030780004310BB1FC301847704700BF4C000020EA
:103088000348D0F8E8300BB1E0301847704700BF6C
:103098004C0000200348D0F8CC300BB1C43018479E
:1030A800704700BF4C0000200348D0F8B0300BB187
:1030B800A8301847704700BF4C0000200348D0F8DC
:1030C80094300BB18C301847704700BF4C0000207B
:1030D8000248836F0BB17030184770474C000020CE
:1030E8000248C36D0BB15430184770474C0000209C
:1030F8000248036C0BB13830184770474C00002069
:103108000248436A0BB11C30184770474C00002036
:103118000248836803B11847704700BF4C0000207D
:10312800F8B505015A4C5B4B625961199A4204EB98
:10313800050704BF01230B730646387A29F09EFC65
:103148003B7A03F01F015B090122022B02FA01F20C
:1031580078D0032B71D0012B67D063190136187909
:103168000DF0EEF9F6B2074610B11223C67183715D
:10317800631958790DF0E4F910B11323C6718371FE
:10318800631998790DF0DCF910B11423C6718371B5
:1031980066190E21F27938460DF096FA70790DF01D
:1031A800CFF9F2790E210DF08FFAB0790DF0C8F948
:1031B800F2790E210DF088FA6359374A934251D0BB
:1031C800344A934259D0354A934240D02C44227B0A
:1031D800002A2FD1012002249A8822F48052120456
:1031E800120C9A80998889B241F4805199801A8882
:1031F80002F4415242F44572024322431A809A88EB
:1032080022F470621204120C42F4E0629A809A8BE3
:1032180022F400621204120C07219A8319821A8878
:1032280092B242F040021A80F8BD1D4B996A0A43D7
:103238009A6292E700200446CEE7194B19690A43BF
:103248001A618AE7164BD9680A43DA6085E702F5FE
:10325800EA32116941F400411161116921F4004118
:103268001161B3E702F56042D16841F48051D16041
:10327800D16821F48051D160A8E702F5EC321169D8
:1032880041F480411161116921F4804111619DE788
:10329800283D00200038004000300140003C00403C
:1032A80000100240F0B53A4C059D00EB800004EB9D
:1032B80080046468002C69D0364E49004FF42040E1
:1032C800CFB23060A169090453D46068DFF8D0E058
:1032D80047F4903100EA0E0001434FF4204061604A
:1032E800306003E0411E002847D00846A1698907DD
:1032F800F8D54FF42040A262306003E0421E002857
:103308003BD01046A2695106F8D5234A6168DFF818
:1033180090E0306042EA0342174301EA0E02174385
:103328006760BBB1013BDBB201332B444FF4204152
:10333800A269316052074FF4204005D4421EE0B123
:103348001046A2695207F9D5626A306005F8012B68
:103358009D42EDD14FF42040306002E0431E60B141
:103368001846A3699B06F9D520233060E361012044
:10337800F0BD411E08B10846A4E7084A1388013386
:103388009BB24FF0FF3113803160F0BD2046F0BD95
:10339800607600207C22002000240002142D0020EA
:1033A800009800FCF0B5037C012B85B0044663D07F
:1033B800022B67D1836913B11A689B8813856069EA
:1033C80040F2E93301E0002B6CD00289013B12F096
:1033D800020F9BB2F7D0C323037340F2E93301E035
:1033E800002B5FD00289013B12F0010F9BB2F7D08E
:1033F800037B60694FF0060E838902AE4FF47A733F
:103408004FF6FF71FF2703E0013B9BB28B423CD094
:1034180002899507F8D507734FF47A7302E0ABB2C7
:103428008B4232D00289D20703F1FF35F7D5027BF0
:10343800D2B20EB132700136BEF1010EE8D1A369E5
:1034480013B11A689B8893619DF80C009DF8086079
:103458009DF809109DF80A509DF80B209DF80D3035
:1034680041EA062143EA002342EA05220120218796
:103478006287A38705B0F0BD90F91400431C01D002
:10348800022805DD002005B0F0BD0DF01BFED6E7D3
:1034980002AB617D009343220623FFF703FF002858
:1034A800D2D1EFE70DF00EFEA3E700BFF0B5037A27
:1034B800012B85B0044663D0022B67D1036913B191
:1034C8001A689B881385E06840F2E93301E0002B15
:1034D8006CD00289013B12F0020F9BB2F7D0BB23DC
:1034E800037340F2E93301E0002B5FD00289013B0E
:1034F80012F0010F9BB2F7D0037BE0684FF0060E85
:10350800838902AE4FF47A734FF6FF71FF2703E009
:10351800013B9BB28B423CD002899507F8D50773D3
:103528004FF47A7302E0ABB28B4232D00289D207F1
:1035380003F1FF35F7D5027BD2B20EB132700136F6
:10354800BEF1010EE8D1236913B11A689B88936113
:103558009DF80C009DF808609DF809109DF80A5028
:103568009DF80B209DF80D3041EA062143EA00231F
:1035780042EA05220120E1822283638305B0F0BD7F
:1035880090F90C00431C01D0022805DD002005B08D
:10359800F0BD0DF097FDD6E702AB617B00933B22AF
:1035A8000623FFF77FFE0028D2D1EFE70DF08AFD52
:1035B800A3E700BF1749184B184A194810B4D1F8A7
:1035C800884044F47004C1F888401C6844F0010441
:1035D8001C605C6822405A601A6822F0847222F4E7
:1035E80080321A601A6822F480221A605A6822F41B
:1035F800FE025A60DA6A22F00F02DA621A6B0024BD
:1036080010404FF0006218639C608A605DF8044BBC
:10361800704700BF00ED00E0001002400CC07FF8CA
:10362800CCFC00FF2DE9F04F80462DED028BB0F960
:1036380008000881C5B28FB028460C4692462CF087
:1036480075F840B101231A46184662810FB0BDECE7
:10365800028BBDE8F08FA5F10A03ED2B00F2F08094
:10366800DFE813F0B701EE00EE00EE00EE00EE002A
:10367800EE00EE00EE00EE00EE00EE00EE00EE00D2
:10368800EE00EE00EE00EE00EE00EE00EE00EE00C2
:10369800EE00EE00FB01EE00EE00EE00EF04EE009F
:1036A800EE00EE00FE04EE000B05EE006A05EE00EB
:1036B8007904EE008504EE008D04EE00B304EE00FC
:1036C800EE00EE00C804CE04EE00D504EE00EE00D5
:1036D800E804EE009706EE00EE00EE007507EE0037
:1036E800EE00EE00EE002507EE00C901EE00F5053C
:1036F8001A06EE00EE00EE00EE00EE00EE00EE0020
:103708003D06EE006906EE001902EE006802EE00C2
:10371800BB02EE00EE00EE00EE00CE02B305EE05B1
:103728004407EA01EE00EE00B203C803EE00FA0314
:103738003104EE00EE00EE00EE001907EE00EE0098
:10374800BF06EE00EE00EE000A07F4020A031D03AE
:10375800EE00EE00EE005E03EE006C037A03EE006E
:10376800EE00EE00EE00EE00EE00EE00EE00EE00E1
:10377800EE00EE00EE00EE00EE00EE00CE02EE00EF
:10378800EE00EE00EE00EE00EE00EE00EE00EE00C1
:10379800EE00EE00EE00EE00EE00EE00EE00EE00B1
:1037A800EE00EE00EE00EE00EE00EE00EE00EE00A1
:1037B800EE00EE00EE00EE00EE00EE00EE00EE0091
:1037C800EE00EE00EE009A03EE00EE00EE00EE00D2
:1037D800EE00EE00EE00EE00EE00EE00EE00EE0071
:1037E800EE00EE00EE00EE00EE00EE00EE00EE0061
:1037F800EE00EE00EE00EE00EE00EE00EE00EE0051
:10380800EE00EE00EE00EE00EE00EE00EE00EE0040
:10381800EE00EE00EE00EE00EE00EE00EE00EE0030
:10382800EE00EE00EE00EE00EE00EE00EE00EE0020
:10383800A8034E04EE00EE00EE00EE00EE00830555
:10384800742D58D0772D10D1D8F80030D8F804202E
:103858009A421EBF5A1CC8F800201978A74A08BF08
:10386800002120462EF0B8FAECE6F52D54D0D8F811
:103878000410D8F80060A5F1210381468A1B362B75
:1038880000F26C87DFE813F00E076A076A076A0719
:103898006A076A076A076A0734076A076A076A07CE
:1038A8006A076A076A076A076A076A076A076A0788
:1038B8006A076A076A076A07FA066A076A076A07E9
:1038C8006A076A076A076A076A076A076A076A0768
:1038D8006A076A076A076A076A076A076A076A0758
:1038E8006A076A076A076A076A076A07C3066A07F0
:1038F800A0066A079B06D8F80030D8F804209A4238
:103908001EBF5A1CC8F8002019787D4A08BF00213C
:1039180020462EF061FA95E6D8F80030D8F8042051
:103928009A4242F00180774BFF221A724FF000084A
:10393800754D1EF03DFA41462022744885F80080F6
:1039480032F0CFFA8DF814809DF81430072B02F26C
:103958001E816F4F6D4E42469DF8143003EB4303B2
:1039680007EBC3035B7CE3B19DF8143003EB43031F
:1039780007EBC30320215B699BB19DF8143003EB6F
:10398800430307EBC303586946F822000DF06EF8AD
:103998002B7856F823000DF02BFA2A780132D2B290
:1039A8002A709DF814300133DBB28DF814309DF87D
:1039B8001430072BD0D92368591C21601A70BAF12A
:1039C800000F3FF43FAE534BCAF8003001231A46AC
:1039D8003AE6514D284630F057F900287FF732AEC5
:1039E8002B460544226813F8011B501C9D42206099
:1039F8001170F7D126E6494E3378002B3FF422AEFA
:103A0800474F0025B846236817F81520591C216030
:103A18001A7098F8011001EB810101EB810101F2A4
:103A2800EE2189B22046FEF7D9FA337801359D4256
:103A380008F10208E7DB05E6384E3378002B3FF43F
:103A480001AE384F002537F8021F2046FEF7C6FAA8
:103A5800337801359D42F6DBF4E5334D05F1500628
:103A680028782EF00DFA2368027A591C21601A7002
:103A780023686A78591C21601A702368AA78591C2F
:103A880021601A702368EA780435591CAE42216017
:103A98001A70E5D1D6E5254E23687279244D591C54
:103AA80021601A702B682046198CFEF797FA2B684C
:103AB8002046D98BFEF792FA71892046FEF78EFAD6
:103AC800B1892046FEF78AFA2B682046598CFEF702
:103AD80085FA2B682046998CFEF780FAF1892046F2
:103AE800FEF77CFA318A2046FEF778FA2A682368BE
:103AF80092F82620591C21601A70A3E55514030872
:103B0800A1140308901E0020F7830020B88300202A
:103B18005851002039350308464C00202033002036
:103B28008C3500201E78002084340020F44F0020BB
:103B38002441002020460021FEF750FA20460021AB
:103B4800FEF74CFA20460021FEF748FA2368AF4DED
:103B580000265A1C22601E7023682A68591C92F895
:103B68002C2021601A7023682A68591C92F8362084
:103B780021601A7023682A68591C92F8372021603E
:103B88001A7023685A1C22601E7023685A1C22600F
:103B98001E7023685A1C22601E702B682046598F9D
:103BA800FEF71CFA2B682046198FFEF717FA2368D0
:103BB8002A68591C92F82E2021601A7023685A1C12
:103BC80022601E702B682046598EFEF707FA2B6874
:103BD8002046998EFEF702FA34E523688C4A8D490F
:103BE800D0788D4A5D1C2560187023684979581C67
:103BF800206019702368D278591C21601A7021E559
:103C08000023DFF84892DFF848B204930393059342
:103C18000693984601214FF6FF7A07E008F101085C
:103C2800B8F10B0F01F0A28519F9011F4F1C4AFAD0
:103C380008F3F3D0DE07F1D5BBF8003043FA08F3F8
:103C4800D807EBD505A8FEF73FFDE7E72268734BD9
:103C580073491878551C2560107022685878551CCF
:103C68002560107022689B78501C20601370C988EA
:103C78002046FEF7B3F9E5E423686A4A64491078F8
:103C8800654A5D1C2560187023688978581C206077
:103C9800197023689278591C21601A70D2E4DFF8F1
:103CA800B4E10027FEB2714600232268501C206050
:103CB80016702268501C20601370226811F8010FDA
:103CC8000133551C062B25601070EED10137062FE5
:103CD8000EF1060EE6D1544900232268501C2060DC
:103CE80017702268501C20601370226811F8010FA9
:103CF8000133551C0B2B25601070EED123684B4AFD
:103D0800581C07212060197023680021581C206066
:103D18001970236892F8F020591C21601A7091E4F8
:103D2800434D2046298AFEF759F9698A2046FEF74D
:103D380055F9A98A2046FEF751F983E4364B3D49E7
:103D4800B3F9003081FB0321DB17C3EBA10189B272
:103D58002046FEF743F975E42368374F591C3A7833
:103D680021601A703B78002B3FF46CAC0025EEB252
:103D780030461BF045FB23684278591C21603046C9
:103D88001A701BF03DFB01892046FEF727F93B78A6
:103D980001359D42EBDB55E42368284A591C12780B
:103DA800216005A81A70FEF70BF823685A1C2260D8
:103DB800187047E4164D2046E989FEF70FF9A989DE
:103DC8002046FEF70BF93DE41D4D20462988FEF7F5
:103DD80005F969882046FEF701F9B5F90430154957
:103DE800DA1781FB0313C2EBA30399B22046FEF74F
:103DF800F5F827E4134B20461968FEF7D7F8124B5D
:103E080020461988FEF7EAF81CE400BF2441002088
:103E1800C43700202C7A0020D4370020BC3700207B
:103E2800E0460020F44F00202348002040470020AF
:103E38001852002067666666AD3D00200A3C0020E7
:103E4800D0400020C8400020CC400020A4600308D7
:103E580020410020FF470020AA4D23682A68591CEA
:103E6800127821601A702B6822689978531C236095
:103E7800002311702A6821681A4401335279481CBA
:103E8800032B20600A70F5D123682A68591C127A1E
:103E980021601A7023682A68591CD27821601A7028
:103EA80023682A68591C127921601A702B682046E9
:103EB8005989FEF793F82A682368527A591C2160B9
:103EC8001A702A68D2E0904D00232268286803EB14
:103ED8004301561C405C266010702A6820680A441A
:103EE800461C5278266002702A6820680A4401330A
:103EF8009278411C0A2B21600270E6D1FFF7A2BB21
:103F0800824B03F1700522681978501C20601170EB
:103F180022685978501C2060117022689978501CCA
:103F2800206011702268D978501C206011702268B6
:103F38001979501C2060117022685979501C206032
:103F48001170226899790733501CAB4220601170B8
:103F5800D9D1FFF777BB6E4D05F1800655F8041FE0
:103F68002046FEF723F8AE42F8D1FFF76BBB236873
:103F7800684A591C527D21601A70FFF763BB664B73
:103F880003F15A0522685979501C20601170226883
:103F98001978501C2060117022685978501C2060D4
:103FA800117022689978501C206011702268D978A5
:103FB800501C20601170226819790633501C9D42EC
:103FC80020601170DED1FFF73DBB544D544E05F112
:103FD800200795F90210534B93F906208A4203F102
:103FE800080301F0A5839E42F6D10835AF42F0D10F
:103FF800FFF728BB00212046FDF7D8FFFFF722BBBB
:1040080023680122991821601A70FFF71BBB2368E7
:10401800454A464990785D1C256018702368527897
:10402800581C20601A7023680A79591C21601A707C
:10403800FFF708BB082237492046FDF79FFFFFF727
:1040480001BB3B4D20462988FDF7C8FFA9882046BB
:10405800FDF7C4FF29892046FDF7C0FFFFF7F2BA34
:104068002368344A581C11782060197023685278E4
:10407800591C21601A70FFF7E5BA264D23682A7A81
:10408800591C21601A70A98B2046FDF7A7FF298BC0
:104098002046FDF7A3FF698B2046FDF79FFF2368A5
:1040A800EA7C591C21601A70A98C2046FDF796FFFE
:1040B800E98C2046FDF792FF2368AA7F591C2160EE
:1040C8001A70236895F82020591C21601A70698C91
:1040D8002046FDF783FF2368EA7A591C21601A708D
:1040E800E9682046FDF762FF23682A7C591C216095
:1040F8001A70236895F82120591C21601A70FFF75F
:10410800A1BA00BF2841002024410020082F002028
:104118003C470020E07A0020003000200C7B002083
:104128008855002068550020E4370020901E0020A4
:10413800202B0020F83C0020BB4D05F14006B5F8C7
:1041480080102046FDF74AFF236895F88220591C05
:1041580021601A70236895F883200435591CAE42F3
:1041680021601A70EBD1FFF76DBA05A8FDF728FE9C
:1041780000283FF467AABDF814102046FDF72EFF6B
:1041880023689DF81620591C21601A7023689DF831
:104198001720591C21601A7023689DF81820591C93
:1041A80021601A7023689DF81920591C21601A7023
:1041B80023689DF81A20591C21601A70BDF81C103C
:1041C8002046FDF70BFFFFF73DBA984B9B8AB3F5E6
:1041D800006F01F2A683B3F5806F01F2FB83B3F59C
:1041E800007F34BF01270227914D05F10C0655F8D1
:1041F800041B91FBF7F1204689B2FDF7EFFEB542AB
:10420800F5D18C4D8C4F05F10C06B5EC010AD7EDB4
:10421800077A80EE270A30F0A7FE81B22046FDF724
:10422800DDFEAE42F1D1854D05F10C0655F8041BB3
:10423800204689B2FDF7D2FEB542F7D1FFF702BAA0
:1042480010227F492046FDF799FEFFF7FBB9236846
:104258007C4D01269A1922601E701AF021FC002854
:1042680041F09383784B2268511C216010702268BA
:1042780041F2B410511C185C216041F278111070A1
:1042880059582046890AFDF791FEA96A204649082F
:10429800FDF78CFEFFF7D6B923686C4D591C012237
:1042A80021601A702368AA78591C21601A7016F0C8
:1042B8008BFC2368664A67495E1C26601870B1F952
:1042C8000010B2F90000FEF7ADF823685A1C22600E
:1042D800187029882046FDF781FEFFF7B3B91FF053
:1042E80027FEFF28054601F05E830EA8002300F88C
:1042F800243D1FF0EFFD2268574B511C21601570BB
:1043080022681978501C2060117022685978501C56
:104318002060117022689978501C20601170226802
:104328009DF81410501C2060117099882046FDF7E4
:1043380055FEFFF787B9494FFB78002B01F0E4825F
:1043480023680822591C21601A70236801229918D1
:1043580021601A702368424D591C2A7921601A700D
:104368002368AA78591C21601A7029882046FDF70D
:1043780035FEE9892046FDF731FE2368FA79591C94
:1043880021601A702368EA78591C21601A70FFF7B7
:1043980059B92368334A344D1178344A581C20607F
:1043A800197011682046FDF701FE2368304A591C30
:1043B800127A21601A7029882046FDF70FFEA98815
:1043C8002046FDF70BFE29892046FDF707FE20460B
:1043D8000021FDF703FE00212046FDF7FFFDFFF752
:1043E80031B9244D05F16006A9882046FDF7F6FD90
:1043F800E9882046FDF7F2FD29892046FDF7EEFD04
:104408002368AA7A591C21601A702368EA7A591C11
:1044180021601A7055F80C1B2046FDF7C7FDB54200
:10442800E2D1FFF70FB900BF40470020D840002075
:10443800084100200C5000207C4D0020743C0020D6
:10444800B03C00209C71002010570020F677002017
:104458000A3600201036002038560020F44F00207D
:1044680018520020F83C0020202B00205C820020FD
:10447800E07A0020482E0020A94D20462988FDF723
:10448800ADFD69882046FDF7A9FDA9882046FDF7FE
:10449800A5FDFFF7D7B8A34952232268501C206016
:1044A800137011F8013F002BF7D1FFF7CBB8236841
:1044B8009D4D591C2A7921601A7023686A79591C04
:1044C80021601A7029882046FDF788FD2368AA799B
:1044D800591C21601A7069882046FDF77FFD236802
:1044E800EA79591C21601A70FFF7ACB88F4D904ECD
:1044F800DFF86082DFF860929FED8E8A05F1200771
:104508000EE0FCEEE77ACDED017ABDF80410204606
:104518000435FDF763FDBD4206F118063FF492A885
:10452800717C0029F3D098F80030D5ED007A012B82
:10453800E7D1D9F80030DB0441F1BC81F5EE407ACF
:10454800F1EE10FA41F05B8240F2DC51DFE72368BC
:1045580000255A1C226029461D702046FDF726FDBD
:1045680029462046FDF722FD29462046FDF71EFD77
:10457800FFF768B80723B2FBF3F3C3EBC301521A82
:104588001DD1DBB203F1FF395FFA89F9002B3FF443
:1045980059A8DFF8A4B109F101091746731CC8F836
:1045A800003096F90010644B002593F902208A42E6
:1045B80003F1080301F057820135042DF5D14FF0BE
:1045C800FF331A46FFF740B8731CC8F80030357837
:1045D800FF2D01F07B82FE2D01F031824046FDF770
:1045E800BBFC98E80C009B1A002B07DD531CC8F88D
:1045F8000030137813B90C2D41F2A982272DDED88B
:104608004E4A012322F815001A46FFF71DB8731CFD
:10461800C8F8003030780328D1D8431E484D49499E
:10462800DBB203EB430305EB430308705D78002816
:104638003FF408A8531EDBB2AB42C0D10022C1F838
:104648000620C1F802208A726BB1581CD8F80030D5
:1046580008444A1C0133C8F8003013F8011C02F85A
:10466800011F8242F6D1384B1B78002B3EF4EAAF8B
:104678002CF07DFC01231A46FEF7E6BF731CC8F830
:10468800003033780A2B01F0A8814046FDF770FC12
:104698004046FDF76DFC4046FDF76AFC01231A46CB
:1046A800FEF7D2BF3346721CC8F80020274D13F816
:1046B800022B6A70C8F8003073782B70F31CC8F8A6
:1046C8000030B378AB704046FDF746FCD8F80030B0
:1046D80028811A46591CC8F8001012F8021B697183
:1046E800C8F800205B78AB7101231A46FEF7ACBF0F
:1046F800731CC8F8003033780A2B01F06581502B01
:1047080040F09C864046FDF727FC114D2880404626
:10471800FDF722FC012368801A46FEF795BF00BF0B
:10472800E046002074600308FC460020C03C0020DE
:1047380058510020000040420C7B00208877002060
:1047480018620308307B002034230020A840002092
:10475800B82300203C52002018500020A5F10B007F
:10476800EF283FF62CAF01A353F820F0ED560008D0
:10477800C7450008C7450008C7450008C7450008E1
:10478800C7450008C7450008C7450008C7450008D1
:10479800C7450008C7450008C7450008C7450008C1
:1047A800C7450008C7450008C7450008C7450008B1
:1047B800C7450008C7450008C7450008C7450008A1
:1047C800C7450008C7450008C745000873560008D4
:1047D800C745000859560008C7450008375600085D
:1047E800C7450008C7450008C74500080B5600081C
:1047F800C7450008A5550008C745000831550008F9
:10480800C745000805550008C7450008295700088E
:10481800C7450008A3540008C74500087D4500089F
:10482800C7450008C7450008C7450008C745000830
:104838004D360008C745000871540008C7450008F0
:10484800C745000855540008C7450008FD5300082F
:10485800C7450008C7450008C7450008C745000800
:10486800C7450008C7450008C7450008C7450008F0
:10487800B1530008C745000863530008C74500083E
:10488800C74500087D510008C7450008C74500080E
:10489800C7450008C7450008C7450008C7450008C0
:1048A800C745000811510008C745000829520008EB
:1048B800C745000875500008C7450008AF520008F2
:1048C800C7450008E3500008BB51000857500008CE
:1048D800C7450008C7450008C7450008C745000880
:1048E800C7450008C7450008C7450008C745000870
:1048F800C7450008C7450008C7450008C745000860
:10490800C7450008C7450008C7450008C74500084F
:10491800C7450008C7450008C7450008C74500083F
:10492800C7450008C7450008C7450008C74500082F
:10493800C7450008C7450008C7450008C74500081F
:10494800C7450008C7450008C7450008C74500080F
:10495800C7450008C7450008C7450008C7450008FF
:10496800C7450008C7450008C7450008C7450008EF
:10497800C7450008C7450008C7450008C7450008DF
:10498800C7450008C7450008C7450008C7450008CF
:10499800C7450008C7450008C7450008C7450008BF
:1049A800C7450008C7450008C7450008C7450008AF
:1049B800C7450008C7450008C7450008C74500089F
:1049C800C7450008C7450008C7450008C74500088F
:1049D800C7450008C7450008C7450008C74500087F
:1049E800C7450008C7450008C7450008C74500086F
:1049F800C7450008C7450008C7450008C74500085F
:104A0800C7450008C7450008C7450008C74500084E
:104A1800C7450008C7450008C745000825500008D5
:104A2800C74500080F500008E14F0008C7450008B7
:104A3800C7450008C7450008C7450008C74500081E
:104A4800C7450008C7450008C7450008C74500080E
:104A5800C7450008C7450008C7450008C7450008FE
:104A6800854F0008C7450008474F0008C74500089C
:104A7800994E0008374E00081B4E0008C74500082D
:104A8800014E0008C7450008D74D0008C54D00086D
:104A9800654D0008C74500083D4D0008C74500089A
:104AA800C74500081B4D0008E74C0008D34C000818
:104AB800A54C00087F4C00085D4C0008C74500085D
:104AC800454C0008C7450008C7450008C745000809
:104AD800C7450008C7450008C7450008C74500087E
:104AE800C7450008C7450008C7450008C74500086E
:104AF800C7450008C7450008C74500082B4C0008F3
:104B0800C7450008C7450008C14B0008C74500084D
:104B1800C7450008C74500084F4B0008C7450008AF
:104B2800C7450008C7450008354B0008C64B1B7829
:104B3800DB073FF544AD01F021FC01F0FBFD01234B
:104B48001A46FEF781BD4046FDF706FAD8F8003050
:104B5800ADF814001A46591CC8F8001012F8021BC8
:104B6800C8F800208DF816105A788DF81720DA1C2E
:104B7800C8F800209A788DF818201A1DC8F8002067
:104B8800DA788DF819205A1DC8F800201B798DF89D
:104B98001A3005A80023ADF81C30FDF737F9AB4BE8
:104BA800AB4A1D68401B4FF0010361F10001C2E9E7
:104BB80004011A46FEF748BD731CC8F80030337864
:104BC8000F2B3FF6FCACB21CC8F80020C3EBC303A4
:104BD800A04A7178D154F11CC8F800101344B27877
:104BE8005A70321DC8F80020F2789A70721DC8F801
:104BF80000203279DA70B21DC8F8002072791A7173
:104C0800F21DC8F80020B2795A7106F10802C8F8F6
:104C18000020F2799A7127F0D5F901231A46FEF798
:104C280013BD4046FDF798F98B4DE8814046FDF7E6
:104C380093F90123A8811A46FEF706BD4046FDF701
:104C48008BF9864900EB8000420001230A801A464E
:104C5800FEF7FABC4046FDF77FF9814D28824046B1
:104C6800FDF77AF968824046FDF776F90123A882B4
:104C78001A46FEF7E9BC3346721CC8F8002013F840
:104C8800020BC8F80030F31C7178C8F80030B2780D
:104C980022F000FB00287EF4D5AC90E43346721C69
:104CA800C8F800206F4A13F8021B1170C8F80030CA
:104CB800694A73789370F31CC8F80030674BB27870
:104CC8009A7001231A46FEF7BFBC674B67491868FC
:104CD8004E222FF075FF01231A46FEF7B5BC324667
:104CE800731CC8F80030624B12F8021B1970C8F820
:104CF800002072785A70F21CC8F80020B2789A70B6
:104D08004046FDF729F95B4A0123D0801A46FEF791
:104D18009BBC4046FDF720F9564D28804046FDF7DC
:104D28001BF968804046FDF717F90123A8801A4649
:104D3800FEF78ABC504F3B78002B3EF483AC4F4EB5
:104D480000254046FDF708F920F0E4F83B78A6EC8A
:104D5800010A01359D42F4DBFEF774BC0D2A7FF48D
:104D68002EAC731CC8F800303578072D3FF627ACF9
:104D7800434F40460C26FDF7EFF806FB05F6BD1934
:104D8800A8804046FDF7E8F8E8804046FDF7E4F8DB
:104D9800D8F8003028811A46591CC8F8001012F8B3
:104DA800021BA972C8F800205B78EB724046FDF739
:104DB800BBF80123B8511A46FEF746BC4046FDF73A
:104DC800CBF8304A012310801A46FEF73DBC731C0D
:104DD800C8F800303078060600F181871A4B1B7836
:104DE800DD073EF52FAC032828BF002001F0AAFA02
:104DF80001231A46FEF728BC134B1B78D8073EF54B
:104E080021AC02F07FF801F095FC01231A46FEF769
:104E18001BBC0D4B1B78DA073EF514AC1A490A780F
:104E2800012342F004020A701A46FEF70DBC064B35
:104E38001B78D9073EF506AC144A4FF4C871012314
:104E480011801A46FEF700BC2F560020C0760020BD
:104E5800901E0020082F0020C4370020D4370020DF
:104E680018520020F44F002024410020AC7E030893
:104E7800BC370020E0460020AD3D00201C2D00205E
:104E8800482E0020C2210020F4770020204700206F
:104E9800092A7FF794ABCF4F3346721C3D68C8F898
:104EA800002013F8022B2A70C8F800307378AB7012
:104EB800F31CC8F80030B378642BA8BF6423321DF4
:104EC8006B71C8F80020F378642BA8BF6423721DA7
:104ED800AB71C8F800203379EB71B31DC8F8003006
:104EE8007379642BA8BF6423F21D2B72C8F80020C5
:104EF800B379EB7006F10803C8F80030F3792B7129
:104F08004046FDF729F8D8F80420D8F80030688121
:104F1800D11A00290DDD591C3868C8F80010521A3A
:104F2800002A1978417204DD9A1CC8F800205B78C1
:104F3800437020F05FFE01231A46FEF785BBA64B9F
:104F48001868F31C02462136991EC8F8001013F899
:104F5800031C1170591EC8F8001013F8021C517078
:104F6800C8F8003013F8011C91700333B34202F102
:104F78000302E9D127F052FCFEF764BBC2F34705F0
:104F8800122D3FF61CABBDB10EAB0DF1120703EBB2
:104F980045093E46A9F126094046FCF7DDFF26F8FB
:104FA800020FB145F8D18D4B37F8022F23F8022FA5
:104FB800BE42F9D1112D09D8894A6B00023B13442E
:104FC8000021223223F8021F9A42FBD1854901228F
:104FD80013460A70FEF738BB731C8349C8F80030C3
:104FE8000A783378002A00F0E985042A7EF42AAB8F
:104FF8007E4A9B00138002F0BDFC7D4A012390612C
:105008001A46FEF721BB7B4D002340462B60FCF778
:105018008BFF012328601A46FEF716BB3346721C25
:10502800C8F8002013F8025BC8F80030F31C707849
:10503800C8F80030B178002D00F0DC85012D7EF431
:1050480001AB1EF057F82B462A46FEF7FDBA731C33
:10505800C8F800303378002B00F0A7854FF40040E3
:105068002AF0BEFE01231A46FEF7EEBA731CC8F8F2
:105078000030594D604F33787B7140462E68FCF7FD
:105088006BFF308440462E68FCF766FFD8F8042092
:10509800D8F80030F083D11A072900F39385D11A84
:1050A800032900F32786D21A002A06DD591C2A682C
:1050B800C8F800101B7882F8263001F09DFA22F01B
:1050C80069FD4E4B28681B68002B00F0638527F0AC
:1050D8000DF801231A46FEF7B7BA3346721CC8F812
:1050E8000020474A13F8021BD170C8F80030454A1F
:1050F80073785371F31CC8F80030434BB278DA70F8
:1051080001231A46FEF7A0BA404B1B68002B3EF459
:1051180099AA1EF00DFFFF283EF494AA4046FCF71A
:105128001BFF3F2840F2F485394E00253570D8F82A
:105138000030D8F80420B080D21A012A7EF782AA5B
:105148001A46591CC8F8001012F8021BB1700EA8B4
:10515800C8F8002000225D7800F8242D1EF0BAFE61
:105168009DF81430AB423EF46DAA28461EF0D6FED8
:10517800FEF768BA274B1B78012B3EF663AA324626
:10518800731CC8F80030244D12F8023BAB70F31CB6
:10519800C91AC8F8002001297278C8F8003040F30D
:1051A8002F854046FCF7D8FE012328801A46FEF7D3
:1051B8004BBA1A4B1B7813F001017FF400AA731C39
:1051C800C8F8003030781DF0CFFE01231A46FEF7EC
:1051D8003BBA00BF2841002024410020363300207C
:1051E800383300205C3300200A3C0020147800206B
:1051F800901E0020F42F0020F44F0020E03C0020F7
:10520800C43700202C7A0020D437002034560020E0
:10521800385600204C820020F67700202F560020B8
:105228003346721CC8F80020CD4F13F8022BBA7011
:10523800C8F80030CB4A73781370F31CC8F80030F4
:10524800C94DB3782B71331DC8F80030F378092B9A
:10525800A8BF09234046AB70FCF77EFED8F80030A3
:10526800D8F804202880D11A012907DD4046FCF728
:1052780073FED8F80030D8F80420E8819A4240F04C
:10528800248501F0B9F9D8F80030D8F804209A42FA
:105298003EF4D8A95A1CC8F800201B78EB700123EB
:1052A8001A46FEF7D1B94046FCF756FE4046FCF7D1
:1052B80053FE4046FCF750FE4046FCF759FED8F82E
:1052C8000030AA4D1946581C2A68C8F8000011F881
:1052D800020B82F82C00C8F80010597882F83610B2
:1052E800D91CC8F800109B7882F837304046FCF784
:1052F8003FFE4046FCF73CFE4046FCF739FE404680
:105308002E68FCF729FE708740462E68FCF724FEBD
:10531800D8F80030D8F804203087D11A01290DDDDB
:10532800591C2A68C8F800101B7882F82E304046AD
:10533800FCF71EFED8F80030D8F80420D31A032B47
:1053480009DD40462E68FCF707FE708640462E6849
:10535800FCF702FEB08628680CE6731CC8F800301B
:105368003778112F3FF62BA9B31CC8F80030804DB1
:10537800737805F817304046FCF7EEFD40F6CA038F
:105388009842A8BF184640F2EE23984205EB47051D
:10539800B8BF18460123A0F2EE211A46192091FB46
:1053A800F0F16970FEF750B93346721CC8F8002056
:1053B800704D13F8022B2A71C8F8003073786B719E
:1053C8004046FCF7C9FDD8F8003028805A1CC8F8B8
:1053D80000201B78AB714046FCF7BEFDD8F80030C2
:1053E80068805A1CC8F800201B78EB7101231A4604
:1053F800FEF72AB9731CC8F800305F4B32785F4F4C
:105408001A7000233B604046FCF78EFDD8F8002058
:105418003B685B495B4D0343501C3B60C8F8000088
:1054280013780B724046FCF797FD28604046FCF75E
:1054380093FD68604046FCF78FFDA8604046FCF786
:105448008BFD4046FCF788FDFEF7FCB84E4B06F195
:1054580008020136C8F8006016F8011C03F8011F9D
:10546800B242F6D1FEF7EEB83346721CC8F80020F7
:10547800464A13F8020B9070C8F8003070785070E4
:105488008B423EF4DFA8F31CC8F80030404BB278DA
:105498001A7101231A46FEF7D7B8731CC8F80030F2
:1054A80033780E2B3FF68BA8B21CC8F80020707812
:1054B80003283FF684A83749062202FB03F28B181B
:1054C800F51C5871C8F80050B0788854321DC8F8D7
:1054D8000020F2785A70721DC8F8002032799A704C
:1054E800B21DC8F800207279DA70F21DC8F80020E1
:1054F800B2791A7101231A46FEF7A6B8731CC8F8C8
:10550800003035781F2D3FF65AA8052A7FF457A892
:105518004046FCF709FD204B43F825001EF064FACD
:1055280001231A46FEF790B81B4D05F14006404688
:10553800FCF712FDD8F80030A5F88000591C1A466F
:10554800C8F8001012F8021B85F88210C8F800206D
:105558005B7885F883300435AE42E8D1FEF772B83F
:10556800F44F0020B83700201852002024410020B2
:105578008C350020FC460020F83C00205C8200208E
:10558800E07A0020202B0020DF7A0020E43700207A
:10559800901E00200030002040470020731CCA4D98
:1055A800C8F8003033782B724046FCF7D5FCA88346
:1055B8004046FCF7D1FC28834046FCF7CDFCD8F8E0
:1055C80000206883531CC8F800301278EA74D8F8B1
:1055D8000420D31A032B00F35383D8F80030D11AD0
:1055E800052900F31983D21A002A7EF72BA85A1C22
:1055F800C8F800201B7885F8213001231A46FEF7E9
:1056080023B8731CC8F80030B04832780270C91A41
:1056180000297EF717A8B31CC8F80030727800324A
:1056280018BF0122012342701A46FEF70DB8404602
:10563800FCF792FCA64D28604046FCF78DFC68609C
:105648004046FCF789FC0123A8601A46FDF7FCBF19
:10565800A04D00232B604046FCF766FC2A68012316
:1056680002432A601A46FDF7EFBF731CC8F80030E2
:105678003578132D3EF6A3AFB31CC8F80030707808
:105688002CF0E4FB00283EF49AAF934B027803F821
:105698002520F21CC8F8002003EB8505B2786A7053
:1056A800321DC8F80020F278AA70721DC8F80020D0
:1056B8003279EA7003F1500202E004339A4208D0CA
:1056C80019780029F9D19878D9788842F5D24FF01D
:1056D8000109824A89F00109012382F800901A46DB
:1056E800FDF7B2BF7E49102A13464FF0000228BFCB
:1056F80010230A604A608A60CA600A74002B3DF46D
:10570800A1AFD8F80020013913440132C8F80020AD
:1057180012F8010C01F8010F9A42F6D1FDF792BF79
:10572800731CC8F80030684B32785A75FDF78ABF89
:1057380023685A1C2260197029882046FCF74EFC01
:105748002368EA78591C21601A7023682A79591C41
:1057580021601A702368AA79591C21601A7023687D
:105768006A79591C21601A70FEF73FBCDFF894A1D2
:105778004FF000084FF0A80908F10108C8F120020D
:1057880009FA02F2A8F120032AFA08F6164329FAC0
:1057980003F31E43B8F1280F06F001024FF000038F
:1057A8000CD01343E8D05FFA88F020F0BFF9002846
:1057B800E2D0414605A8FCF787FFDDE7494B1B7897
:1057C800DA0700F1EB800026474FB04602E00136C9
:1057D800282E0ED031463846FCF786FF0028F6D032
:1057E800314605A8FCF780FF00285ED108F10108C2
:1057F800EDE73E4B3E4EB3F850102046FCF7EEFB6B
:105808003C4B1988204689B2FCF7E8FB3A4B1A68EA
:10581800530103F02001C2F340030B43C2F380019C
:1058280043EA4103C2F3C00143EA8103C2F34011D2
:1058380043EAC10102F0100211432046FCF7CEFBF7
:1058480003A904222046FCF799FB236831782B4AE8
:10585800581C2060197011886429A8BF642120464B
:10586800FCF7BCFB962D00F0A48000212046FCF735
:10587800B5FB2168B8F1190348BFA8F11203A3F3D7
:10588800C4034A1C226020461A460B7004A9FCF780
:1058980075FB23681A4A581C112120601970116879
:1058A8002046FCF783FBFDF7CDBE414603A8FCF775
:1058B8000BFF9BE7F4EEC87AF1EE10FA80F235811F
:1058C8004FF47A71FEF723BEE07A0020F83C0020FE
:1058D800202B00205C820020843400202C02002031
:1058E800464C00202F560020E08000202003002096
:1058F800574C0020142D0020C4400020182D0020F3
:105908001C41002090E33FF42368B978CD4A581C25
:105918002060197023681278591C21601A70FEF7EC
:1059280019BD0827FEF760BC5A1C1946C8F80020A4
:10593800C54811F8022B0272C8F800105B78437250
:10594800042A0BD9FF2A3DF4F1AF216800204A1C34
:10595800012322601A460870FDF776BEBB49097814
:10596800994203D8022AF0D1FF2BEED122680123F5
:10597800D11821601370BAF1000F3DF463AEB44A38
:10598800CAF800201A46FDF75FBE95F82420B14BEF
:10599800002A40F092803046FEF765BC059B43F034
:1059A800010305930FE723685A1C22601870FDF75E
:1059B80049BE23680322591C21601A702368727833
:1059C800591C21601A7054E74046FCF7C5FAA24DED
:1059D800FEF79CBE0427FEF707BCB31CC8F80030CE
:1059E8009E4B72781A70F21CC8F80020B2785A7070
:1059F800321DC8F80020F2789A70FDF723BEF4EE45
:105A0800C87AF1EE10FA3EF59FAD9FED957AF4EE67
:105A1800C77AFDEEE77AF1EE10FA17EE901A00F267
:105A2800A7806FF4F973303903FB01F140F2E733D3
:105A380091FBF3F101F2DB5189B2FEF768BDB31CAB
:105A4800C8F800307578022D3EF6B9AD4046FCF72F
:105A580083FA844A02EB45024FF0FF33A2F856005E
:105A68001A46FDF7F1BD0BEBC50A40468AF802104D
:105A7800FCF772FAD8F800302BF835001A46591C92
:105A8800C8F8001012F8021B8AF80310C8F80020A2
:105A98005A788AF80420DA1CC8F800209A788AF81C
:105AA80006201E1DC8F800600137DB788AF805302B
:105AB800B9457EF473ADFDF7C5BD5978022951D0BB
:105AC80003290CBF04203046FEF7CDBB4046FCF747
:105AD8004FFAD8F80030634D1A46591CC8F8001020
:105AE80012F8021B85F85510C8F800205B7885F875
:105AF80054304046FCF730FAA5F850004046FCF711
:105B08002BFA4046FCF728FA98E80C009B1A012B60
:105B1800A5F852007DF796AD4046FCF71DFA012323
:105B2800A5F85A001A46FDF78FBDFDEEE77A40F258
:105B3800E73317EE901A303903FB01F140F2CF73C7
:105B480091FBF3F101F2E93189B2FEF7E0BC454B74
:105B580000301D4418BF0120012385F85E001A4655
:105B6800FDF772BD042A34BF02200320FEF77BBB79
:105B780040F2F313A1F5836103FB01F140F2E7332F
:105B880091FBF3F101F2DD5189B2FEF7C0BC424648
:105B9800FDF711BF344B354A354836491A600123A1
:105BA80002600A601A46FDF74FBD33490A680123AF
:105BB80022F400420A601A46FDF746BD04220A7024
:105BC800FFF716BA4046FCF7C7F978814046FCF75C
:105BD800C3F9B88140462E68FCF7BEF97084404688
:105BE8002E68FCF7B9F9D8F80030D8F80420B0844A
:105BF800FFF755BA26F09DFC01231A46FDF724BD90
:105C08001E4BB0781988012311FB02F11A4691FB4B
:105C1800F0F12980FDF718BD5A1CC8F800201B7840
:105C2800EB724046FCF780F9D8F80030E8605A1C5F
:105C3800C8F800201B782B74D8F80030D8F8042056
:105C4800D1E400BFB8370020901E0020AD3D0020F1
:105C580085F4020810570020B4370020F580002092
:105C680000E0824488770020FC7400205D0500086D
:105C780050750020B87500201C4100200A3600200D
:105C88004046FCF769F9A8844046FCF765F9D8F85E
:105C98000030D8F80420E884D11A03297FF79FAC94
:105CA8001A46591CC8F8001012F8021BA977C8F840
:105CB80000205B7885F820304046FCF74DF9D8F88D
:105CC8000030D8F80420688489E45A1CC8F80020F9
:105CD8001B78003318BF0123FB71FFF7D2BA00F01D
:105CE8007F00032828BF00201DF020FA01231A4650
:105CF800FDF7AABC4046FCF72FF9F8814046FCF7AF
:105D08002BF9D8F80030D8F804203882FFF7CBB93F
:105D1800C50800F0070301350133EDB2034E2846EC
:105D28001946737019F012FBFFF700BA38560020B5
:105D380038B50B4C23688BB15A68821A002A05467D
:105D480004DA0CE05A68AA1A002A07DB9A6822606B
:105D580018461A6890472368002BF3D138BD38BD20
:105D6800203400200B4B002210B4027203F1DC0433
:105D7800012102E0072A09DC9979890702D51979F6
:105D8800815401329C4203F11403F3D15DF8044BB2
:105D9800704700BF388603081F230370704700BF91
:105DA80030B40123022514241521222205724470DF
:105DB8004171C27003700371837030BC704700BFBB
:105DC8002DE9F0410B78057BDB43DFB200F11302CC
:105DD80000F11D0302F8015F9342FBD1DFF890E068
:105DE80000F12701002203F8012F9942FBD1142169
:105DF8000524002647FA04F303F00103002B1E4490
:105E080014BF4FF019084FF00A0814F0010FF6B24A
:105E180014BFAC464FF0000C0023CA1810FA82F2E7
:105E28000133434582F814C0F7D15A1E92B20132A9
:105E3800013C8B18621C9BB201D01946DAE716F0B8
:105E4800010F14BF19240A240022991810FA81F1AD
:105E58000132A2420D75F8D113449BB25A1C034477
:105E6800002192B21975AEF800200261BDE8F081F8
:105E7800B81E00202DE9F04FDFF890A0BAF80230E4
:105E88000B3383B01FFA83F901F1060B4FF00108B9
:105E98004FF0000C002711F801EB3E464C4601225A
:105EA800A4F10B039BB2019105E001339BB2017B86
:105EB80029759C4208D0C518002AF6D1C5180133A7
:105EC8009BB29C422A75F6D103190136092F019914
:105ED80083F814C0F6B20CD0092E15D008FA07F3CF
:105EE80013EA0E0F14BF012200220C34A4B20137AA
:105EF800D6E709F1780959451FFA89F9CAD1AAF8EC
:105F080002C003B0BDE8F08F0022EEE7B81E002003
:105F18002DE9F047DFF85C80B8F8043004331FFA45
:105F280083FC01F109094FF0010E11F8017B644669
:105F38000026231F0EFA06F29BB23A40C2B1B0F80F
:105F48000CA0C51801339BB29C4285F814A0F5D16A
:105F580001360434082EA4B2EBD10CF1200C4945CB
:105F68001FFA8CFCE1D10023A8F80430BDE8F087C3
:105F78009246E6E7B81E002010B50168047B0A685F
:105F88000223A3401A420AD0054A4068002414702C
:105F9800026822F001021204120C02604B6010BD6C
:105FA800362300202DE9F0478C4B1B78DB0707468A
:105FB80044D58B4B8B4D1C788B4E012C59D01CD360
:105FC800022C07D189498A4A09881288914201D945
:105FD80001241C70EB7AE3B12B89D3B1854B1B7874
:105FE800BBB10BF04FFD002800F09B802B7B834258
:105FF8002CBF0121002131700CE07C497E4A0988C0
:1060080010886A7B801A8842E2DAEB7A0024002B37
:10601800E2D131782A79632A06D8022C774E00F02B
:10602800BA803378002B5DD1754AAB7A8C4238BF81
:106038000C461470002B4CD1BDE8F0876B4B694DB2
:1060480019885B88E878CB1A83EAE3728142A2EB6D
:10605800E3721DD32B788B421AD3614B1C78E01E58
:10606800012861D96749097802294FD0012C5E4E71
:10607800A5D15F4A5D491288687B0988121A914246
:1060880039DD5D4A12888A42A4D200241C70A1E737
:10609800B1EB400FE1DC524B1C78E11E012940F2C4
:1060A8009480022ADEDC57494F4E0878DFF8448195
:1060B800DFF844C1DFF838E10021032402283470F6
:1060C8001C7088F80010ACF80010AEF8001081D1F0
:1060D8001FE0012C71D0022C0BD10720BDE8F0473E
:1060E8002BF0DCBC7068381A474B984258DD727048
:1060F8009AE7BDE8F08702241C706BE7022AD2DD1C
:106108004049097802294FF0040464D13949364ED0
:1061180009783E48022ACCBF00220122C280818031
:106128004BE70221317075E7022A9BDC95F800C025
:1061380091FBFCFC0CF1010CBCF1080FDFF8B4A0DA
:10614800304EA87895F801E096F800802A4CDFF8E0
:10615800A090254EA8BF4FF0080C8AF800C01FFA7F
:106168008CFA10FB0AF01EFB0AFE80B2DFF88CA046
:106178002080A9F800E000244FF0640EB8F1020F67
:1061880034701C70CAF804408AF801E07FF439AF13
:106198000FFA8CF1BDE73078A0B90123776033702E
:1061A800C2F164021A4B00FB02F083FB0023C01704
:1061B800A0EBA3506430707036E70820BDE8F047C4
:1061C8002BF06CBC7368F81A8EE7032C96D10D4936
:1061D800097802299AD0044EFCE600BF2F56002009
:1061E800D8220020A8400020E8220020D43E002029
:1061F800DC220020EA3E0020DA220020E0220020F3
:1062080050780020CC3D00207F969800D03D00209B
:106218006BCA5F6B2DE9F0470569C3681D4028D03C
:106228000F4606464FF000484FF00009B5FA85F3CF
:1062380028FA03F2D2431B3B32611540042B16D8CF
:10624800DFE803F03129211903007B6A002B32D0E3
:1062580003F1FF3A1FFA8AFAC7F824903C6A34B16E
:1062680023682046514698476468002CF8D1002DD1
:10627800DCD1BDE8F0873868716B036889B298474C
:10628800002DD3D1F5E77868B16B036889B29847D8
:10629800002DCBD1EDE7B868F16B036889B2984758
:1062A800002DC3D1E5E7F868316C036889B29847D7
:1062B800002DBBD1DDE7F36A1FFA83FACEE700BFF2
:1062C8001C4C08B5012102200AF0A2FD237803F036
:1062D8000502052A2AD003F00903092B08D000215A
:1062E80001200AF095FD002108460AF091FDFEE71D
:1062F800114A124B11681A680B68114C4FF6FE7060
:1063080003400B601388206823F001031B041B0C57
:10631800138018B12A2200238271C37102224E21F0
:106328000AF0D2F920680AF05DFDD8E71EF006FFF2
:106338002378D0E7F02A00204023002044230020BF
:106348003C2B0020022828BF022010B4084C094B1F
:10635800207000EB8002C0EBC20207495DF8044BD5
:10636800013003EB4203C0B20B602BF07DBC00BFD1
:10637800574C00200A8100202441002008B512F063
:106388004BFFFBF72DFBBDE8084012F02DBF00BF07
:106398002DE9F04F013085B0C3B203938E4D8F4F76
:1063A8008F4C904E0A2302933220DFF8409226F059
:1063B800EBFF4FF4FA7A4FF0100C4FF47A70D9F8DB
:1063C8000430C3F30803002B40F0C880EFF31183B7
:1063D800002B40F0C3802968A26800BF2B6899424F
:1063E800F9D1D7F800E000FB0EF39B1AB3FBFEF3DC
:1063F80000FB01314FF0010E0191D9F80430C3F3CD
:106408000803002B40F08E80EFF31183002B40F03F
:1064180089802B68A16800BF2A689342F9D1D7F810
:1064280000B000FB0BF2521AB2FBFBF200FB032395
:10643800019A9B1AB3F57A7FDFD3BAF1010ABED16C
:10644800039B002B40F0C4804FF47A7ADFF89C91CC
:1064580050464FF0100CD9F80430C3F30803002B52
:1064680040F09980EFF31183002B40F09480296865
:10647800A26800BF2B689942F9D1D7F800E000FB69
:106488000EF39B1AB3FBFEF300FB01314FF0010E34
:106498000191D9F80430C3F308033BBBEFF3118330
:1064A80023BB2B68A16800BF2A689342F9D1D7F8AB
:1064B80000B000FB0BF2521AB2FBFBF200FB032305
:1064C800019A9B1AB3F57A7FE3D3BAF1010AC2D1D4
:1064D800029B013B02937FF467AF4349434B444817
:1064E800444A0860DA6005B0BDE8F08FEFF3118820
:1064F8008CF31288A1682368DB0344BFC6F800E068
:10650800A1682B6832685FFA88F888F31188D7F891
:1065180000801A4400FB08F35B1AB3FBF8F300FB96
:106528000233CDE7EFF311888CF31288A168236852
:10653800DB0344BFC6F800E0A1682B6832685FFA45
:1065480088F888F31188D7F800801A4400FB08F30C
:106558005B1AB3FBF8F300FB023369E7EFF3118230
:106568008CF31288D4F808E02368D90303D50123F3
:106578003360D4F808E02B683168D2B282F311880E
:106588003A68194400FB02F3A3EB0E03B3FBF2F3E2
:1065980000FB01312EE7EFF311828CF31288D4F857
:1065A80008E02368D90303D501233360D4F808E051
:1065B8002B683168D2B282F311883A68194400FB1B
:1065C80002F3A3EB0E03B3FBF2F300FB01315DE72B
:1065D800184626F049FD37E7C0760020C47600202B
:1065E80010E000E0BC760020FC9F002000ED00E0F9
:1065F800EFBEADDE0400FA0538B5434B5A899989D8
:10660800914224BF00225A81198ADA89914224BF13
:106618000022DA81DA788AB3072A2FD03B493C4D29
:1066280091F85300012400210A282C709C70D9711C
:106638003DD00C2865D0DFED377A8ABB364C9FED0C
:10664800370AA278002918BFF0EE407A062A04D843
:10665800334901EB820191ED000A217959B3013ADE
:10666800032A4DD8F7EE007A87EE800A2EF07CFCDC
:106678002388984228BF1846208038BDD97921B18F
:1066880098780428B8BF04209870204890F85300E0
:106698000A280CD00C28CED1DFED227A002ACDD0E2
:1066A800072ACBD00A282CD1DFED1F7AC6E70A20AB
:1066B800DFED1E7AC1E79B78154A07EE103A11788C
:1066C800B8EEC77A27EE277A07EE901AF8EEE77A3F
:1066D80067EE877AB4EEE70AF1EE10FA10DDC0EE45
:1066E800077AFDEEE77A17EE903A102BA8BF102331
:1066F800012BB8BF0123DBB28B4238BF0B461370A6
:1067080038BDDFED0B7A99E7F44F00207C4D00206F
:10671800B83700206F120339185200206F1203385F
:10672800B46003080AD7A3390F506E3A5304E93806
:106738006F12833A2DE9F047A84FA94E12F06CFD6D
:10674800BE421ED2DFF81483DFF81493444625882E
:1067580062197DB14A450DD2052D0BD93388618860
:10676800C3F30B03994200F0DD80144625886219B3
:10677800002DEFD17168304614360AF086FFBE420C
:10678800E4D3984A1378A3F1170102290FD996493F
:1067980011F83300002840F0F180D800014449780E
:1067A80029B1924911F83330002B00F00F81904B3A
:1067B8005A78022A40F2DC8000228E495A701A78F0
:1067C8008D48022A016000F2CF8002EB82018B4BD8
:1067D800C2EBC10203EB4203998C5A8C884C91425C
:1067E800236001D300225A84864B9A78042A00F049
:1067F800E48032B91A88B2F5F07F84BF4FF4F072A2
:106808001A80814DFFF7F8FE2B68804A1A40002A4B
:1068180000F0DF80D80700F1CB80590400F1C38075
:106828001A0700F1BB809B0400F1B1802AF0DAF965
:1068380010B977482AF010FE40200AF05DFF80204A
:106848000AF05AFF4FF400700AF056FF4FF4003078
:106858000AF052FF4FF000700AF04EFF4FF08060D0
:106868000AF04AFF1FF0C6F90021302269482FF0CC
:1068780038FB206825F07AFE674B276803F1500142
:1068880002E0043399426DD01A78002AF9D19C7835
:10689800D8788442F5D26149614B0D7961496248E3
:1068A8000A70624E624C8460C822642111FB052183
:1068B800002259609A60DA601A615A619A61DA6155
:1068C80083F8202083F82120376016F0CDFC594B3F
:1068D8009FED595A1B88594A9FED596A5079594971
:1068E80006EE903AF8EEE66A1388C5EE265A07EEE9
:1068F800103A53881279C1ED005A07EE903AB8EE73
:10690800C77A514BF8EEE77A18725A7227EE067A70
:1069180067EE867ABDE8F04783ED017AC3ED007A29
:1069280012F062BC63799B077FF41FAF716894F81B
:1069380004A030460AF0A9FE3388BAEB133F04D00E
:106948001436BE42FFF402AF1BE773887068AA1FB3
:10695800C3F30B039A4204F10601A8BF1A462EF0AE
:106968002FF9EDE7012296E700221A70234B33E74F
:10697800204902EB420201EB820120E7D8000C1803
:106988006468002C7FF40AAF1724147006E72F48B8
:106998000AF0B2FE40200AF0AFFE47E72C480AF0A2
:1069A800ABFE2B683FE72B480AF0A6FE2B6837E7BB
:1069B80029480AF0A1FE2B682FE79A8AB2F57A7F58
:1069C800BFF41FAF4FF47A729A821AE71823137034
:1069D800EDE643F001032B601CE700BF34C6030853
:1069E800C0C10308F83C0020B0800308888403086D
:1069F800574C002016820020284100200A810020E0
:106A080024410020185200205C8200200960000206
:106A18000C7B0020D81F002084340020FC46002076
:106A2800EC4800202C020020B81E00200C2000207A
:106A3800CA370020C4210020C0C9FB48901E00208E
:106A480017B7D138C8210020384600200940000275
:106A580001600002092000020860000202F0030839
:106A68000000040808B512F0D7FBFAF7B9FF12F0D6
:106A7800BBFBFFF75FFE0120BDE808402BF0F4B830
:106A88002DE9F047B54C82B0636820469847002846
:106A980000F0BF80B24B1B780122042B84F83C2005
:106AA80000F0BA80B4F91610B4F91820B4F91A3005
:106AB80021636263A363AB4B1B88002B69D0AA4D8B
:106AC800D4ED0C7AD5ED004A95ED050A95ED015AFD
:106AD80095ED067AD5ED035A95ED026AF8EEE76A68
:106AE800D5ED047AA4EEA60AA5EE267A67EEC07A5A
:106AF800A5EEC07AE6EE267A85ED057AC5ED067A2A
:106B08002EF032FAD4ED0D6AD5ED094A95ED0E0A4C
:106B180095ED0A5A95ED0F7AD5ED0D7AD5ED0C5A0B
:106B280095ED0B6A2063F8EEE66AA4EEA60AA5EED8
:106B3800267A67EEC07AA5EEC07AE6EE267A85ED6B
:106B48000E7AC5ED0F7A2EF00FFAD4ED0E6AD5ED58
:106B5800124A95ED170A95ED135A95ED187AD5ED69
:106B6800167AD5ED155A95ED146A6063F8EEE66A63
:106B7800A6EEA40AA6EE857A67EEC07AA0EE657A3C
:106B8800E6EE867A85ED177AC5ED187A2EF0ECF9DF
:106B9800A063764FA17F764816F0E8FA3B88002B71
:106BA8007CD1744EB568744B1B685B0742D4B5F949
:106BB8000070216B636BA06B704A714E92ED026A94
:106BC800D2ED006AD2ED015AC91B2163B5F90270F2
:106BD800DB1B6363B5F904703568C01B07EE900AC8
:106BE800B8EEE75A07EE901AB8EEE77A07EE903A51
:106BF800F8EEE77A36EE056A36EE877A77EEA57A0A
:106C08000135A06382ED026A82ED007AC2ED017A55
:106C1800356002B0BDE8F0875A4BB4F91600B4F9F4
:106C28001810B4F91A2018802063598061639A807B
:106C3800A26340E7544F3B88322B7ED0002B5BD1B8
:106C480052480378002BB2D0DFF848E1716AB26A83
:106C58008EFB01730027C9170770C1EB23118EFB48
:106C68000203D217C2EB2312F36A29806A80A08A32
:106C780047498EFB03E2DB17C3EB22131B1AAB80D9
:106C8800CF6012F0C9FAFAF7ABFE12F0ADFAFFF7CF
:106C980051FD01202AF0E8FFB56888E7354E226BE0
:106CA800B568B3F5C87F4FF0000323632B8039889C
:106CB80018BFF068B7F8008008BF0020B1F5C87F9A
:106CC80018BF3369616B02440B440020B8F5C87FD4
:106CD8006063F260336168803AD0D4F838E0716953
:106CE800A0637144B8F1010FA880716154D008F114
:106CF800FF38A7F8008056E7716A226B00232363E8
:106D08002B80B7F800E00A44BEF1320F616B636371
:106D18006B807262A26B6BD0F06A0190B06AA36359
:106D280001440198B1620244BEF1010FAB80F262E6
:106D380063D00EF1FF333B8082E7154B2988D86872
:106D48006A88AB88318330627283B3830021D4E7C9
:106D5800A36B7361A063A880C9E700BFD840002077
:106D6800CC3D00202438002028380020204700206F
:106D780008410020B81E0020185000202C46002092
:106D880028460020D03D0020D41F0020D11F00201D
:106D9800C43700201F85EB51DFF80CC1DFF8F8E09D
:106DA800C8328CFB02A9C833D217C2EBE9128CFB9C
:106DB80003A9DB17C3EBE913C8316B802A808CFB6E
:106DC800013CA28ACB17C3EBEC139B1AAB80CEF81D
:106DD8000C0012F021FAFAF703FE12F005FAFFF799
:106DE800A9FC40462AF040FFB7F80080B5687EE766
:106DF800A363B162F262AB809BE7234A234812681F
:106E08002349037012F4003281F800E032D11346AE
:106E18002049C85C0B2803F10C030ED00132182A54
:106E2800F7D1338B2B80728B1B4B6A80B18B326A04
:106E3800A980B7F800E0DA607BE71848D0F800C00E
:106E48005300BCF1000F09D003EB020E01EB8E0ECC
:106E58009CF801C09EF801E0E645E2D21344DFF851
:106E68004CE00F4A01EB830100230160AEF80030CB
:106E78001360D6E70B4A1278032A01D01A46C7E7EF
:106E88002AF0F0FDB568CCE7F42F0020D61F0020CB
:106E9800D01F0020DC750308C437002040210020E3
:106EA8002C220020507800201F85EB51282200203A
:106EB80038B50D4C0D4DAC4206D2616820461434ED
:106EC8000AF0E3FBAC42F8D3FBF71CFC084A094B79
:106ED800094C1460002209491A705A700848086061
:106EE800BDE838401CF080BDC0C1030834C60308A3
:106EF80024410020574C00200A810020284100200E
:106F08001682002008B5FFF7D3FF12F085F9FAF7CB
:106F180067FDBDE8084012F067B9054B10B51A6B5C
:106F2800044C2178501C09B91A6310BD0246F8E7D1
:106F3800B81E002036230020F0B50C292BD8DFE836
:106F480001F06F2A2A2A4C2A2A2A2B2A2A2A0700E1
:106F5800046AB2F80CE097881668674D24F48054E8
:106F68000462036A4468C16923F4005343EA0E3398
:106F780021F4E641A84243EA073341EA062100F03A
:106F8800B58005F50065A84200F0B08092684460BD
:106F9800C16102640362F0BD046A96899588D2F8DB
:106FA80000E0554F24F480740462036A4468C169A0
:106FB80023F4007343EA062321F07301B84243EA3D
:106FC800052341EA0E017ED04C4DA8427BD0926841
:106FD8004460C161C2630362F0BD046A9689958802
:106FE800D2F800E0444F24F010040462036A4468B5
:106FF800816923F0200321F0807143EA061321F40C
:10700800E641B84243EA051341EA0E2148D03B4D18
:10701800A84245D092684460816182630362F0BDF2
:10702800046A9389B2F804E01768334E24F0010427
:107038000462056A4468816943EA0E0321F48031D9
:1070480025F002059BB221F07301B04243EA050323
:1070580041EA070114D0294DA84211D005F5406531
:10706800A8420DD005F58065A84209D005F58065D0
:10707800A84205D092684460816142630362F0BD12
:10708800D689158A578A23F0080333433D43D688A7
:1070980024F4407423F00403ADB233432C43E9E7EE
:1070A800D589178AD68823F0800343EA051324F488
:1070B8004064558A23F0400344EA870443EA0613F0
:1070C80044EA8504A6E7D589178AD68823F400639D
:1070D80043EA052324F44054558A23F4806344EAA0
:1070E800071443EA062344EA051470E7158A24F4D2
:1070F800804444EA851449E7002C014000340140EB
:107108002DE9F04FF022002183B07848784CDFF861
:107118000492784D784E794FDFF8FC812EF0E1FE2D
:1071280077487849DFF8F4E1DFF8F4C10022135911
:10713800834200F0C180B3F1804F00F0BF80AB42C2
:1071480000F0C880B34200F0C780BB4200F0C680A0
:10715800734500F0C580634500F0C480434500F0E6
:10716800C380DFF8C0A153457ED00AF5806A534535
:1071780008BF092379D01432F02AD8D15C4C624D6B
:10718800624E604F04F1F00802E01434A04568D064
:10719800A379002BF9D023794FEA131909F1FF39A4
:1071A800B9F1050F03F00F03EFD835F8190040FACD
:1071B80003F2D207E9D54FF0010A0AFA03F3013BBB
:1071C80018402DF07BFA16F809305149184411EB94
:1071D800C002DAD051F83000DFF84CE1217A00F132
:1071E80038439B0A1EF8033003F01F0E5B09022B7D
:1071F8000AFA0EFA69D0032B62D0012B03D17B69FE
:107208004AEA03037B6193880093B3FA83F3C3F1DB
:107218001F039BB2DA0800EB820203F00703D2F8DF
:1072280020E09B004FF00F0C0CFA03FC2EEA0C0E2A
:10723800C2F820E0D2F820E001FA03F343EA0E0393
:10724800136269460023022214348DF804208DF855
:1072580005308DF806308DF8073022F0A3FCA045E4
:1072680096D103B0BDE8F08F082309EBC3034FF0B4
:10727800010B93F820A00AF01F034FEA5A1ABAF13B
:10728800020F0BFA03F30BD0BAF1030F0ED0DA4555
:107298007FF471AFD1F814A043EA0A034B616AE79F
:1072A800D1F818A043EA0A038B6164E7D1F81CA05F
:1072B80043EA0A03CB615EE70023D6E70123D4E75C
:1072C800FB694AEA0303FB619DE7BB694AEA0303DA
:1072D800BB6198E70223C8E70323C6E70423C4E792
:1072E8000523C2E70623C0E70723BEE79041002035
:1072F80038860308000400400008004000100040E1
:10730800002C0140001002404888030854880308F4
:10731800F87E0020B46003080040014000140040DB
:1073280000340140004401405C88030801490248D8
:10733800FEF770BF3042002000400140014902487A
:10734800FEF768BF084200200034014001490248A6
:10735800FEF760BF0842002000340140014902489E
:10736800FEF758BFE04100200004004002494FF0FA
:107378008040FEF74FBF00BFB841002010B5064C53
:1073880006482146FEF746FF04F1C8010448BDE857
:107398001040FEF73FBF00BF90410020002C014085
:1073A8000044014001490248FEF734BF90410020E3
:1073B800002C01402DE9F04104684E4DA30AAB4270
:1073C8007AD00AD94C4DAB425FD00135AB4277D069
:1073D800043DAB425DD0BDE8F081B3F5801F67D0B6
:1073E8004A3DAB4259D14FF0700E022647794FEA19
:1073F800970C002968D0B000634685190227D4F895
:107408000C809F400CEB4503BFB23C4D03F1040CCC
:1074180047EA080745F8231045F82C20E760EFF302
:107428001181502282F31288821905EBC202136976
:10743800002B34D013620433821905EBC20257695A
:1074480017B11F6053690433821905EBC2029769AB
:1074580017B11F6093690433821905EBC202D7691B
:1074680017B11F60D36904330027CAB21F6082F3C3
:107478001188304405EBC000036A9BB9E3684FF6F6
:10748800FE721340E360BDE8F0814FF0C00E0426A1
:10749800ACE74FF0980E0326A8E7BDE8F08105EBAE
:1074A8000E03C9E7E36843F00103E360BDE8F08138
:1074B8004FF0480E012699E74FF0200E002695E779
:1074C8004FF0E80E052691E7BF08022306FA03F0FD
:1074D800BB40DB43E768094D9BB23B4087190CEB87
:1074E800470CE3600CF1040345F82C1045F8232001
:1074F80095E700BF4B00100050001000904100209D
:1075080030B503685C4D18885C4CB4FBF2F2013965
:10751800013AAB4294B283B089B282B266D058487D
:10752800834263D0B3F1804F60D0A0F59830834296
:107538005CD000F58060834258D0524883425BD0CB
:1075480000F5806083427DD022F4407200F58C30D3
:1075580092B283421A80D9621C850ED0484A93425F
:107568000BD002F54062934207D002F58062934245
:1075780003D002F58062934201D100221A860122CB
:107588005A611A883C4992B242F001028B421A8031
:1075980062D0B3F1804F61D03B4A934260D002F58C
:1075A800806293425ED002F5006293425CD002F59D
:1075B800806293425AD002F59032934258D002F535
:1075C8004062934256D002F5806293421ED002F583
:1075D8008062934208BF092219D002A84FF0012304
:1075E80040F8043D22F0A8FA03B030BD254822F047
:1075F8007002834292B2A3D101201A80D9621C85FD
:1076080058611A8892B202431A80C5E708221F4BB4
:1076180003EBC20301A893F821408DF8044001232D
:1076280000228DF805308DF807308DF8062022F0FD
:1076380083FA1B2CD8D1164B019301A822F07CFAAF
:1076480003B030BD01201A80D9621C8558611A88A0
:1076580092B202431A809CE70022D8E70122D6E7BB
:107668000222D4E70322D2E70422D0E70522CEE79C
:107678000622CCE70722CAE7002C014000A24A04F0
:10768800003401400010004000040040B4600308CA
:1076980019010001204B98422DD0B0F1804F2CD019
:1076A800A3F5943398422AD003F58063984228D0F2
:1076B80003F50063984226D003F58063984224D0EE
:1076C80003F59033984222D003F54063984220D0C6
:1076D80003F58063984207D003F58063984208BF9A
:1076E800092202D00020704708220C4B03EBC2038A
:1076F80093F8200070470022F7E70122F5E70222FD
:10770800F3E70322F1E70422EFE70522EDE706227B
:10771800EBE70722E9E700BF002C0140B46003084B
:107728002DE9F04F013085B0C3B203930B460291A7
:107738008B4C8C4E002B00F09A8032208A4D8B4F58
:10774800DFF82C9225F020FE4FF4FA7A4FF0100C57
:107758004FF47A70D9F80430C3F30803002B40F0D3
:10776800DE80EFF31183002B40F0D9802968A268EE
:1077780000BF2B689942F9D1D7F800E000FB0EF35F
:107788009B1AB3FBFEF300FB01314FF0010E019190
:10779800D9F80430C3F30803002B40F08780EFF3D7
:1077A8001183002B40F082802B68A16800BF2A68F3
:1077B8009342F9D1D7F800B000FB0BF2521AB2FB92
:1077C800FBF200FB0323019A9B1AB3F57A7FDFD300
:1077D800BAF1010ABED1039B002B40F0BD804FF4E3
:1077E8007A7ADFF88C9150464FF0100CD9F80430B3
:1077F800C3F30803002B75D1EFF31183002B71D16C
:107808002968A26800BF2B689942F9D1D7F800E02F
:1078180000FB0EF39B1AB3FBFEF300FB01314FF0A4
:10782800010E0191D9F80430C3F3080313BBEFF339
:107838001183FBB92B68A16800BF2A689342F9D16C
:10784800D7F800B000FB0BF2521AB2FBFBF200FBB8
:107858000323019A9B1AB3F57A7FE3D3BAF1010A9D
:10786800C4D1029B013B0293002B7FF466AF05B0A5
:10787800BDE8F08FEFF311888CF31288A1682368B4
:10788800DB0344BFC6F800E0A1682B6832685FFAE2
:1078980088F888F31188D7F800801A4400FB08F3A9
:1078A8005B1AB3FBF8F300FB0233D2E7EFF311885E
:1078B8008CF31288A1682368DB0344BFC6F800E094
:1078C800A1682B6832685FFA88F888F31188D7F8BE
:1078D80000801A4400FB08F35B1AB3FBF8F300FBC3
:1078E800023370E7EFF311828CF31288D4F808E0C2
:1078F8002368D90303D501233360D4F808E02B6843
:107908003168D2B282F311883A68194400FB02F355
:10791800A3EB0E03B3FBF2F300FB01317FE7EFF3B8
:1079280011828CF31288D4F808E02368D90303D5B0
:1079380001233360D4F808E02B683168D2B282F3AF
:1079480011883A68194400FB02F3A3EB0E03B3FB5A
:10795800F2F300FB013118E7184625F085FB3EE7F6
:1079680010E000E0BC760020C0760020C47600203D
:1079780000ED00E0204B5B68C3F3080330B4BBB9EB
:10798800EFF31183A3B91D4B1D4C1868A16800BF04
:107998001A689042F9D11B4B1C684FF47A7202FBAB
:1079A80004F3591AB1FBF4F130BC02FB0010704724
:1079B800EFF31182102383F3128811498C680B6846
:1079C80013F4803F104B02D0012018608C680B49DB
:1079D800D2B20D68186882F311880A4B19684FF4FF
:1079E8007A72284402FB01F31B1B30BCB3FBF1F392
:1079F80002FB0030704700BF00ED00E0C0760020B9
:107A080010E000E0C4760020BC7600202DE9F84F95
:107A18008046FFF7AFFF254E2549DFF8A0E0254A4D
:107A2800254D844610274FF47A740120DEF804307F
:107A3800C3F30803D3B9EFF31183BBB90B68D2F8CA
:107A480008A000BFD1F800904B45F7D1D6F800B098
:107A580004FB0BF9A9EB0A09B9FBFBF904FB039337
:107A6800A3EB0C034345E1D3BDE8F88FEFF3118A8C
:107A780087F31288D2F808B01368DB0344BF286084
:107A8800D2F808B00B68D5F800905FFA8AFA8AF342
:107A98001188D6F800A0994404FB0AF3A3EB0B0362
:107AA800B3FBFAF304FB0933DAE700BFC47600201E
:107AB800C076002010E000E0BC76002000ED00E079
:107AC8002DE9F04FDFF830C1474A4849484E494D43
:107AD8008046102718F1FF38C0F08480DCF80430A5
:107AE800C3F30803002B5CD1EFF31183002B58D1AB
:107AF8000B68946800BF08688342F9D1D6F80090F3
:107B08004FF47A7000FB09FEAEEB040EBEFBF9FEE3
:107B180000FB03EEDCF80430C3F308034FF47A7477
:107B28000120FBB9EFF31183E3B90B68D2F808A081
:107B380000BFD1F800904B45F7D1D6F800B004FB50
:107B48000BF9A9EB0A09B9FBFBF904FB0393A3EBB7
:107B58000E03B3F57A7FBDD2DCF80430C3F3080313
:107B6800002BDFD0EFF3118A87F31288D2F808B020
:107B78001368DB0344BF2860D2F808B00B68D5F857
:107B880000905FFA8AFA8AF31188D6F800A099441F
:107B980004FB0AF3A3EB0B03B3FBFAF304FB09336F
:107BA800D5E7EFF3118487F31288D2F808901368A9
:107BB800D80303D501232B60D2F808900B682868F6
:107BC800E4B284F31188D6F800A04FF47A7400EB7D
:107BD800030E04FB0AF3A3EB0903B3FBFAF304FB5C
:107BE8000E3E97E7BDE8F08F10E000E0C076002079
:107BF800C4760020BC76002000ED00E030B4EFF33E
:107C08001183102282F312880649074C0A68074834
:107C1800013200250A602560DBB2026883F311880F
:107C280030BC7047C0760020BC76002010E000E031
:107C38000F4B1B88014643B90E4B0F4A1B7810683F
:107C48000BB981F0010109F0D9B80C4B5A691AB186
:107C580018B91A68106058747047094A186811886A
:107C6800084A92FBF1F2012102605974704700BF83
:107C7800987600209A7600209C760020A076002036
:107C8800B876002020A107001D4B70B59C68236DB5
:107C9800626BDD69C2B1A36B2BB12B0702D5236DD3
:107CA80008221A6270BD2A06F7D5A26A616A8A425A
:107CB80020D0511CA069A162825C2069266D814296
:107CC8003285EAD3A362E8E7A906E4D5E26A22B1DD
:107CD800988C216B80B29047DDE7E1699B8C6069E5
:107CE800DBB24E1CE6614354E169E368994228BF60
:107CF800E261D0E7226D136823F080031360CCE7BC
:107D0800F42A00201D4B70B55C68236D626BDD6939
:107D1800C2B1A36B2BB12B0702D5236D08221A62BF
:107D280070BD2A06F7D5A26A616A8A4220D0511C22
:107D3800A069A162825C2069266D81423285EAD3FE
:107D4800A362E8E7A906E4D5E26A22B1988C216B20
:107D580080B29047DDE7E1699B8C6069DBB24E1C1D
:107D6800E6614354E169E368994228BFE261D0E7DC
:107D7800226D136823F080031360CCE7F42A0020F7
:107D88002DE9F04FBF4B1E788BB0002E40F0BC8021
:107D9800BD4BBE4C1D78DFF814A3DFF81493DFF851
:107DA800148305F00105A4F10A0B54F80A3CBBB191
:107DB800CC2707FB06B7184608F026F880B154F818
:107DC8000A0C08F019F814F8023C8BB9242831D0B1
:107DD800F5B154F80A3C184608F016F80028EED118
:107DE8000136032E04F1CC04DFD10BB0BDE8F08FCF
:107DF800012B23D0022B2BD0032B37D0042B67D099
:107E0800052B40D0062B4FD054F80A2C1346D2E746
:107E180054F80A3C23281A4600F087819C4991F8B7
:107E280022108142C7D19B4BCAF80090C3F80C803E
:107E38001346C0E7012304F8023CCAE74D2854F86A
:107E48000A2C0CBF0223002304F8023C1346B2E7B5
:107E580000233C2804F8023C45D03E28D4D1012216
:107E6800032304F8012C04F8023CB2E7C02814D814
:107E78000022042304F8050C04F8040C04F8062C6A
:107E880004F8023CA5E714F8063C14F8052C9A42BD
:107E98002FD814F8043C834203D0002304F8023C92
:107EA80097E7062304F8023C14F801ECBEF1000F32
:107EB80000F08081BEF1010F00F0C481013600237B
:107EC800032E04F8023C04F1CC047FF46EAF8CE777
:107ED80014F8043C04F8030C5840052304F8040C77
:107EE80004F8023C75E7032204F8013C04F8022C6C
:107EF8006FE714F8042CF9184240013304F8042CF5
:107F080004F8063C887264E7634B186800283FF45D
:107F18006CAF09F0F1FADFF8A0A1604DDFF89C9191
:107F2800DAF8000007F070FF00283FF45EAFDAF8D7
:107F3800000007F061FF09281BD03F2819D02B68E3
:107F4800002B66D1042800F0AC810C2800F0E680F4
:107F58007F28E5D0A0F12002D2B25E2AE0D80BB982
:107F68002028DDD05A1C09F803002A6023F0FEFA05
:107F7800D6E72C68002C5AD1494B264603F594784D
:107F8800002E08BF1E4608334345F9D1002E00F0E5
:107F98007C81A3F1080B3068DBF80020075D135DD6
:107FA8009F42204402EB040140F06D81671E4F445C
:107FB80022460BB9FD2A5CD907F8013F01322A6035
:107FC80010F8013F11F801EF9E45F2D00AB1B34510
:107FD80012D0344823F0D2FAB34508D356F8080B28
:107FE80023F0CCFA092023F0C1FA5E45F6D92E48D1
:107FF80023F0C4FA2A680024944291D2661E4E44A3
:1080080016F8010F23F0B2FA2B6801349C42F7D31B
:1080180086E70C2800F082800A2851D00D284FD01E
:108028007F2800F0FC80FF2B3FF67AAF92E71C4FC9
:108038004FF0000B07F594785E4602E00837474595
:108048000DD0224639684846F9F710FF0028F5D1C7
:10805800BB46002EF2D13E4608374745F1D1002EE7
:1080680099D1BBF1000F3FF45BAF0E4823F086FABD
:10807800B4E7511C202009F80200296009F80130F2
:108088000A46A4E7244500202F560020CA420020B3
:108098000C7B002000ED00E03C2D0020442E002049
:1080A80094630308608B0308688B0308FC9F002017
:1080B800EFBEADDE0400FA05402D0020442D00205F
:1080C80023F0D2FA23217F482DF022FF002800F068
:1080D800E680A0EB0900286088B1431E19F8031058
:1080E800202940F0EC8009EB030204E012F8011D9E
:1080F800202948D10346581E002BF7D12B604FF496
:108108008072002148462DF0ECFE6F4B1B78002B47
:108118003FF46BAE6D4823F031FA01E76C4823F069
:108128002DFA6A4823F02AFAFAE66A496A48C978B1
:108138006A4ADFF8DCE15363003118BF012101709E
:10814800674991634021D36382F8401082F8415017
:10815800644965480B603832CEF800205A4A01233A
:10816800137023F042FB594823F008FA4FF40060DB
:1081780027F036FE5D4B93F82230232B00F09780D2
:1081880014F8023C3EE62B60594C002204F5947822
:1081980009F8032002E0083444457CD021684846A9
:1081A8000FF094F80028F6D0444574D263689847D5
:1081B8000023A3E74F4BADF822E00FCB0DF1280CBD
:1081C80002AF87E80F004CF824ED14F8051C14F8EA
:1081D800033C069404EB010E624639464FF0010C4D
:1081E80006A8CDF81CE0ADF820308DF824C0FBF7C8
:1081F80019FAE8B9019F002304F8023C002F3FF464
:10820800EFAD54F80A0C29F05BF9013654F80A0C62
:10821800B847032E04F1CC047FF4C7ADE5E5013B74
:10822800002235482B6009F8032023F0A7F977E6E8
:10823800029A324B03923946A4F10A00029309F0DC
:108248002FFED7E714F8053C14F8032C06942344B2
:1082580007936E2A4FF0000308930993ADF8202086
:108268007FF42CAE06A8F9F783FE06A8F9F774FE8A
:10827800074606A8F9F770FE06A8F9F76DFE204B29
:108288001F6058601AE62246A0E61E48A3F1080BB4
:1082980023F074F9A2E61C4823F070F988E72868EF
:1082A8001AE708480EF059FC0BB0BDE8F08F174AE2
:1082B80014F8023CC2F80C80CAF80090A2E5034604
:1082C80062E700BF442D002024450020688B030886
:1082D800708B0308574C0020AC230020B81E0020E8
:1082E800C9FA0008402D00209C8B03080C7B002055
:1082F8009463030820610308988B0308FC8300201B
:108308002C230020608B03087C8B030800ED00E021
:108318003C2D00202DE9F04F2DED068BAB4BAC4AE0
:108328001C7897B000F59C41203181460B91116073
:10833800002C00F0D986A74A1268904240F2838048
:10834800A54A06921668A549A54A0591013C1C70E4
:10835800A44B049206F480560893002E40F08180C6
:10836800A14B1B78022B01F00981042B01F09D81A0
:10837800012B01F051819D4B9945089B9B7800F298
:108388008485002B40F08585994B0793069B1E68D2
:1083980016F4805740F07686DFF894A2049BB3F970
:1083A8000610059B5D8BA942B4BF00250125914BA2
:1083B8001B6813F080535ED0079A127812F00102FE
:1083C8005FD00598408C884241F3C182002D5ED170
:1083D800894C94F88C10002959D18848884900683C
:1083E80090F82D0000240C604C608C6085490028B2
:1083F8004ED10870002A4FD0F1064DD5824A127826
:10840800D20649D4002F47D1002B45D1740243D45A
:108418007E4B1B78002B02F04D827D4B9B78002D04
:1084280042F0E0823BB17B4A7B4B12681B689B1A87
:10843800002BC2F2E38210206F4C29F02FFB01239E
:1084480084F88D3028E0644B06931E68644B634AB9
:10845800049306F48056634B05920893002E3FF46C
:108468007FAF00216348FAF73FF900287FF478AF1F
:1084780019F0DAFC74E770029ED4079A127802F0B9
:1084880001025D4C002184F88C10002DA5D05D49B7
:1084980001200870002AAFD1604B1A78002A79D1E0
:1084A8000599049C488BB4F90070898BB4F9024093
:1084B800B842B4BF8026002646F04003B942D8BF70
:1084C80033469B0843F08006A042B8BF3346049F5A
:1084D80043F04006A142C8BF33469B08B7F90440A1
:1084E800B7F9066043F08007A042B8BF3B4643F0A7
:1084F8004007A142C8BF3B469B0843F080073E4C5B
:108508008642C8BF3B4643F0400794F88EE08E424F
:10851800B8BF3B469E4501F09584A4F8902084F8A6
:1085280092203A4984F88E300E78002E01F0538359
:108538005F2B01F0E3836F2B01F04984079B1B78C5
:10854800DA0727D494F8921021BBB4F99030322B73
:1085580020DD94F88E200120572A84F8920001F03B
:108568009487069B1B685F0741F1A1825A2A41F054
:108578009E8294F89430002B42F0B08194F89630A3
:1085880083F0010384F89630002B42F0F5810C202B
:1085980029F084FA224B0993224B234D0A93069B18
:1085A8001B685C0700F1EB860DF150091F4E0B9517
:1085B8000022C9F804203446149240F6330B4FF0D9
:1085C800190840F28337049D37E000BF1C340020AF
:1085D800343300201834002018500020E07A00209E
:1085E80020780020EC4800200A3C0020404B4C003A
:1085F8002F560020A43700203C1F002024410020D3
:108608005C3C002094210020F47700202C020020FC
:10861800E4370020C0760020804200207745002003
:10862800C44000202841002020410020843400203C
:10863800D43400200434544520D0A178E3789942FA
:1086480018FB0170F6D26178043118FB037335F911
:1086580011105945A8BF5946B1F5617FB8BF4FF40D
:1086680061718142E6DD9942E4DC21782729E1D86D
:1086780048460434FAF728F85445DED1664A0B9D7B
:108688001378664A99E8030082E80300002B40F05B
:108698002E86634B1A78002A00F0A88501215F48CE
:1086A800FAF722F8002840F0E482089BDB78002BD8
:1086B80040F0DF822B881FB227F001071FFA87F8E6
:1086C8004345A5F8008001F00880564F4FF0020995
:1086D8000E204FF0140B4FF0FF0A87F8009087F830
:1086E80001B087F802A029F0D9F949464B48B5F8F6
:1086F8000080F9F7F9FF002841F0CF8228F0020343
:108708009BB243452B800BD0464B02201421FF22FD
:1087180018700E2059709A7029F0C0F9B5F80080C9
:10872800414B424A197850680C9318F0030F08BF60
:1087380081F00201C1F340010B9208F05FFB242194
:108748003648F9F7D1FF30B9079A1378590744BF6B
:1087580023F004031370099B1B6813F00A0F1BD046
:1087680005212E48F9F7C0FF002801F0C6802F88A0
:108778007B0741F1458229480621F9F7B5FF002812
:1087880001F0A880780641F1338207212348F9F7E0
:10879800ABFF002840F0C4870C212048F9F7A4FF5C
:1087A8002A88002800F0458342F480739A422B807F
:1087B80009D01C4B022214211A700E20FF22597076
:1087C8009A7029F06BF91A4B1B78082B00F03D833F
:1087D8000E2B00F03A83069BD3F8008018F4806FC4
:1087E80060D0144B1B79002B00F0258214210B4814
:1087F800F9F77AFF002840F0238225F093FC012046
:1088080029F09AF800284AD0DFF82CA000274FF06A
:10881800CC0BA14615E000BF3C520020A437002035
:10882800244500201C310020887600208C7600200A
:10883800F83C0020DC3E0020C0420020DFB2022FBE
:108848002CD80BFB07F87B1C5AF80840002CF5D1F4
:10885800032290F9023002940192C278E24951F859
:1088680022200092184622462346012128F0E8FEDD
:10887800034607EB470000EB0010099353B121466C
:108888000AEB8000CC222DF02CFB099B4AF808301B
:108898000137FFB228F09EFB0028D0D14C46069B3A
:1088A800D3F80080079B93F800A0D04B1AF0010A78
:1088B80000F0408201221A700A9B04991B68B1F9E2
:1088C80006105A89CA4801279142077080F2188217
:1088D800C84B4FF07E521A60059BC74FB3F81890EB
:1088E800049B97F90420B3F90030387897F801C051
:1088F800002AA3EB090714BF01224FF0FF32002F13
:10890800B8BF7F42B7F5FA7FA8BF4FF4FA77B842ED
:1089180080F2F3813F1A07EE907AF8EEE77AB74FC4
:108928004B45C7ED007A03DAF1EE677AC7ED007AB6
:10893800049BB3F902E0AEEB0903002BB8BF5B421E
:10894800B3F5FA7FA8BF4FF4FA73984280F2D28148
:108958001B1A07EE903AF8EEE77AF145C7ED017A6F
:1089680003DDF1EE677AC7ED017A049BB3F90400E1
:10897800A0EB0903002BB8BF5B42B3F5FA7FA8BF91
:108988004FF4FA736345CCBFA3EB0C03002302FB3F
:1089980003F207EE902AF8EEE77A4845C7ED027A27
:1089A800BCBFF1EE677AC7ED027A18F4805800F080
:1089B8007E81B1F5FA6F924BA8BF4FF4FA61B1F519
:1089C8007A7F1A78B8BF4FF47A71A1F57A71002AC4
:1089D80041F033818B4ADFF844E282FB0130CB1748
:1089E800C3EB6013581C6FF0630C3EF910003EF99E
:1089F80013E00CFB0313A0EB0E0003FB00F382FB58
:108A08000312DB17C3EB62139E440FFA8EFE07EEC8
:108A180090EAB8EEE78A87ED038AB8F1000F40F0D4
:108A2800A5832B885A0640F1FB807749774A91ED58
:108A3800018AD2ED019A92ED026A91ED034A92ED14
:108A4800030A91ED029A92ED007AD1ED005AD7ED22
:108A5800011A97ED002A6E4A6E4938EE445A79EEAB
:108A6800C63A77EE007A65EE233A75EEC96A75EE76
:108A7800890A37EE401A66EEA76AB0EE633AA0EEAE
:108A8800813A13F00303B0EE665A78EE044A79EEA1
:108A9800867AA0EE815AF0EE638AA4EEA73AD4EE65
:108AA800A78AA4EEE75A33EE263AF0EE687AF0EE9B
:108AB800674AF6EE008A35EE88AAE0EEC14A28EE4B
:108AC800C33A35EE635A77EE293A77EEE67AAAEE9C
:108AD800233A25EE285A76EE403A34EE49AAE0EEDB
:108AE800817A74EEA64AAAEE235A34EE094A37EE82
:108AF800697A64EEA84A63EE036AE4EE074A75EE03
:108B0800C85A36EE006A67EEA87AB0EE667A95EE35
:108B1800057AE5EE056AE5EE867AB1EE648AF0EE4E
:108B2800665AF0EE476AB1EE674AE8EE246A63EEE9
:108B3800270A67EEA43AE4EE275AB1EE450AB0EEEA
:108B4800606AB0EE631AA4EE277A23EE244AE7EEB1
:108B5800A76AA5EE246AA0EE031AE8EE245AB0EE3E
:108B6800448A31EEA19AE0EE240AA5EE278A66EE41
:108B7800A16A72EE028AE5EE033A61EE211A26EE48
:108B8800096AA4EEA47AA0EE274A0CBFD7ED022A00
:108B9800DFED212A82ED005AA2EE256AE0EEA86AEE
:108BA800E2EE081A73EEA33A27EE227A34EE044A6C
:108BB800F0EE005AE3EEA26AA4EE226AA1EEA57ACC
:108BC800C7ED016AC1ED366A81ED356A87ED006A45
:108BD80081ED377A82ED013AC2ED027AC2ED034A9D
:108BE800F3B987ED027A1BE034870308305600207A
:108BF800CC21002048210020BC370020EC3E00207A
:108C0800E02200201F85EB51D4010020E401002060
:108C18001C0200203C1F0020000000000447002028
:108C2800BAF1000F40F024811DF0D4F917B0BDEC63
:108C3800068BBDE8F08F079B1B78D9077FF5DDAD64
:108C48004FF40F7022F05EF900283FF428AE09F0C7
:108C5800C9FA4FF40F7022F0BDF800283FF41FAE98
:108C680009F0C0FA4FF40F7022F0B4F80028EED1E2
:108C780015E6099B1B6898077FF51CADB5F80080C1
:108C880018F0010F7FF43AAD48F0010398452B80A6
:108C98003FF434ADC14B022214211A700E20FF227A
:108CA80059709A7028F0FAFEB5F8008026E5059B01
:108CB8005A8B9142C0F20785B1F5FA6FD4BFC2EB67
:108CC8000101C2F5FA614FF47A7303FB01F1B4486C
:108CD8000378C2F5FA62B1FBF2F1002B3FF47AAEE9
:108CE8004378B04A01FB03F182FB0123C917C1EBAA
:108CF80063116FE6DFEDAC7A2FE6DFEDAB7A0EE6B7
:108D0800B1F5FA6F80F2E284187A8B1A03FB00F34C
:108D1800C2F5FA6293FBF2F3C3F1640307EE903AEB
:108D2800F8EEE77A9FEDA17AA14B67EE877AC3ED5B
:108D3800007AD1E51B780693002B7FF4BDAD9D4AE0
:108D48001268002A3FF4B8AD9B4A079212F8030C48
:108D5800DFF8A0B21146D71E1CF0B0FE9BF80090B9
:108D6800079A002800F04A86069BB9F1000F41F0E7
:108D7800568507F1080178791CF0A0FE002841F01B
:108D880061858E49B87A1CF099FE002800F0498662
:108D9800B9F1020F41F05E858949F87B1CF08EFE1F
:108DA800002841F053858749387D1CF087FE00284C
:108DB80000F04986B9F1040F41F05C858249787E5C
:108DC8001CF07CFE002841F051858049B87F1CF0DA
:108DD80075FE002800F04986B9F1060F41F042857A
:108DE8007B4997F823001CF069FE002841F036857E
:108DF800784997F828001CF061FE002800F04986A1
:108E0800B9F1080F41F01A85734997F82D001CF045
:108E180055FE00283FF450AD0922134602EB8202AA
:108E280017446E4A7878B9788BF800301070517012
:108E380042E522F480739BB29A422B807FF4B9AC4E
:108E4800674B1B78082B7FF4C3AC2A8822F04003B9
:108E58009BB29A422B803FF4BEAC504B02221421A5
:108E68001A700E20FF2259709A7028F017FEB2E48B
:108E78000C9B19780B9B01F00101186807F0BEFFE5
:108E880017B0BDEC068BBDE8F08F13B9089A012323
:108E98009370544B089A1D7892F8214007931B2031
:108EA8001CF044FE012C05F00108814600F068879B
:108EB80005F00205089A4C4E92F82030DFF838A1E8
:108EC8004A4F09959346052B00F2D487DFE813F043
:108ED800BF00B5000600FD00FF00F200012C04BF32
:108EE80005238BF82030B8F1000F12D0059B30888D
:108EF800B3F918100022134661F30F0260F31F4202
:108F080061F30F03049861F31F4303600323426076
:108F18000993374DDBF814102A68914280F04B868C
:108F280047F230510322CBF81C108BF82020022086
:108F380026F056FF18F078FF2968DBF81C200A4451
:108F48000421CBF818208BF82010012C40F0D8878A
:108F58002A68DBF81810914280F08C879AF8000094
:108F680020B91CF0E3FD002840F084873A6822F01D
:108F780002023A602A687388642101FB03234FF4D4
:108F880080600022CBF810308BF820208BF803206B
:108F980026F0F6FE9BF8203095E700BF1C31002034
:108FA800E02200201F85EB51000000000AD7233C77
:108FB8004821002034560020EA300020F4300020F8
:108FC800F9300020FE300020033100200831002055
:108FD8000D310020123100201731002038560020B2
:108FE800F83C00202F560020FC4600201C410020A1
:108FF800C0760020000000202C0200201CF09CFD00
:10900800012807D1BB4D72882B68642101FB02330C
:10901800CBF81030B9F1000F02D0B379002B4BD147
:10902800012C00F02787B34DDBF810102A68914215
:10903800C0F0738701238BF82030012C3AD0F379E4
:10904800012B46D01CF0F8FC9BF820303BE7B8F128
:10905800000FD3D1099D4FF48060B9F1000F00F0E3
:109068005C8326F0A5FE089A00231361002D3FF4C7
:109078008DA9284628F012FD069B1E6816F4805715
:109088003FF48AA91D219C48F9F72EFB00287FF49C
:1090980083A99A4B03F1500A03E004339A4500F080
:1090A800EF861A78262AF8D19978DA789142F4D29C
:1090B800FFF774B98F4D5DE71CF0BEFC03224FF437
:1090C8007A738BF82020CBF81C308A4D2FE7894D16
:1090D8003BE71CF0B1FC032240F6B8338BF82020A4
:1090E800CBF81C30834D22E7854F3B78002B01F0ED
:1090F800B282844BDFF82482DFF824B2DFF824A29E
:10910800059345465E46049099460EE019F804100A
:109118009847032C28DC88B93B782AF8020F0134D9
:109128009C4205F1040580F24F81072CE1B23046DC
:10913800DBF80430EADD984700B2EDE738F8242080
:109148006B88801A4FF47A719B1A01FB00F040F685
:10915800CA0290FBF3F00844904240F2EE23A8BF05
:1091680010469842B8BF184600B2D5E71D2162489C
:10917800F9F7BAFA28B100F03FBE0436B4423FF41A
:1091880050AC31782629F8D1B278F3789A42F4D2E3
:10919800089BDB78002B7FF444AC5748F9F7A4FA16
:1091A800DFED597A002801F06D8238EE678A574A58
:1091B8005749FDEEC87ACDED047ABDF910301B038E
:1091C80082FB0302DB17C3EBA212C9F57A731BB249
:1091D80003FB02F343F30F334B4407EE903AF8EEE8
:1091E800E77A0123C7ED037A0B701AE4DFF83891A8
:1091F800DFF838A1474F0B9209F15A084FF0010BDD
:10920800494619F8010C1CF059FC00B399F8040000
:1092180099F8023099F803E000EB400107EB81016F
:10922800013BD1F8A02003EB4303534493420ED0F3
:1092380097F8CC20C1F8A0300BFA00F022EA000021
:109248000B9B81F89CE0C1F8A43087F8CC0009F1A9
:109258000609C145D4D1304B264A1B780B930A9B8B
:10926800DFF8CCA012681B680C93AAF19C094FF098
:10927800000B9046DAF8043083B31F7877B3DAF836
:109288000820A8EB0202002A0CDB99F8CC20012167
:1092980001FA0BF122EA010208F5FA7189F8CC20EB
:1092A800CAF808100B9ACAB19AF800205978043203
:1092B800D2B2002940F0518305990498098B30F9FE
:1092C800122001F1C800824240F3EC8599F8CC10D5
:1092D8009A7841FA0BF3D90740F177860BF1010B25
:1092E800BBF1040F0AF10C0AC4D1FFF7D7B9034B3D
:1092F80024E000BFC0760020A4370020843400207A
:1093080044350020E07A002000007A44D34D6210F2
:10931800C02100203C1F0020BD48002058350020F7
:10932800203300203A1F002001300020306103085C
:10933800D81F00200433A3423FF4ABA9197823298E
:10934800F8D19878DA789042F4D29F48F9F7CCF9B6
:1093580000283FF49EA99D4B1B6813F4003341F08D
:10936800558200229A4B1046995C142902F10C028E
:1093780001F0088101301828F6D1FFF78AB9954C19
:1093880094F896305BB1079B1B78D80707D5049BE8
:10939800B3F90620059B5B8B9A4200F308861121DE
:1093A8008948F9F7A1F9002800F0BF8294F89A30AB
:1093B8002BB994F8943013B93223A4F898300123C8
:1093C80084F89A30FFF7F0B8DDF81090824A0692D8
:1093D8008249126842F2010AA1FB091B12EA0A0A31
:1093E8004FEA9B1B00F09E827D4D7E487E4C7F4954
:1093F8002E780078267008701EB17C490E7886F0A9
:109408000106744C0F2184F82410002B00F01884F6
:10941800059D774BB5F826C0B5F824E0059D109357
:1094280018462D8B0078734B129594F825500995A2
:10943800714D0495A3FB00535B0803EB4303C31A68
:10944800DBB20F90CDF834C002F480520C9304F1D3
:1094580028000BF59673CDF8449097F80080DDF856
:109468002490DFF8ACC10994634C0E91139200214B
:109478000A930896CDF81CE0089B002B00F03D836A
:10948800099B079D33F911201FFA82FEAE454FEA6A
:10949800410303D30D9DAE4540F274835CF821204F
:1094A800934580F03483E25EBAF1000F40F04983BF
:1094B80001314145E25200F10600DDDB0E9A099CBC
:1094C8004E4B84F824200F2A49460CBF0122002263
:1094D800DDF8449084F825101A7000F0B883484BE2
:1094E8004049424ADFF82CB108931C460420012366
:1094F8000B70137026F074FCDBF80030A16862680A
:10950800E3605B1A934284BF002384F82130069BF2
:109518003C781E68002C01F0D680059A394DB2F8C7
:1095280024E0178B344916F48056284640F0C88347
:1095380032460EE0437803EB830303EB830303F225
:10954800EE239BB20132A24221F8023B00F1020055
:109558000ED015F81230002B00F01883022BE9D03A
:1095680001320B8821F8023BA24200F10200F0D13F
:10957800109A137801331370FEF7EFBE059A049919
:10958800537DD27D013B31F913301AB1C3F53B63EA
:1095980008331BB2A3F57A7307EE903A9FED1A7A57
:1095A8001A4AF8EEE77A40F2FF3167EE877AFCEE66
:1095B800E77ACDED077ABDF81C308B4228BF0B4601
:1095C8001380FEF7D8BE00BFA4370020F42F002078
:1095D800DC7503083C1F002018500020D34D621092
:1095E800FC3200209C010020BD4800209D01002085
:1095F80039340020ABAAAAAA20780020043D002014
:10960800EC4800208C3500206F12833F147800202E
:109618003C340020C0760020DA4CD4F88830A9EB1E
:109628000303002BFEF6A7AED74AD84B527C059908
:1096380033F812308A7DDFEDD66A9FEDD66AC97D90
:109648009BB207EE102A07EE903AB8EEC77AF8EE0A
:10965800E77A27EE267A67EE867A0B9AC4F888208E
:10966800C7EE876A40F2FF32FCEEE67ACDED077A64
:10967800BDF81C30934228BF134609B1D31A9BB2D8
:10968800C548C64D0178C64C35F81160226825F8E2
:109698001130921B13440131C24D236001F00F02B7
:1096A8001B0902702B80FEF766BEFEF763F9BE4BFE
:1096B800BE4A1B68C31A93427EF75DAEB94B0022BF
:1096C8001A80FEF758BE4146FFF701BB1B7AC3F16B
:1096D800640307EE903AFFF723BB0221B448F9F779
:1096E80003F800283FF40AA82F8018F0020F7FF42F
:1096F80017A848F0020343452B803FF411A8AD4B4F
:10970800022214211A700E20FF2259709A7028F034
:10971800C5F9B5F80080FFF703B826F031FBA2E4DD
:10972800A54AB2F90030002BB8BF5B42B3F5E17F20
:10973800BFF632A8B2F90230002BB8BF5B42B3F5CE
:10974800E17FBFF629A89D4B93ED096AD3ED076A1F
:1097580093ED057AD3ED037A76EE866A77EE877A0B
:1097680076EEA66AB7EE007A37EE666A77EEA77AE3
:10977800B0EEC66AF0EEE75AB4EEE56AF1EE10FA1A
:10978800B4BFB0EE655AB0EE465AB5EE405AF1EEA7
:1097980010FA40F0DC839FED8A7AB4EEE56AF1EEC8
:1097A80010FA44BF9FED876A36EE477AB7EE006A33
:1097B800F4EEC66AF1EE10FAC8BFDFED836AF5EE83
:1097C800C07AC8BF36EEC77AF1EE10FA48BFB1EEDC
:1097D800477AF6EE007A27EE677ADFED7A7A77EE47
:1097E800276ABDEEE66A16EE103A2033402B40F2A7
:1097F8008186DFED766A764ADFED747AC2ED006A1B
:10980800FDEEC76AC2ED017A16EE903A2033402B7E
:10981800C2ED027A49D8DFED6C7AB4EEE77AF1EE60
:1098280010FA41F343809FED6B6ADFED6B6A01E04C
:10983800B0EE677AB4EEE67AF1EE10FA77EE467A91
:10984800F6DC9FED667AF4EEC77AF1EE10FA41F194
:1098580041809FED606ADFED626A01E0F0EE477AD1
:10986800F4EEE67AF1EE10FA37EE867AF6D4DFED0A
:10987800557AB4EEE77AF1EE10FA40F3D686DFEDCA
:10988800527A37EEC77A27EE076ADFED565ADFEDD0
:10989800566ADFED567AE6EE256A67EE065AE6EE78
:1098A800267AA5EEA77AF0EE477A514BC2ED037AF5
:1098B8001A6812F4003240F095864E4B1046995CB7
:1098C8000A2902F10C0200F0858501301828F6D12A
:1098D800FEF762BF27F040039BB2BB422B803EF4E9
:1098E80054AF344B022214211A700E20FF225970F3
:1098F8009A7028F0D3F8FEF748BF2B8823F00407A6
:10990800BFB2BB422F803EF436AF2A4B022214214D
:109918001A700E20FF2259709A7028F0BFF82F880D
:10992800FEF729BF34490E7866E594F89430002B89
:109938003EF43AAE079B1B7813F001037EF434AE75
:10994800012284F8943084F89520FEF72DBE0D4C42
:10995800012184F88C10FEF79ABD012900F0588582
:1099680099F8CC20012303FA0BF30BF1010B1343F5
:10997800BBF1040F89F8CC300AF10C0A7FF47AACF9
:10998800FEF78CBE3C1F0020387600205876002059
:109998000000C842000080440B3C0020103C00201E
:1099A8000C3C002014780020A81E002060E316005C
:1099B800A43700201C310020D0400020F4010020F2
:1099C800A7DFA834DB0FC93FDB0F494000000000C8
:1099D800D4010020DB0FC940E4CB1641DB0F49C09E
:1099E800E4CB16C192E741B99730083C15A82ABEC6
:1099F800F42F0020DC750308BD480020511D78793C
:109A08001CF05CF800283FF4BCA9B9F1010F40F044
:109A1800198707F10D01B87A1CF050F8002840F0BA
:109A28001987C149F87B1CF049F800283FF4BBA905
:109A3800B9F1030F40F00A87BC49387D1CF03EF8A5
:109A4800002840F01787BA49787E1CF037F80028BC
:109A58003FF4BBA9B9F1050F40F00887B549B87FB5
:109A68001CF02CF8002840F0FD86B34997F8230035
:109A78001CF024F800283FF4BBA9B9F1070F40F007
:109A8800ED86AE4997F828001CF018F8002840F039
:109A9800D586AB4997F82D001CF010F800283EF445
:109AA8000BAFB9F1090F3EF407AFFFF7B5B95D2A5F
:109AB80000F090825B2A00F0D2855E2A00F08C8646
:109AC800562A00F08E86972A00F0D886A72A00F03A
:109AD80077869C4D2B889E0740F04286A2F1B703FB
:109AE800072B00F2B182DFE813F0A102AF02AF0248
:109AF800AF029302AF0285028502079B002B3FD07D
:109B08005CF8212093454FEA4103FFF4CCAC8E4A20
:109B18008D4DD25C05EB030E002A00F0B180022ABD
:109B280047D19EF8012002EB820202EB820202F288
:109B3800EE2292B2032933DD12B2BAF1000F3FF4DC
:109B4800B7AC0C9D20F81520B9F1000F03D10F9D7B
:109B5800022D7FF6ADACB0F802900288B0F804E0B0
:109B68004A449644794A0FFA8EFE82FB0E52784D8B
:109B7800A2EBEE7225F803E012B24FF0010997E468
:109B88001A464B000A9D4CF821508DE4D3B2022BA3
:109B980004D9032B7FF4E4AC7346D3E43B46D1E409
:109BA800012505FA01FE0E9D25EA0E0512B20E9555
:109BB8007AE4E25ABEE7674A1278002A7FF4B0A92D
:109BC800B8F1000F3FF4ACA9012C40F053819BF889
:109BD8002030FFF778B931465F48F8F785FD00284F
:109BE80000F0D18084F8936018F00CFCFEF7A6BC56
:109BF80047F04003BB422B807FF473AEFEF7C5BD30
:109C080047F004039F422B800AD0544B02221421B0
:109C18001A700E20FF2259709A7027F03FFF2F8884
:109C28004F4B504AB3F904304F4982FB0302DB170C
:109C3800C3EBA2030B80FEF79EBD5B78FFF751B81C
:109C48004A4B4B4A109201221A704A4B04931B212B
:109C58004148F8F749FD00287FF441AC464BDFF84E
:109C68001CB108931946DBF80030CA688B609B1A50
:109C7800C82B00F2F884069B1E6806F4805677E429
:109C8800CAB2022A40F2C183032A92D1129A139DC2
:109C9800079E002D08BF32464CE728F001039BB20F
:109CA80043452B803FF421AD0E2087F8009087F8BC
:109CB80001B087F802A027F0F1FEB5F8008014E59E
:109CC80000220FE0437803EB830303EB830303F2E3
:109CD800EE239BB20132A24221F8023B00F10200BE
:109CE8003FF446AC15F812301BB1022BEAD00B88B2
:109CF800F0E7D3B2032BFAD83B46EBE7B2F5FA7F8D
:109D0800FEF648AC94F89230002B7EF443AC079BE7
:109D18001B7801210B4084F8921000F0D38318F0CF
:109D280083F8FEF737BC00BFF9300020FE30002072
:109D380003310020083100200D31002012310020AD
:109D480017310020204100208C35002056555555EC
:109D5800AC1F002084210020A43700201C310020E3
:109D6800D040002067666666C2210020043D0020BE
:109D78003934002020780020EC480020C0760020EC
:109D88000025FFF797B8079BC14A1B781060D807D2
:109D98007EF5D8ABBF4B1B78002B3EF4FBAB089B82
:109DA800DB78002B7EF4F6AB94F893300133DBB20A
:109DB800032B84F893307EF6EDABB74B5B7813B981
:109DC800002D7EF4E7AB18F02FF8FEF7B7BBB2F51D
:109DD800FA7FFEF6DFAB94F89230002B7EF4DAAB14
:109DE800079A1278012184F89210D10700F12A8489
:109DF80018F008FBFEF7CEBB089BDB78002B7FF43E
:109E0800C0A9DFEDA67AA64938EE678AC9F5FA63D4
:109E1800FDEEC87A1BB2CDED047ABDF9102012030D
:109E280081FB0201D217C2EBA11203FB02F343F339
:109E38000F334B4407EE903AB8EEE78A87ED038A72
:109E4800FFF79FB9974A96491068B4F99020C669F8
:109E580081FB06018911F617701A00F5FF407F3063
:109E680082423EF75EAB891B0A4412B2A4F89020E6
:109E7800FEF757BB099D002D3EF488AAFFF7F9B8F5
:109E8800894A059BD588049A1B8BB2F906105A1B80
:109E9800914240F389802B449942B4BF00250125A3
:109EA800FEF785BAC8398A4242DA99F8CC109A780E
:109EB80041FA0BF3DB073FF511AA524201200D923C
:109EC80027F0D2FE7B1E0D9A162B00F28581DFE863
:109ED80013F006021A02EE013F022E025302D901C4
:109EE800C401AF019A01860183013F027501530243
:109EF800D901C40161014D013901680223010F0133
:109F0800AB460899DBF80020CB69099D13448B61A7
:109F1800002D3EF43BAAFFF7ACB81BF08DFD0321E2
:109F280040F6B8328BF82010CBF81C20FEF7FFBFA4
:109F380099F8CC30012202FA0BF223EA020308F561
:109F4800FA7289F8CC30CAF80820FFF7C7B9B4EE1E
:109F5800E56AF1EE10FA8CBFB0EE654AB0EE464AFB
:109F6800C4EE054A9FED512A9FED515ADFED511A73
:109F7800DFED512A9FED513ADFED513A9FED514AFD
:109F8800A4EE825AE4EEE12AA4EE857AA4EEA23A7F
:109F9800B0EE475AB0EE637AA4EE837AA4EE874A0D
:109FA80084EE057AFFF7F9BB0125FEF700BA002118
:109FB8004548F8F799FB00287FF4F1A9322384F883
:109FC8009600A4F89830FFF7EAB9002A0CBF0120E0
:109FD800022074E73D4B002201203D493D4C0B60B7
:109FE8003D4B09933D4B22703D4D0A9327F03CFEB3
:109FF800FEF7D5BA394A374B0A921146394A0A60F0
:10A0080002225A70344B09931BF0F4FDFEF7C7BACD
:10A01800324A304B0A921146334A0A6000225A707B
:10A028002D4B09931BF0E6FDFEF7B9BA2B4A294BD5
:10A038000A9211462D4A0A6001225A70264B09934A
:10A048001BF0D8FDFEF7ABBA9E2A00F08D849D2A3E
:10A0580000F08284AE2A00F07784AD2A00F06C8488
:10A06800EF2A00F06684FD2A00F05184FB2A00F0F4
:10A078008C84FE2A00F08684F72A00F080847B2AEC
:10A0880000F03E84144B0993144B0A93FEF787BAE9
:10A0980084420020BD480020E437002000007A44B4
:10A0A800D34D62103C7A0020E046002099FB243F03
:10A0B80069A2163E39094E3DE3B59E3E88FA163E22
:10A0C80045FE7F3FA7DFA834A43700200A8100207F
:10A0D80024410020574C0020C44000202841002083
:10A0E800204100202E82002016820020228200209B
:10A0F800D9F8D000B64B90F836109B7811446429F3
:10A10800A8BF642121EAE17180F83610002B40F0E5
:10A11800518422F083FB23E4D9F8D000AC4B90F8AB
:10A1280037109B781144FE29A8BFFE2121EAE1716E
:10A1380080F83710002BECD016201BF041FDD9F821
:10A14800D000E6E7D9F8D000A14B81781144C8299E
:10A15800A8BFC82121EAE17181709B78002BD8D073
:10A1680014201BF02DFDD9F8D000D2E7D9F8D00083
:10A17800974B41781144C829A8BFC82121EAE17149
:10A1880041709B78002BC4D013201BF019FDD9F81F
:10A19800D000BEE7D9F8D0008D4B01781144C8290A
:10A1A800A8BFC82121EAE17101709B78002BB0D0CB
:10A1B80012201BF005FDD9F8D000AAE7844B0C98B3
:10A1C8009B78417911446429A8BF642121EAE1718F
:10A1D8004171002B40F01A84D9F8D00099E7D9F8DA
:10A1E800D0007B4B017A9B781144C829A8BFC821AD
:10A1F80021EAE1710172002B8BD00B201BF0E0FCEF
:10A20800D9F8D00085E7D9F8D000714BC1799B788F
:10A218001144C829A8BFC82121EAE171C171002BE6
:10A228003FF477AF0A201BF0CBFCD9F8D00070E7D9
:10A23800D9F8D000664B81799B781144C829A8BF0A
:10A24800C82121EAE1718171002B3FF462AF092036
:10A258001BF0B6FCD9F8D0005BE7D9F8D0005C4B0E
:10A26800417993F802E01144C829A8BFC82121EA1E
:10A27800E1714171BEF1000F40F08A83112F7FF424
:10A2880064AF46E7D9F8D000514B017993F802E062
:10A298001144C829A8BFC82121EAE1710171BEF1A2
:10A2A800000F40F09583102F7FF463AF31E70C99CE
:10A2B800474B0F790D931744642FA8BF642727EAEB
:10A2C800E7770F711BF096FC0D9B9B78002B83D0D2
:10A2D800032039461BF074FCD9F8D00019E70C9814
:10A2E8003B4B01781144FA29A8BFFA2121EAE17110
:10A2F80001709B78002B3FF46FAF01201BF060FCCE
:10A30800D9F8D00005E70C98314B817811446429BD
:10A31800A8BF642121EAE17181709B78002B3FF48A
:10A328005BAF02201BF04CFCD9F8D000F1E60C988A
:10A33800274BC1799B78114481F30801C171002B27
:10A348003FF44AAF05201BF03BFCD9F8D000E0E60B
:10A358000C981F4B817993F802E011446429A8BF37
:10A36800642121EAE1718171BEF1000F40F01A8386
:10A378000D2F7FF424AF2FE7D9F8D000144BC17804
:10A3880093F802E01144C829A8BFC82121EAE17165
:10A39800C170BEF1000F40F011830F2F7FF4FDAEA6
:10A3A800B7E60C980A4B41781144B1F5967FA8BFDF
:10A3B8004FF4967121EAE17141709B78002B3FF4CC
:10A3C8000BAF15201BF0FCFBD9F8D000A1E600BFAD
:10A3D800F6770020C449D1F800E04200BEF1000F32
:10A3E80008D0171803EB87079EF801E07F787745B8
:10A3F800BEF4D2A91044BD4FBD4A03EB8003002030
:10A408000B6038801060FEF7C7B9129AFFF792BB4D
:10A4180004999B7831F91220B2F5617F4FF4966167
:10A4280091FBF3F3C0F2E68040F633019142A8BFF6
:10A4380011460C2FA1F5617191FBF3F100F0FC813D
:10A44800182F7FF48DAAC9B2C8290B46A8BFC82304
:10A45800D9F8D020D77DD8B2B8423FF481AADF1B03
:10A46800A44BD07548BF0737FF109B780137FFB260
:10A478003BB9002F3FF474AA384627F0F5FBFFF7E5
:10A488006FBA18201BF09CFBF3E79B4A9B4B099281
:10A4980010461A689A494FF47A73B3FBF2F3C3EB88
:10A4A800431203EB82030268DB00A1F8A8305307CC
:10A4B8007EF572A8934B944D0A221A80934B0A9307
:10A4C800FEF76DB89249096811F4003140F098819F
:10A4D800904B08465D5C0F2D01F10C016DD00130E9
:10A4E8001828F7D1FA3A0023A4F8902084F892307B
:10A4F800FEF750B8B4EEE77AF1EE10FA40F3D381E4
:10A50800DFED855A9FED856A01E0F0EE676AF4EEAB
:10A51800C66AF1EE10FA76EEE57AF6DCDFED806ACF
:10A52800F4EEE67AF1EE10FA40F1B381DFED7A5AF3
:10A538009FED7C6A01E0F0EE667AF4EEC67AF1EE01
:10A5480010FA77EEA56AF6D4DFED777AF4EEE76ACB
:10A55800F1EE10FA40F3BB80DFED747A77EEE66A2D
:10A5680066EEA65A9FED725A9FED726ADFED727A17
:10A57800A5EE856A26EEA55AE5EE867AE5EE276A07
:10A58800FFF739B95849D1F800E04200BEF1000F91
:10A5980008D0171803EB87079EF801E07F78774506
:10A5A800BEF477A80244514F514803EB82030022BE
:10A5B8000B603A800260FEF76CB84B490F684500A3
:10A5C80037B12E1803EB86067F787678BE4289D29B
:10A5D8000544464E464803EB850300250B6035804D
:10A5E80005607FE7554B1B78032B00F02181002283
:10A5F800FFF763B90C2F40F0158100273946504BFF
:10A608000E915B78BB423FF4ABA93A4B0D933846A9
:10A6180018F08CFD0D9B0E999B781BB1C9B20C20CC
:10A628001BF0CEFA0137FFB223E7DFED467AB4EE2E
:10A63800E77AF1EE10FA44BFDFED397A37EEC77AE0
:10A64800FFF721B9404A2C491360304B09912E4D30
:10A658000A93FDF7A4BF3D4A0592FEF7B7BE3C4BEF
:10A6680001220220B9E43B4A069B1E68136823F0C6
:10A6780004031360089A012306F4805682F82130F7
:10A68800FEF776BF38EE678A334B34491870FDEE13
:10A69800C87AC9F5FA63CDED047ABDF91020120322
:10A6A80081FB0201D217C2EBA1121BB203FB02F31A
:10A6B80043F30F334B4407EE903AF8EEE77AC7EDD1
:10A6C800037AFEF7AEB906F48056FEF751BFDFED08
:10A6D8001D7AF4EEE76AF1EE10FA44BFDFED107A66
:10A6E80077EEE66A3CE700BF4021002028220020E0
:10A6F8002C220020F6770020C440002008500020BB
:10A708007C4D00201E4700202041002028410020C9
:10A71800F42F0020DC750308DB0FC940E4CB164199
:10A72800DB0F49C0E4CB16C1DB0FC93FDB0F494043
:10A7380092E741B99730083C15A82ABE5078002006
:10A74800574C0020DB0FC9BF84420020E07A00206C
:10A75800588100201C410020C0210020D34D6210E8
:10A768000023BB2A149300F0C880B72A00F0C180E8
:10A77800BE2A00F09680BD2A7FF466AC4FF6FE71C3
:10A78800A64AA748D6890990908933440144D381C1
:10A7980091810EF041FDF7F723F90EF025FDFBF747
:10A7A800C9FF012027F060FAB4F890309D4A0A9258
:10A7B800FA3B0022A4F8903084F89220FDF7EFBE0F
:10A7C800994A974B09931378984D43F004031370F3
:10A7D800944B0A93FDF7E3BE954B02220320FFF743
:10A7E800FCBB0EF019FDF7F7FBF80EF0FDFCFBF7CC
:10A7F800A1FF012027F038FA94F88E20FFF763B9FB
:10A808008C490978032947D0194661E6894B1B789A
:10A81800032B7EF4A6AD27F025F9FDF73ABF1A46BB
:10A82800FEF7FCBA182F7FF49BA800210B460FE611
:10A8380027F018F9FDF7B0BFCFB2E0E608221346BB
:10A84800FEF7ECBA01221346FEF7E8BA03221346D4
:10A85800FEF7E4BA02221346FEF7E0BA07221346CF
:10A86800FEF7DCBA06221346FEF7D8BA05221346CD
:10A87800FEF7D4BA04221346FEF7D0BA6E4B684AE4
:10A8880009924FF4C8721A80664B684D0A93FDF717
:10A8980086BEF0EE676A57E627F0E4F8B4F9902030
:10A8A80020E602216CE7F0EE667A37E6F0EE477AAA
:10A8B800FEF7C7BF002D3DF4BEAD604C94F88D3057
:10A8C800002B3DF4E9AD27F0CDF8002384F88D3056
:10A8D800FDF7E2BDB0EE677AFEF7C9BF504B0993AA
:10A8E800504B84F8941084F89500504D0A93FEF765
:10A8F80047BD19464FF6FE7342E7194602233FE764
:10A908004FF4FA61022018F02FFBFFF7BBBB0021C0
:10A91800012018F029FBB4F89030414A0992963B7F
:10A92800404AA4F8903000230A9284F89230FDF748
:10A9380036BE00210846ECE7FF2100201FF0D8FBB7
:10A9480094F88E20FFF78CBB012100201FF0D0FB6C
:10A9580094F88E20FFF781BB0021FF201FF0C8FB71
:10A9680094F88E20FFF776BB002101201FF0C0FB72
:10A9780094F88E20FFF76BBB0B20FDF709BE002172
:10A988000420C6E700210320C3E700210220C0E716
:10A9980011200E930D921BF013F9D9F8D0000E9BDD
:10A9A8000D9A6BE40D200E930D921BF009F90E9B86
:10A9B8000D9ADDE417201BF003F90DE40F200E9328
:10A9C8000D921BF0FDF8D9F8D0000E9B0D9AE4E427
:10A9D80010200E930D921BF0F3F8D9F8D0000E9BBF
:10A9E8000D9A60E4002B3FF468AF1549154A0968D1
:10A9F8004FF47A7000FB031313605EE70F4C17F0F7
:10AA080013FA002384F88D30FDF746BD0E201BF0A5
:10AA1800D7F8D9F8D000FFF77CBB00BFC4370020B7
:10AA2800C440002028410020F47700202041002065
:10AA3800A681002050780020204700203C1F0020DD
:10AA4800C0760020804200202DE9F04F2DED0E8BBE
:10AA5800DFF8A8A393B0DAF804300490504698477A
:10AA6800002875D0BAF8A85000228AF85120002D85
:10AA780041F07684DAF84830BAF93C60BAF938001F
:10AA8800DAF82050BAF93A10DAF82440DFF870B34F
:10AA9800F71A87EAE772A2EBE772B2F5804FDAF8A5
:10AAA8002820DCBFCAF848603346401B091B9B1AA4
:10AAB800CAF82C00CAF83010B4489AF85210CAF8EC
:10AAC800343012F053FBDBF80030990041F1608517
:10AAD800DAED0C5ADFF82C93DAED0B7AAC4999EDE4
:10AAE800406AD9ED416A99ED427AD9F80C21096892
:10AAF800A84B0293B8EEE58ADAED0D5AF8EEE77A3C
:10AB0800F8EEE58A013277EE867A38EE268A78EE14
:10AB1800878A8A42C9ED407A89ED418AC9ED428A1D
:10AB2800C9F80C2102F088821F78142F03F0DF8106
:10AB38000023D9F814410393062C01F2B781DFE80A
:10AB480014F0CB1551158E148D1625096215EE14C7
:10AB5800904BDFF8B0921C780293072C01F0F98132
:10AB680099F82831069353B15F1E89F82871012C92
:10AB780001F0C48413B0BDEC0E8BBDE8F08F864A9B
:10AB88005279002A01F05982844A1278013AD2B2E5
:10AB9800072C89F8282102F01083002307938049A5
:10ABA800D9F83421D1ED006A7E49059104999FEDC9
:10ABB8007E6AD9ED4C9A7D4BDFF84CB21B6899ED53
:10ABC8004BDADFF848829FED7A9ADFED7AAA9FED9B
:10ABD8007ACA9FED7AAADFED7ABA9FED7ABA7A4FF0
:10ABE8007A4ECDF80CB08A1A07EE902AF8EE677AFA
:10ABF800B7EE007AC6EE278A0024C9F83411254634
:10AC08009B4677EE69CA6CEEA6CAF4EEC7CAF1EEA7
:10AC180010FA88BFF0EE47CA6D4B98ED008A2344BE
:10AC2800D3ED007AF5EE407AF1EE10FA17D0694BC1
:10AC3800234493ED007A78EE476AB0EEE66AF4EEC4
:10AC4800C67AF1EE10FA08D5F5EEC06AF1EE10FA00
:10AC5800CCBF37EE878A37EE678A83ED008A5E4B72
:10AC68001A88930739D0022D37D09BF82E105B4BEA
:10AC780007EE901A234493ED007A4B42F8EEE76A08
:10AC880007EE903A26EE877AF8EEE77AB4EEE77A9E
:10AC9800F1EE10FA0AD407EE901AF8EE677AF4EE9D
:10ACA800C77AF1EE10FA88BFF0EE477A4C4B4D495F
:10ACB80003EB450331F91500B3F90C30C31A07EE5D
:10ACC800103AB8EEC77AD007E7EE497A41F14B81DE
:10ACD800454B93ED008A27EE888A059B99F86821F1
:10ACE800234493ED01EA78EE4EDA002A00F0DA8088
:10ACF8003E4BD9F86C2104991B688A1A9A4240F392
:10AD0800D1809BF84830022B02F0A682022D04F075
:10AD1800D385374B1B6899077AD4364B86ED00CA22
:10AD28001B689342C0F2AE80F7EE007AF4EEE79A21
:10AD3800F1EE10FA40F1B68005992F4BD1ED017A6A
:10AD480093ED007AF0EEE77AF4EEC77AF1EE10FAB6
:10AD580040F1A880D1ED027AF0EEE77AB4EEE77A16
:10AD6800F1EE10FA40F39E80D1ED037AF0EEE77A27
:10AD7800B4EEE77AF1EE10FA40F394801C4B1B68AE
:10AD88009B077FD51749164B63E000BFA84D0020ED
:10AD980098380020CC3D0020F44F0020B837002020
:10ADA8000C7600200850002000247449244100201B
:10ADB800CDCCCC3DAE47813F000000000000C8422A
:10ADC80000003443610BB63B683C00205C3C00202B
:10ADD8000076002060210020204100206C21002006
:10ADE800C4370020D0400020E875002014760020E9
:10ADF800C4400020107600201C7600207C4D0020E6
:10AE0800185000201C200020503C00205421002015
:10AE1800D34BD449DFF8C8E331F915C09EED008A59
:10AE2800DFF8C0E386ED00CA03EB450028EE098A87
:10AE3800B0F90C00A0EB0C0007EE900AF8EEE77AE8
:10AE4800DEF8000027EE888A904278EE4EDABFF6E8
:10AE58006BAFB3F90C20B1F900E0C348AEEB020EBA
:10AE680000688EEAEE72A2EBEE7282421ADAB3F949
:10AE78000E30B1F90220D21A82EAE273A3EBE27330
:10AE880098420FDDB94B1A88002389F86831002AE7
:10AE980043F08B86B64AB74B1178186881F00101E8
:10AEA80005F0ACFFB44B234493ED000A039B2DEE51
:10AEB800000A022D20EE2D0AA3EC010A039304F0E8
:10AEC800AD84AE4BD6ED006A93ED007AAC4BD3ED72
:10AED800007AAC4B93ED006AAB4B67EE277A2344BC
:10AEE80027EEAC7AD3ED007A67EE277AF0EE665A51
:10AEF800EDEEA75AB1EE467AB4EEE57AF1EE10FA25
:10AF080008DCF4EEC65AF1EE10FA8CBFB0EE467AC1
:10AF1800B0EE657A99ED4C6AF7EE007AB4EEE76A1E
:10AF2800F1EE10FAACBF0123002343B1F0EEE66A5C
:10AF3800F0EEC77AF4EEE67AF1EE10FA01D586ED76
:10AF4800007A022D04F0D283904A914B52F82500E2
:10AF58001B68B0EE4E0A98478E4A8F4B52F8250070
:10AF68001B6898479BF8373023B18C4B1B88002B04
:10AF780001F0EE80B0EE4C8A894B38EE400A23444B
:10AF880093ED008A83ED000A9BF8483030EE480ABA
:10AF980020EE288A002B33D0824B1B7813F0010354
:10AFA80000F0BF86F7EE007AF4EEE79AF1EE10FAB9
:10AFB80099F86831C1F2C185002B01F07981D9F87F
:10AFC8006C31049AD31A784A12689A4218DD774B82
:10AFD800D3ED007AF0EEEDDAF4EEE7DAF1EE10FAFE
:10AFE80042F14B81614B1A88002389F86831002AA5
:10AFF80000F0A3866E494A6912B10A6813604B745F
:10B008006C4B99F87821234493ED000A2DEE000A41
:10B0180020EE088A87ED008A32B9039B86ED00CAC4
:10B0280003ED01CA87ED00CA0135032D08F10408B4
:10B0380007F1040706F1040604F104047FF4ECADFB
:10B04800029B1A78072A01F08E85012A02F0A38054
:10B058000023059399F88021002A41F08382DFF8C4
:10B0680088B1554BDBF800201968D50491F82C00FD
:10B0780001F19A80DFF87481504AB8F81A30D2ED9D
:10B08800005A4F4A4F4CD2ED004AD4ED036A4E4A5B
:10B09800C9ED645A07EE103A4C4B92ED005AD3EDC5
:10B0A800007AD3ED013A93ED026AC9ED625AB8EE1F
:10B0B800C77A34EEE54A012236EEC77A89ED614A4D
:10B0C800C9ED654A89F89821C7EE055A0A8D534299
:10B0D80006EE903A3E4BDFED3F4A93ED005A3E4B69
:10B0E80093ED004AB7EE007AF4EEC75A35EE045AEB
:10B0F800F1EE10FA88BFF0EE475A35EE275AF8EE0F
:10B10800E66AF4EEE45AF1EE10FA07EE902AB4EE8D
:10B11800E65AB8BFF0EE645AF1EE10FAC9ED685A73
:10B12800B8EE677A01F18683B4EEC75AF1EE10FAE9
:10B1380088BFB0EE475A264BDFED284AD3ED017A97
:10B14800254B93ED014A77EE847A25EE245A77EE63
:10B15800A37AF4EEE76AF1EE10FA52DC48E000BF99
:10B16800C4370020D04000201876002098760020B0
:10B178009A7600209C760020BC750020F874002088
:10B188000400002030760020C875002000750020DB
:10B19800FC740020547500205075002020410020C8
:10B1A8008C2100202F5600201476002020760020C5
:10B1B800A0760020D47500202441002034360020D9
:10B1C800B0370020EC3E0020E84600205C3C002020
:10B1D800503C002000000000683C00206F12833AB9
:10B1E800E87500201076002018500020E07A002032
:10B1F800B4EEE77AF1EE10FA8CBFF0EE676AF0EE83
:10B20800476AEC4B4A8DD3ED027A9FEDEB7A5342B5
:10B2180004EE103A76EE277AB8EEC44A66EE876AEC
:10B22800F4EEC47AF1EE10FA0AD407EE102AB8EE5A
:10B23800474AB4EEE74AF1EE10FA88BFB0EE674A23
:10B24800DE4ADFEDDD7A527824EE274A0AB9B1EEFC
:10B25800444A002841F0B486B7EE003AD84D2A781F
:10B26800002A02F05986D7499FEDD76AD1ED024AE4
:10B2780091ED017AD1ED037A66EEA44AE5EE074A2C
:10B28800E4EE274A63EE244AF4EEC64AF1EE10FAD9
:10B29800B4BFF0EE463AF0EE643A98BFB0EE646A96
:10B2A800012ACDED0A4A02F08486D1ED067AD1ED65
:10B2B800052A91ED077A66EEA77AE5EE227AE4EEA2
:10B2C800077A23EE277AB4EEC67AF1EE10FAB4EED6
:10B2D800E37A8CBFF0EE467AF0EE477AF1EE10FA98
:10B2E80098BFB0EE676AB4BFF0EE637AF0EE477AC3
:10B2F800022A8DED0B7A00F0DE8091ED0A7AD1ED0D
:10B30800092AD1ED0B3A26EE877AA5EE227AA4EE29
:10B31800237A23EE077AB4EEC67AF1EE10FAB4EE89
:10B32800E77A8CBFF0EE463AF0EE473AF1EE10FAC3
:10B3380098BFB0EE636AA8BFF0EE477A032A8DED96
:10B348000C7A00F0B88091ED0E7AD1ED0D2AD1ED8E
:10B358000F3A26EE877AA5EE227AA4EE237A23EE18
:10B36800077AB4EEC67AF1EE10FAB4EEE77A8CBF3B
:10B37800F0EE463AF0EE473AF1EE10FA98BFB0EE2A
:10B38800636AA8BFF0EE477A042A8DED0D7A00F0C3
:10B398009280D1ED123AD1ED112A91ED137A66EE31
:10B3A800A33AE5EE223AE4EE073A63EE233AF4EEE6
:10B3B800C63AF1EE10FAF4EEE73A8CBFB0EE467AF0
:10B3C800B0EE637AF1EE10FA98BFB0EE476AA8BF04
:10B3D800F0EE637A052ACDED0E3A6CD0D1ED163A2F
:10B3E800D1ED152A91ED177A66EEA33AE5EE223AE9
:10B3F800E4EE073A63EE233AF4EEC63AF1EE10FAB9
:10B40800F4EEE73A8CBFB0EE467AB0EE637AF1EE2E
:10B4180010FA98BFB0EE476AA8BFF0EE637A062A22
:10B42800CDED0F3A47D0D1ED1A3AD1ED192A91ED69
:10B438001B7A66EEA33AE5EE223AE4EE073A63EEAB
:10B44800233AF4EEC63AF1EE10FAF4EEE73A8CBF7E
:10B45800B0EE467AB0EE637AF1EE10FA98BFB0EE2D
:10B46800476AA8BFF0EE637A072ACDED103A22D0DA
:10B4780091ED1E7AD1ED1D2AD1ED1F3A26EE877A7D
:10B48800A5EE227AA3EE847A27EE037AB4EEC67A82
:10B49800F1EE10FAB4EEE77A8CBFF0EE466AF0EE01
:10B4A800476AF1EE10FA8DED117A98BFB0EE666A30
:10B4B800A8BFF0EE477A77EEC67AF7EE006AF4EEA8
:10B4C800E67AF1EE10FAC9ED4C7A43F3B08686EECF
:10B4D800A77A022ADDED0B7A64EE874A67EE877A4F
:10B4E800CDED0A4ACDED0B7A2DD0DDED0C7A67EE65
:10B4F800877A032ACDED0C7A25D0DDED0D7A67EE3B
:10B50800877A042ACDED0D7A1DD0DDED0E7A67EE2F
:10B51800877A052ACDED0E7A15D0DDED0F7A67EE24
:10B52800877A062ACDED0F7A0DD0DDED107A67EE19
:10B53800877A072ACDED107A05D0DDED117A27EE4E
:10B54800877A8DED117A2149096811F0805C01F044
:10B55800A982F6EE005AC9ED685A002A02F0D6848C
:10B568001B4B99ED656A1B491B4E1C781B4F99F9BB
:10B57800983199ED645AB6F90660C878DBF800107E
:10B58800D7ED004A0396BDEEC66A07EE103AB8F842
:10B598001A60134B079616EE107ABDEEC56A04F0D2
:10B5A800010E01F4805601F0100401F480010891A5
:10B5B8001B7817E0503C00206F12833AF83C0020BB
:10B5C800AD3D00205846002000000000A4370020B0
:10B5D8002F560020EC4800202078002054460020F8
:10B5E8003C520020D9ED616AD9ED627AB8EEC77A8B
:10B5F80016EE101A002840F0FB87002C41F0AF83AC
:10B60800D44C9DED0A5A94ED006AD34825EE866A1B
:10B61800A5EE076AB0EE675AA6EE265ABDEEC56AD1
:10B6280016EE10CA16EE106ABC45A8BF3E46614524
:10B63800C8BF0E4606EE106AB8EEC66A012A80ED4B
:10B64800006A00F0DC8094ED046A9DED0B5A25EE4B
:10B65800866AA5EE076AB0EE675AA6EE265ABDEED0
:10B66800C56A16EE10CA16EE106ABC45A8BF3E465B
:10B678006145C8BF0E4606EE106AB8EEC66A022AD1
:10B6880080ED016A00F0BB8094ED086A9DED0C5ACC
:10B6980025EE866AA5EE076AB0EE675AA6EE265A28
:10B6A800BDEEC56A16EE10CA16EE106ABC45A8BFF4
:10B6B8003E466145C8BF0E4606EE106AB8EEC66A39
:10B6C800032A80ED026A00F09A8094ED0C6A9DEDE1
:10B6D8000D5A25EE866AA5EE076AB0EE675AA6EE01
:10B6E800265ABDEEC56A16EE10CA16EE106ABC459B
:10B6F800A8BF3E466145C8BF0E4606EE106AB8EEC2
:10B70800C66A042A80ED036A79D094ED106A9DED2B
:10B718000E5A25EE866AA5EE076AB0EE675AA6EEBF
:10B72800265ABDEEC56A16EE10CA16EE106ABC455A
:10B73800A8BF3E466145C8BF0E4606EE106AB8EE81
:10B74800C66A052A80ED046A59D094ED146A9DED05
:10B758000F5A25EE866AA5EE076AB0EE675AA6EE7E
:10B76800265ABDEEC56A16EE10CA16EE106ABC451A
:10B77800A8BF3E466145C8BF0E4606EE106AB8EE41
:10B78800C66A062A80ED056A39D094ED186A9DEDDF
:10B79800105A25EE866AA5EE076AB0EE675AA6EE3D
:10B7A800265ABDEEC56A16EE10CA16EE106ABC45DA
:10B7B800A8BF3E466145C8BF0E4606EE106AB8EE01
:10B7C800C66A072A80ED066A19D094ED1C6A9DEDB9
:10B7D800115A65EE865AE7EE055AE6EEA57AFDEEB1
:10B7E800E77A17EE904AA742A8BF2746A142D8BFDA
:10B7F800394607EE901AF8EEE77AC0ED077ABEF1FF
:10B80800000F01F00280554A1268002A41F00A80B0
:10B81800534A127882B1287858B14F4E514F0024BC
:10B82800E0B23B68B6EC010A9847287801348442B4
:10B83800F6DB4D4A12689047029B1A78072A01F0F6
:10B8480081810025DBF80020510500F1F787474B7F
:10B858001A68120701F10080454A1278BAB14549C1
:10B86800B8F81A20B1F90610914210DC424A127851
:10B87800012A01F0B784192A01F0B4840E2A06D0EF
:10B88800082A04D03D4C0022A260C9F8402199F84A
:10B89800AA4124B13A4B1A88960741F0618499F875
:10B8A800B021002A41F0508098F81E60002E00F068
:10B8B8001C86022E01F0B983032E41F0B28398F85A
:10B8C8002010C1EB411001EB8001C90089B298F842
:10B8D8001F700237FFB2002A00F05F86002900F0CF
:10B8E8005C8628480668B1FBF6F10EB2A9F8E0615B
:10B8F800002F03F0648107EE906AF8EEE77AF7EE1E
:10B90800006A86EEA77A1D4C012FD9ED7D6AD4ED29
:10B91800007A77EEE67A67EE877AC9ED797A3DD0D4
:10B92800D4ED017AD9ED7E6A77EEE67A022F67EEDA
:10B93800877AC9ED7A7A31D0D4ED027AD9ED7F6A67
:10B9480077EEE67A032F67EE877AC9ED7B7A25D002
:10B958001AE000BF58460020C03C0020F4740020C4
:10B96800645500203052002038520020C440002086
:10B978002C02002020780020F83C0020EC3E00201B
:10B9880020410020E03C0020D4ED037AD9ED806A04
:10B9980077EEE67A67EE877AC9ED7C7A029B1978AA
:10B9A800092903F06582002E40F3A5859FB399ED20
:10B9B8007D7AD9ED797A77EE877A012FC9ED7D7A8C
:10B9C800C4ED007A21D099ED7E7AD9ED7A7A77EEB6
:10B9D800877A022FC9ED7E7AC4ED017A15D099EDE8
:10B9E8007F7AD9ED7B7A77EE877A032FC9ED7F7A54
:10B9F800C4ED027A09D0D9ED807A99ED7C7A77EE98
:10BA0800877AC9ED807AC4ED037A013F022FB8BF67
:10BA18000227FBB20693002A069B18BF0223CC4AD2
:10BA2800DFEDCC6A1168029A887817780A7807EEF1
:10BA3800902AF8EEE77AB0EE007A67EEA67AF4EE8E
:10BA4800C77AF1EE10FA40F3F186DFEDC36A37EEFC
:10BA5800C77AB0EE676AA7EE266AF0EE466A94EDFA
:10BA6800007A9FEDBE6A27EE066AF0EEC65A89EDA7
:10BA7800546AC9ED575A98B107EE100AB8EEC75A7A
:10BA88009FEDB47A66EE064A25EE075AB7EE007ABD
:10BA980037EE457A64EEA54AA4EE857A26EE076A63
:10BAA8009FEDAF7A4A7926EE877A27EE067ACAB1F1
:10BAB800DFEDA86A9FEDAB6A65EEA65A06EE902AFE
:10BAC800F8EEE66A66EEA56AF4EEC66AF1EE10FADA
:10BAD80001F34D82F7EE005A75EEE66A85EEA66A26
:10BAE80027EE067A0C2F9FEDA08ADFEDA06A01F001
:10BAF8000780B4EEC87AF1EE10FA98BFB0EE478A24
:10BB0800B4EEE68AF1EE10FAB8BFB0EE668A89EDB7
:10BB18004E8A002B00F0DC80B0EE007AF4EEC77A93
:10BB2800F1EE10FA05DD37EEC77ADFED8B6AE7EE46
:10BB3800267A94ED017ADFED896A27EE267AF0EE0F
:10BB4800C75A89ED557AC9ED585A98B106EE900A48
:10BB58009FED806AF8EEE66A27EE075A66EE866A77
:10BB6800B7EE006A36EE666A25EE255AA5EE266A15
:10BB780027EE067ADFED7A6A8A7967EEA67A67EEAB
:10BB8800877AAAB107EE102AB8EEC77A9FED716AD4
:10BB9800DFED746A27EE257A27EE067AB4EEE67AA8
:10BBA800F1EE10FA41F3E781DFED716A67EEA67AEC
:10BBB8000C2F00F07E87DFED6C6A9FED6C7AF4EE57
:10BBC800E67AF1EE10FA88BFF0EE667AF4EEC77AFC
:10BBD800F1EE10FAB8BFF0EE477A012BC9ED4F7AB3
:10BBE80076DD4B78DFED5B6A4A7A07EE903AF8EE3D
:10BBF800E77AB0EE007A67EEA67AF4EEC77AF1EE4D
:10BC080010FA05DD37EEC77ADFED536AE7EE267ADC
:10BC180094ED027ADFED516A27EE267AF0EEC75AE4
:10BC280089ED567AC9ED595A9AB106EE902A9FEDD8
:10BC3800496AF8EEE66A27EE075A66EE866AB7EEB4
:10BC4800006A36EE666A25EE255AA5EE266A27EEC4
:10BC5800067ADFED436ACA7967EEA67A67EE877AD5
:10BC6800FAB107EE102AB8EEC77A9FED3A6ADFED0F
:10BC78003D6A27EE257A27EE067AB4EEE67AF1EEEB
:10BC880010FA01F38681B5EEC07AF1EE10FA02F1EE
:10BC98006383B7EE006A36EE477AC6EE076A67EE48
:10BCA800A67A0C2F00F02487DFED2F6A9FED2F7AFC
:10BCB800F4EEE67AF1EE10FA88BFF0EE667AF4EE6A
:10BCC800C77AF1EE10FAB8BFF0EE477AC9ED507AAC
:10BCD800092F00F0DA8698F82140002C40F08F8672
:10BCE800002289F8B02112F013FC002840F01384D8
:10BCF800204B1B7823B9204B9B78002B41F04682C0
:10BD0800049805F05BFE029B1C78072C7EF42FAF8D
:10BD1800FBF730FE194B029A401B1478D880FEF7C7
:10BD280026BF99F86821002A3FF46AA9144A89F8BD
:10BD380068311288002A7FF45DA9124A124B1178E3
:10BD4800186881F0010105F059F8FFF759B900BFEB
:10BD5800284100200AD7233CD7A368416F12033B30
:10BD680000004843A4707D3F00C0F94400C0F9C4F6
:10BD78000000C84224450020F6770020D03D00206E
:10BD8800987600209A7600209C760020AC4A11789C
:10BD9800D9F81861AB4B9FEDAC7AF5005A1982EDD2
:10BDA800007A002978D0A948B0EE476AF0EE476AD1
:10BDB8000022F0EC017A013267EEA77A05EE902AAC
:10BDC800B4EEE77AF1EE10FAF8EEE55AB8BFB0EE45
:10BDD800677A8A4276EEA76AA7EEA56AE9D1F5EEF8
:10BDE800C06A5A19F1EE10FA82ED007A54DDC6EEF7
:10BDF800265A974A97490988F7EE007A75EEE75A66
:10BE0800D2ED007A65EEA77AFDEEE77A17EE902A72
:10BE1800812A42F309828A42A8BF0A4607EE902A7D
:10BE2800F8EEE77A8C4AA81902EB800292ED057ABF
:10BE3800D2ED003A92ED066A92ED014AD2ED046A1B
:10BE4800D2ED034A92ED025AA3EEA77AA4EE276A2E
:10BE580066EEC76AA7EE646ABDEEC77AE5EE276AA2
:10BE680017EE100A812882ED056AC2ED066A42F3D0
:10BE7800D8818142A8BF014607EE901AF8EEE77A0A
:10BE8800FCEEE77ACDED057ABDF8142059198A80C1
:10BE980016B9132F03F0B381152F41F033831D44D6
:10BEA8006E4BAA8823F81620D9F814416C4A01343D
:10BEB80082FB04321119E217C2EBA102C2EBC202E3
:10BEC800A41AC9F814416748D9F81C21049B664C88
:10BED80001682478C9F81C319A1A11440160002CB1
:10BEE80040F0D28007EE902A604DDFF89881604ECE
:10BEF800B8EEE78A05F5F07405F51377F5EC017AE5
:10BF08009AED070ADAF80832F8EEE77A204627EEC3
:10BF1800800A9847A4F1E000DAF828319847A4F19C
:10BF28007000DAF898319847D5F8EC00DAF8AC30B8
:10BF38009847D6ED007AA8EC010AE0EE087A243496
:10BF4800A742E6EC017AD9D1029B1C78072C7EF433
:10BF580007AEFBF70FFD029A404B1478049A801A3B
:10BF68001880FEF7FDBD99ED577AB1F90000D9EDBB
:10BF7800586AB1F902E03F4AF4EEC76A80EAE07312
:10BF88008EEAEE71A3EBE073F1EE10FAA1EBEE711D
:10BF9800B8BFF0EE476A8B42B8BF0B4607EE103ABF
:10BFA8001378B8EEC77A27EE097A002B00F057818C
:10BFB800314B93ED005AB5EEC05AF1EE10FA40F34A
:10BFC8006D852E4BD3ED004AF5EEC04AF1EE10FA1E
:10BFD80040F3648534EEC77A66EECA5A87EE246A5F
:10BFE800C5EE856AB7EE007AB4EEC76AF1EE10FACC
:10BFF80088BFB0EE476AB5EEC06AF1EE10FA76EE89
:10C00800876AB8BFB0EE4C6A66EE266AF4EEC76A75
:10C01800F1EE10FA88BFF0EE476AF5EEC06AF1EE6D
:10C0280010FAB8BFF0EE4C6A154B93ED007A67EE44
:10C03800877AA7EEA68AFEF750BE0122FEF7A8BDB2
:10C048009E380020943B0020000000001C200020A7
:10C05800A03800209C380020BC3A0020D03D0020A9
:10C06800932449921846002094380020A84D0020B7
:10C078001C460020F4750020F0750020F87500209B
:10C08800EC7500200C50002007EE902A9E4B9F4C28
:10C098009F49A04FCDF81490F8EEE78A039304F572
:10C0A800B875984600268946029BDAED077A1B7810
:10C0B800172B6DD094ED007AB8EEC78A082B28EEBE
:10C0C800278A07D1B0EE480A069328F04DFF069B51
:10C0D800A8F80000DBF8002092000BD5002E03F032
:10C0E8008283B0EE480ADAF8083205F17000984702
:10C0F800B0EE408AB0EE480ADAF82831A5F17000AF
:10C108009847DAF8983128469847029B1B78032B02
:10C11800B0EE408A37D0D4F8F000DAF8AC30B0EEA0
:10C12800480A9847D7ED007AA9EC010AE0EE287A88
:10C138000136032E05F1240508F1020804F1040470
:10C14800E7EC017AB0D1029BDDF814901C78FDE68B
:10C15800714B724A234493ED007AD2ED007A704B0A
:10C1680067EE277AF7EE006AF4EEE67AF1EE10FA57
:10C1780093ED007A88BFF0EE667A67EE877A27EE4D
:10C18800888AFEF7F9BE28F0EFFEA8F80000C2E79B
:10C1980094ED007A0AEB4602B8EEC78A128FA8F827
:10C1A800002028EE278A95E75E4BDFF8B0811A78E1
:10C1B800D4075CBFB8F81820A9F88C215A4A5B4C00
:10C1C8001288D4ED037A07EE102AB8EEC77AF4EE97
:10C1D800C77AF1EE10FA41F24786554C238807EEEC
:10C1E800103AB8EEC77AF4EEC77AF1EE10FAC1F257
:10C1F8000580504A504C92ED006AD4ED006A99F9D6
:10C208009821C9ED646A76EE665A012AC9ED626A18
:10C21800C9ED615A89ED656A01F0E884049BC9F8A3
:10C228009C31002437EEC77AFCEEE77A434D89ED5E
:10C23800687A17EE902AA9F88C21012295ED005A08
:10C2480089F898213E4A944241F23E863D4BD3ED0F
:10C25800007AD3ED013A93ED026AFEF735BF3A4B07
:10C2680093ED006AB4EEEA6AF1EE10FA40F17387D2
:10C27800F7EE005A75EEC65A3BEEC77A65EE8B5A52
:10C28800324BA7EE256A93ED007A26EE076AB5EEE3
:10C29800C06AF1EE10FA40F20184CAEE065AB7EE0F
:10C2A800007AB0EE476AA6EEE56AF0EE466AADE6B9
:10C2B800274AD2ED007AB0EEC87AB4EEE77AF1EE0A
:10C2C80010FA7EF79DAE234AD2ED007AB0EEED7AF1
:10C2D800B4EEE77AF1EE10FA7EF792AE1E4AD8ED88
:10C2E800007A92ED007AF0EEE77AF4EEC77AF1EE92
:10C2F80010FA7EF585AE01220499C9F86C1189F807
:10C308006821FEF760BE00BFD03D0020A84D002088
:10C318000C5000201C46002078210020E4750020E5
:10C32800E07500202F560020EC460020EC3E00204F
:10C33800EE460020B0370020D8460020F446002002
:10C348008FD003005C3C0020FC750020F0750020B5
:10C35800247600202076002028760020E07A00202D
:10C36800934C9448944B9549059326461B68029034
:10C3780003944F780478B6F906004FF47A71B1FB4C
:10C38800F3F3C3EB431603EB8603DE00B6B2B54204
:10C3980001F04E87DAF87CE0BAF93820DAF8603034
:10C3A8000EF1010107EE902A13440129CAF87C1006
:10C3B800CAF86030F8EEE77A01F04787DAED1B5AE1
:10C3C800DAED1D6A07EE101A37EEE56AB8EEC75ABD
:10C3D800012D86EE057A37EE257A77EEC77A8AED53
:10C3E8001C7AE7EE866A8AED1B7AF0EE667ACAED69
:10C3F8001E6ACAED1D6A02F08883DAF890E0BAF97D
:10C408003A20DAF864300EF1010107EE902A13445D
:10C418000129CAF89010CAF86430F8EEE77A01F0FA
:10C428002F87DAED205ADAED226A07EE101A37EE76
:10C43800E56AB8EEC75A012D86EE057A37EE257AF9
:10C4480077EEC77A8AED217AE7EE866A8AED207A56
:10C45800F0EE667ACAED236ACAED226A02F07D839D
:10C46800DAF8A4E0BAF93C20DAF868300EF10101F4
:10C4780007EE902A13440129CAF8A410CAF86830B4
:10C48800F8EEE77A01F01787DAED255ADAED276A30
:10C4980007EE101A37EEE56AB8EEC75A012D86EE98
:10C4A800057A37EE257A77EEC77A8AED267AE6EEB0
:10C4B800276A8AED257AF0EE667ACAED286ACAED0F
:10C4C800276A02F01583039BDFF81891D880BAF821
:10C4D800A820029B013A1C78AAF8A82005990022F6
:10C4E8004A608A60CA60FEF738BBA9F8E061002A92
:10C4F8003FF4F9AB324C0223FFF791BA314B324A81
:10C50800196812882A4BC96919805A8013B0BDEC82
:10C518000E8BBDE8F08F2D4C11F0B6FE6378022B20
:10C5280000F05086032B7FF4E3AB41F2B813E35CD1
:10C53800002B41F0568341F2A403E35C002B41F049
:10C548004B8341F2E803E35C002B41F0408341F266
:10C558002C13E35C002B3FF4CBAB1D4814F0E4FA3A
:10C56800FFF7C6BB1B4B1C4D1A7812F0010F2A7837
:10C5780040F02483002A00F01D85920017491848CE
:10C58800DFF864B0DFF8648028F01AFBFFF73BB9E6
:10C59800084B0293DFF84C9095E4B9F8E061013E4E
:10C5A80036B2002EA9F8E061A1DD054CFFF7FEB90F
:10C5B800D03D0020CC3D002008500020F44F002042
:10C5C800EC3E00203C7A0020182D00201057002057
:10C5D8003C6800202F560020AD3D00201C2D002077
:10C5E800C03C00201C20002018500020E07A0020C9
:10C5F800002C01F0A781BEF1000F42F0EF82C44C7D
:10C60800002B42F0278194ED006A9DED0A5AC1483B
:10C6180025EE866AFDEEE44AA5EE076AB0EE675A93
:10C62800A6EE265A14EE901ABDEEC56A16EE10EA6A
:10C6380016EE106ABE45A8BF3E467145C8BF0E46F5
:10C6480006EE106AB8EEC66A012A80ED006A00F0AC
:10C65800DF8094ED046A9DED0B5A25EE866AA5EEFF
:10C66800076AB0EE675AA6EE265ABDEEC56A16EE00
:10C6780010EA16EE106ABE45A8BF3E468E45B8BF02
:10C688000E4606EE106AB8EEC66A022A80ED016A06
:10C6980000F0BE8094ED086A9DED0C5A25EE866A7E
:10C6A800A5EE076AB0EE675AA6EE265ABDEEC56A31
:10C6B80016EE10EA16EE106ABE45A8BF3E468E4535
:10C6C800B8BF0E4606EE106AB8EEC66A032A80EDB9
:10C6D800026A00F09D8094ED0C6A9DED0D5A25EEDE
:10C6E800866AA5EE076AB0EE675AA6EE265ABDEE30
:10C6F800C56A16EE10EA16EE106ABE45A8BF3E4699
:10C708008E45B8BF0E4606EE106AB8EEC66A042A11
:10C7180080ED036A7CD094ED106A9DED0E5A25EEEB
:10C72800866AA5EE076AB0EE675AA6EE265ABDEEEF
:10C73800C56A16EE10EA16EE106ABE45A8BF3E4658
:10C748008E45B8BF0E4606EE106AB8EEC66A052AD0
:10C7580080ED046A5CD094ED146A9DED0F5A25EEC5
:10C76800866AA5EE076AB0EE675AA6EE265ABDEEAF
:10C77800C56A16EE10EA16EE106ABE45A8BF3E4618
:10C788008E45B8BF0E4606EE106AB8EEC66A062A8F
:10C7980080ED056A3CD094ED186A9DED105A25EE9F
:10C7A800866AA5EE076AB0EE675AA6EE265ABDEE6F
:10C7B800C56A16EE10EA16EE106ABE45A8BF3E46D8
:10C7C8008E45B8BF0E4606EE106AB8EEC66A072A4E
:10C7D80080ED066A1CD094ED1C6A9DED115A65EE39
:10C7E800865AE7EE055AE6EEA57AFDEEE77A17EEE9
:10C7F800904AA742A8BF2746A142D8BF394607EEAC
:10C80800901AF8EEE77AC0ED077A002A3EF4FBAFFB
:10C81800920041493F4828F0D3F9404A1268002A5B
:10C828003EF4F6AF1FF002F8FEF7F2BFF0EE676ACB
:10C83800FFF715B9B0EE665AFEF77DBCDAF80820A6
:10C84800002A3FF404A83649A1F14C009047354B23
:10C858001A6812077FF500A8334CD4ED027AB2EEBD
:10C868000E7AF0EEE76AF4EEC76AF1EE10FA41D5F7
:10C878002E4B1A8853073DD52D4A2E48B2F904206D
:10C88800B9F8A61180FB0230D217C2EBA002521AE7
:10C8980092B210B210F1B30FBCBF02F5B47210B26D
:10C8A800B328C4BFA0F5B47210B2234A2349127941
:10C8B8000978002A4FF6FF7218BF01220F077EF58C
:10C8C800CBAF1F4B196810FB02F2087E1D4992B2CC
:10C8D80010FB02F281FB02311144D217C2EB211284
:10C8E80007EE102AB8EEC77A77EEC77AC4ED027A57
:10C8F800FEF7B2BF0E4A0F49B2F9042081FB02319C
:10C90800D217C2EBA102A9F8A621FEF7A5BF00BF66
:10C9180058460020C03C00201C2D0020F474002044
:10C92800C84D0020C4400020EC3E002020410020DB
:10C93800D040002067666666BC370020F477002088
:10C94800244100208988888891489249D0F8EC00D1
:10C95800096844F62064A042A8BF2046B0F57A7F53
:10C96800B8BF4FF47A7080B211F0100FA9F8B20175
:10C97800DBF8001000F03D84CB0441F1CC85864BF8
:10C988001F687E8E7608854C854BD9F8B411D4ED96
:10C99800037AA3FB00308409642090FBF4F0142888
:10C9A800BDEEE77A09EB410EA8BF14200131884299
:10C9B800C9F8B41117EE10CADCBF0021C9F8B411C8
:10C9C80009EB4101AEF8B8C1B1F9B83107EE103A38
:10C9D800B8EEC77A77EEC77AFDEEE77ACDED037A3F
:10C9E800BDF90C3083EAE371A1EBE371B14201F3C5
:10C9F800ED866C4B4FF07E511960FEF755BF1E2136
:10CA08006448F5F771FE00283FF46AA9664B1A8856
:10CA180052063FF565A999F80422A24242F04582E0
:10CA2800604BD9ED827AD3ED016A99ED505ADFED6A
:10CA38005F5A9FED5F6A27EEC57A67EE887AA6EEA1
:10CA4800887AE5EE267AB4EEE57AF1EE10FA88BF38
:10CA5800B0EE657AB4EEC67AF1EE10FAF4EEE57A45
:10CA6800B8BFB0EE467AF1EE10FA88BFF0EE657AFC
:10CA7800F4EEC67AF1EE10FAB8BFF0EE467A89ED18
:10CA88004E7AC9ED507AFFF72BB9FDEEC87A4949BD
:10CA980017EE902A8E80CA80FFF71DB9DFED466A2F
:10CAA800FFF7C2BADBF8001048023EF552ADFEF7B8
:10CAB80054BD9FED3E7ADFED3E6A3E48F4EEC77AFC
:10CAC800F1EE10FA98BFB0EE677AFDEEE77AB4EEB1
:10CAD800E67AF1EE10FA17EE902AB8BFB0EE667A51
:10CAE800012B89ED4F7A42803FF77BA8FFF7F3B817
:10CAF800BDEEE77A2F4A17EE101A9180FFF7D4B8E7
:10CB0800B4EEC87AF1EE10FA98BFB0EE478ABDEEDF
:10CB1800C77AB4EEE68ADFF89CC0F1EE10FA17EE99
:10CB2800102AB8BFB0EE668A89ED4E8AACF80020AC
:10CB3800002B7EF4F1AFFFF7CEB8002B3EF460AACD
:10CB4800FEF73DBAFAF716FF029B1A491A78059BB9
:10CB5800072AA0EB030088807EF473AEFAF70AFF79
:10CB68000546FEF76FBEFAF705FF029A0799127895
:10CB7800104B0393401A012A588000F00E83072AAD
:10CB88007EF466AAFAF7F6FE0590FEF763BA00BFD0
:10CB980020030020A437002024410020EC3E002080
:10CBA800D34D6210040000202041002000C0F94449
:10CBB80000C0F9C4D03D002000000000002A00F0A9
:10CBC800F981D9ED583A99ED576AD9ED627AF34966
:10CBD80099ED617AD1ED005A99ED554AD9ED544A4B
:10CBE800EF4CF048F4EEC63AF3EE046AF1EE10FAB0
:10CBF80037EEA65A00F1808394ED026A26EE446A65
:10CC0800F0EE674AE6EE074AF4EEC54A34EEE66A05
:10CC1800F1EE10FA48BFB0EE656A012A80ED006AAD
:10CC280000F0C88194ED066A26EE446AF0EE674A81
:10CC3800E6EE074AF4EEC54A34EEE66AF1EE10FA7B
:10CC480048BFB0EE656A022A80ED016A00F0B28141
:10CC580094ED0A6A26EE446AF0EE674AE6EE074A61
:10CC6800F4EEC54A34EEE66AF1EE10FA48BFB0EECB
:10CC7800656A032A80ED026A00F09C8194ED0E6AD1
:10CC880026EE446AF0EE674AE6EE074AF4EEC54A35
:10CC980034EEE66AF1EE10FA48BFB0EE656A042A8F
:10CCA80080ED036A00F0868194ED126A26EE446AEC
:10CCB800F0EE674AE6EE074AF4EEC54A34EEE66A55
:10CCC800F1EE10FA48BFB0EE656A052A80ED046AF5
:10CCD80000F0708194ED166A26EE446AF0EE674A19
:10CCE800E6EE074AF4EEC54A74EEE66AF1EE10FA8B
:10CCF80048BFF0EE656A062AC0ED056A00F05A8161
:10CD0800D4ED1A6A66EEC46AF0EE674AE6EE874A20
:10CD1800B3EE046AF4EEC54A74EEC66AF1EE10FA90
:10CD280048BFF0EE656A072AC0ED066A00F0428146
:10CD3800D4ED1E6ADFF874B2DFF8748226EEC44AB6
:10CD4800E4EE077AF4EEC57A77EEC67AF1EE10FAD9
:10CD580048BFF0EE657AC0ED077AFEF754BD904CF7
:10CD68009DED0A5A94ED006ABEF1000F41F056811C
:10CD780025EE866A8B48A5EE076AB0EE675AA6EEDE
:10CD8800265ABDEEC56A16EE10EA16EE106ABE45C2
:10CD9800A8BF3E467145C8BF0E4606EE106AB8EEFB
:10CDA800C66A012A80ED006A3FF432AD94ED046A48
:10CDB8009DED0B5A25EE866AA5EE076AB0EE675A16
:10CDC800A6EE265ABDEEC56A16EE10EA16EE106AF1
:10CDD800BE45A8BF3E467145C8BF0E4606EE106A5E
:10CDE800B8EEC66A022A80ED016A3FF411AD94EDEF
:10CDF800086A9DED0C5A25EE866AA5EE076AB0EE24
:10CE0800675AA6EE265ABDEEC56A16EE10EA16EE69
:10CE1800106ABE45A8BF3E467145C8BF0E4606EE1D
:10CE2800106AB8EEC66A032A80ED026A3FF4F0ACD5
:10CE380094ED0C6A9DED0D5A25EE866AA5EE076AFB
:10CE4800B0EE675AA6EE265ABDEEC56A16EE10EA8F
:10CE580016EE106ABE45A8BF3E467145C8BF0E46CD
:10CE680006EE106AB8EEC66A042A80ED036A3FF43B
:10CE7800CFAC94ED106A9DED0E5A25EE866AA5EEAC
:10CE8800076AB0EE675AA6EE265ABDEEC56A16EED8
:10CE980010EA16EE106ABE45A8BF3E467145C8BFE7
:10CEA8000E4606EE106AB8EEC66A052A80ED046AD8
:10CEB8003FF4AEAC94ED146A9DED0F5A25EE866AE8
:10CEC800A5EE076AB0EE675AA6EE265ABDEEC56A09
:10CED80016EE10EA16EE106ABE45A8BF3E4671452A
:10CEE800C8BF0E4606EE106AB8EEC66A062A80ED7E
:10CEF800056A3FF48DAC94ED186A9DED105A25EE45
:10CF0800866AA5EE076AB0EE675AA6EE265ABDEE07
:10CF1800C56A16EE10EA16EE106ABE45A8BF3E4670
:10CF28007145C8BF0E4606EE106AB8EEC66A072AF3
:10CF380080ED066A3FF46CAC94ED1C6A9DED115AC5
:10CF480065EE865AE7EE055AE6EEA57AFDEEE77A33
:10CF580017EE904AA742A8BF2746A142C8BF0F466E
:10CF680007EE907AF8EEE77AC0ED077A4DE49FED88
:10CF78000E6AFEF7B5BDB5EEC07AF1EE10FA01F112
:10CF8800E781B7EE006A36EE477AC6EE076AFEF723
:10CF98000DBEDFED056AFEF782BE00BF54460020D5
:10CFA80058460020C03C00200000C842185000200D
:10CFB800E07A0020DFF838B3DFF83883FEF723BCC7
:10CFC800B5494A79002A3EF447A9B44A1278002A9A
:10CFD8003EF442A90B78B249DFEDB24A07EE903A27
:10CFE8000B88B8EE677A07EE902A06EE103AF8EE4C
:10CFF800E77AB8EE466A67EE277AB7EE007A87EEE8
:10D00800863AB4EEE43AF1EE10FA88BFB0EE643A2C
:10D01800B4EEC73AF1EE10FAB8BFB0EE473AFEF7F1
:10D028001DB9A1494988FEF752BCB9F8B21101F5FA
:10D038007A7189B2FEF74BBC9C49039107EE102A1E
:10D0480008461978B0F904009AED070AB9F81051A2
:10D05800B8EEC77AF7EE006A0022132986EE879A9F
:10D06800C9F80C2101F08C81914A924901EB85069F
:10D078000024C9F80041C9F8044167EE897A92EDA5
:10D08800001AD2ED053A92ED122A92ED173AD2ED36
:10D09800091AD2ED0E4A92ED016A92ED064A92ED16
:10D0A8000A7AD2ED0F5AD2ED132AD2ED186A92ED10
:10D0B800045AD2ED030A69EE288A29EE088AE1EEBD
:10D0C800273AA2EE283AE1EE884AA6EE274AE7EE8A
:10D0D800085A92ED167A92ED0D6A92ED021AD2ED87
:10D0E8000C1AC6ED003AE2EEA86A25EE635A27EE5E
:10D0F800437A92ED0B2AD2ED152AC6ED204AA0EE0E
:10D10800E34A26EE646AD2ED143A82ED054AA1EEAE
:10D11800275AF0EE477AE1EEE45AA2EE086AE2EE08
:10D12800C36AE3EEA87A82ED065AC2ED0E5A82ED82
:10D138000F6A86ED403AC2ED176AC2ED187AC9F84F
:10D148000841039B6A1C02F01F029880A9F810216D
:10D15800029BFDF7E9BC584B93ED006AFFF797B8BF
:10D16800564A9FED577AD2ED087AF4EEC77AF1EE77
:10D1780010FA00F2D0849FED537A534CD4ED037A21
:10D1880077EE877AC4ED037AFEF789BB04980DF031
:10D1980031FDFEF7B5BD454B0393FAF7EBFB4B4961
:10D1A800D9F87C2109680590821AC9F87C0103988E
:10D1B800511A8280C180FDF74DBFFAF7DBFB07905B
:10D1C800FDF7EDBCA3784FF0010A072B3EF690ADB2
:10D1D800DFE813F00F06270624050406A1058A05D3
:10D1E800940530053A4A927B002A3EF44BABFEF791
:10D1F8004EBBCC003FF5C0ABFEF756BBB9F88C412F
:10D20800944240F2D38499F8A441002C40F0A786B8
:10D21800304A314D92ED007AD5ED007A99F998218E
:10D22800C9ED647A77EE676A012AC9ED627AC9EDB9
:10D23800616A89ED657A01F0F487049BC9F89C312D
:10D24800264A9FED207A92ED005A89ED687A0122EC
:10D2580089F89821FEF7F6BF214B1B88002B40F078
:10D26800CB84204A204B1178186803F0C7FDD9F801
:10D278006C21049B9A1AFDF749BD1C4BD8ED007A26
:10D2880093ED007AF0EEE77AF4EEC77AF1EE10FA51
:10D298007DF7B6AEFDF7A6BEA8400020EA3E002006
:10D2A800D43E0020713DAA3F20330020D03D00200D
:10D2B800283B0020BC380020F0750020F0450020F5
:10D2C8008FC2753C00000000EC3E0020E03C0020CE
:10D2D800287E0020B0370020D8460020F4460020E1
:10D2E800987600209A7600209C76002028760020E8
:10D2F80018500020E07A002094ED016A26EE646A56
:10D30800B0EE674AA6EE074AB4EEC54A34EE666A3E
:10D31800F1EE10FA48BFB0EE656A012A80ED006AA6
:10D328003FF448AE94ED056A26EE646AB0EE674AAB
:10D33800A6EE074AB4EEC54A34EE666AF1EE10FA74
:10D3480048BFB0EE656A022A80ED016A3FF432AE4A
:10D3580094ED096A26EE646AB0EE674AA6EE074ABB
:10D36800B4EEC54A34EE666AF1EE10FA48BFB0EE84
:10D37800656A032A80ED026A3FF41CAE94ED0D6ADB
:10D3880026EE646AB0EE674AA6EE074AB4EEC54ACE
:10D3980034EE666AF1EE10FA48BFB0EE656A042A08
:10D3A80080ED036A3FF406AE94ED116A26EE646AD6
:10D3B800B0EE674AA6EE074AB4EEC54A34EE666A8E
:10D3C800F1EE10FA48BFB0EE656A052A80ED046AEE
:10D3D8003FF4F0AD94ED156A26EE646AB0EE674A44
:10D3E800A6EE074AB4EEC54A74EE666AF1EE10FA84
:10D3F80048BFF0EE656A062AC0ED056A3FF4DAAD6B
:10D40800D4ED196A66EEE46AB0EE674AA6EE874A7A
:10D41800B3EE046AB4EEC54A74EE466AF1EE10FA49
:10D4280048BFF0EE656A072AC0ED066A3FF4C2AD50
:10D43800D4ED1D6ADFF898B2DFF8988266EEE44A08
:10D44800E4EE877AF4EEC57A77EEC67AF1EE10FA52
:10D45800B8BFF0EE657AC0ED077AFEF7D4B9914D02
:10D46800D9ED017A99ED006A29886A6977EEA77A79
:10D47800F0EE006AB0EE677AA6EE267A4D1E09EB4A
:10D48800C501D6EE267A08391032F6EE003A27EEB4
:10D49800237A67EEA37A89ED207AC9ED217ADFF83D
:10D4A8001C924E4609F1800091ED027A91ED036AD3
:10D4B800D6ED036AD6ED027A52ED014A12ED025A10
:10D4C80037EE674A76EEC65A77EE277AE4EE845A44
:10D4D800013DA1F10801E5EE047A06F1080602F122
:10D4E800080236EE267A00F10800E4EE877AE5EEC7
:10D4F800475A67EEA37A25EEA37AC0ED007A80ED4D
:10D50800017AD1D1142F7EF4D1ACFAF733FA039A09
:10D51800654B801A5880D9F81441FEF7C7BCD9F872
:10D528001881B9F810E1614ACEF12003DBB20EEBA5
:10D53800481602EB86069A0801F06E86013215013C
:10D548005B485C4906EB050C06F1100212ED024A35
:10D5580012ED035A12ED016A12ED047A50ED024AF7
:10D5680050ED035A50ED016A50ED047A64EE244AF6
:10D5780065EE255A66EE266A67EE277A10329445DC
:10D5880041ED024A41ED035A41ED016A41ED047A49
:10D5980000F1100001F11001D8D14748A5F11001A0
:10D5A8000E4400EB010C494413F0030209D0B6EC19
:10D5B800017AFCEC017A67EE277A013AE1EC017A0C
:10D5C800F5D1BEF1000F40F05487142F7EF46EACF5
:10D5D800FAF7D0F9039A344BD9F81441801A5880D5
:10D5E800FEF764BC2F4D3548AA68A98926F0E2FAEF
:10D5F800029B1F78142F01F07686D9F81441013464
:10D60800C9F814412CE7D9F818412D492D482E4B5B
:10D61800E200114414448A88196800EE102A643A1A
:10D62800C82AA8BFC822782AB8BF782207EE902A4D
:10D63800B8EEC07AF8EEE77A00EB840477EE670A72
:10D6480077EE876A67EE877A20EEA67AB8EE400A08
:10D65800C7EE870A2046D4F81880E669256A94ED53
:10D66800058A23F0ADF9029B84ED058A1F78C4F87A
:10D678001880142FE661256201F03F86D9F8182139
:10D688001249D9F81441013281FB0213A3EBE27865
:10D6980008EB4803A2EB03080134C9F81881C9F85C
:10D6A80014413EE7A4380020D03D0020BC380020BB
:10D6B8004C3A00202C2000203C3A00201C2000205E
:10D6C800943B0020884F002008500020565555559F
:10D6D80018500020E07A0020954D29886B684FEAA1
:10D6E80051084FEA88005FEAD10E09EB000209EB06
:10D6F800810400F0A18000F110010EF1010E8D4EA1
:10D7080002EB0E1E2144103203F1100704F1100041
:10D7180050ED032A50ED043A16ED043A16ED032AAB
:10D7280050ED026A10ED016A16ED020A16ED018A43
:10D7380011ED044A11ED035A52ED044A52ED035A11
:10D7480012ED027A52ED017A51ED020A11ED011A39
:10D7580073EE238A72EE221A46ED048A46ED031A06
:10D7680070EE268A78EE061A46ED028A46ED011A10
:10D7780074EE848A75EE851A42ED048A42ED031A26
:10D7880077EE208A77EE811A42ED028A42ED011A7D
:10D7980073EE633A75EE655A17ED035A32EE623A44
:10D7A80074EE644A65EE631A17ED044A23EE052AFF
:10D7B80064EE652AE3EE041A1032964524EE843AA4
:10D7C800A3EE842A06F1100607F11007A5EE853AA4
:10D7D80000F1100001F11001E4EE852A40ED071A6E
:10D7E80000ED082A01ED073A41ED082A57ED055AE0
:10D7F80017ED065A70EE666A38EE466A30EEC77A5A
:10D8080071EE677A26EE253A65EEE63A25EE674A26
:10D8180067EE054AE6EE053AA6EE853AA7EE254AF2
:10D82800E7EEA54A00ED063A40ED053A01ED064A55
:10D8380041ED054A7FF46CAF1FFA88F81A46414655
:10D848003D4822F0DDFD6A684146204622F0D8FDB9
:10D85800029B1A78142A7FF45EAE56E6DFF8E08061
:10D8680098F800108E0801F0C085344D06F1010CBF
:10D878004FEA4C1C05EB0C0E05F12002A5F17000D7
:10D8880012ED076A52ED056A12ED037A52ED017A3C
:10D8980052ED025A12ED084A52ED064A12ED045AA8
:10D8A80026EE066A66EEA66A27EE077A67EEA77A7C
:10D8B800A4EE046A20329645E4EEA46A00F1100052
:10D8C800A5EE057AE5EEA57AF1EEC65AB1EEE66A5E
:10D8D800F1EEC76AB1EEE77A40ED085A00ED076A43
:10D8E80040ED066A00ED057ACAD1ACF120022A445F
:10D8F80009EB061611F0030018BF08320FD052EDDD
:10D90800017A12ED027A67EEA77A0138E7EE077A14
:10D9180002F10802B1EEE77AA6EC017AEFD1142FF2
:10D9280001F0D3840134C9F81441FEF731BA00BFBD
:10D93800A43800202C2000201C2000209C2000203F
:10D948009E380020BD4C002B40F0FC8594ED006A09
:10D958009DED0A5ABA4825EE866AFDEEE44AA5EE20
:10D96800076AB0EE675AA6EE265A14EE901ABDEE74
:10D97800C56A16EE10CA16EE106ABC45A8BF3E4628
:10D988006145C8BF0E4606EE106AB8EEC66A012A9F
:10D9980080ED006A3DF433AF94ED046A9DED0B5AB7
:10D9A80025EE866AA5EE076AB0EE675AA6EE265AF5
:10D9B800BDEEC56A16EE10CA16EE106ABC45A8BFC1
:10D9C8003E468C45B8BF0E4606EE106AB8EEC66AEB
:10D9D800022A80ED016A3DF412AF94ED086A9DEDCC
:10D9E8000C5A25EE866AA5EE076AB0EE675AA6EECF
:10D9F800265ABDEEC56A16EE10CA16EE106ABC4568
:10DA0800A8BF3E468C45B8BF0E4606EE106AB8EE73
:10DA1800C66A032A80ED026A3DF4F1AE94ED0C6A01
:10DA28009DED0D5A25EE866AA5EE076AB0EE675A97
:10DA3800A6EE265ABDEEC56A16EE10CA16EE106A94
:10DA4800BC45A8BF3E468C45B8BF0E4606EE106AD8
:10DA5800B8EEC66A042A80ED036A3DF4D0AE94EDB0
:10DA6800106A9DED0E5A25EE866AA5EE076AB0EE9D
:10DA7800675AA6EE265ABDEEC56A16EE10CA16EE0D
:10DA8800106ABC45A8BF3E468C45B8BF0E4606EE98
:10DA9800106AB8EEC66A052A80ED046A3DF4AFAE96
:10DAA80094ED146A9DED0F5A25EE866AA5EE076A75
:10DAB800B0EE675AA6EE265ABDEEC56A16EE10CA33
:10DAC80016EE106ABC45A8BF3E468C45B8BF0E4648
:10DAD80006EE106AB8EEC66A062A80ED056A3DF4BD
:10DAE8008EAE94ED186A9DED105A25EE866AA5EE65
:10DAF800076AB0EE675AA6EE265ABDEEC56A16EE5C
:10DB080010CA16EE106ABC45A8BF3E468C45B8BF81
:10DB18000E46FDF752BEF0EEE76AB7EE005A35EE54
:10DB2800665A9FED484ADFED485A9FED486A9FEDD7
:10DB3800487A99ED6B0AF1EEC54AE6EE845AF5EE9D
:10DB4800C07AA6EEA56AF1EE10FAA6EE867A48BF6C
:10DB5800DFED407A27EE247A48BF37EEC77A27EE02
:10DB6800000A27F001FAB0F5617F00F34A8607EE54
:10DB7800900AF8EEE76ADFED387A66EEA76A07EEF4
:10DB8800904ABDEEE67AF8EEE77A17EE102A2032D0
:10DB9800402A41F28C849FED310A27F0E5F900B262
:10DBA80007EE900AB8EEE77AFFF7E7BA2C4A02F1D7
:10DBB800500403E00432944200F0D1811378262BFC
:10DBC800F8D19578D3789D42F4D2FFF71CBB25484D
:10DBD80012F0AAFFFEF7BBBC234812F0A5FFFEF720
:10DBE800B0BC224812F0A0FFFEF7A5BCD9F89C41B2
:10DBF800049B1C1BFEF716BB1D494B69002B3DF40B
:10DC080085A81C481C4B008893FBF0F00B684FF06C
:10DC1800010E186081F811E0FDF778B8174B0093F2
:10DC28000320A070302305221549164813F02AFC5A
:10DC3800FEF75EB803236370FEF75AB85846002013
:10DC4800C03C0020306E99BC2716983D843459BEDC
:10DC5800A40DC93FDB0F4940D06D393A00000000E0
:10DC680084340020F8670020B4670020C8680020CA
:10DC7800A0760020B876002020A1070095000208B1
:10DC8800A48B03088068002023690622652BA270F4
:10DC980034D92278032A14BF6FF0FF026FF07F0295
:10DCA800A3F1650303EA020303F1010314BF4FF470
:10DCB800807280229A42236120D23A68E768023251
:10DCC80003EB0708904581F00285C34A6760D16F6E
:10DCD800C4F80880490203FB01F30521176042F8E4
:10DCE8001C3C42F8183CA170A268BC4901200FF006
:10DCF80031FF012841F0E1840623A3700021B848D0
:10DD08000FF0F0FE012841F0D884A3780133DBB28C
:10DD1800A370FFF75ABA2278237DB24FDFF8BC927E
:10DD2800032A14BF4FF480784FF08008002B41D0AD
:10DD3800012BFBD1AC4B62681968386800234FEAA5
:10DD4800412E4FF0FF31B1FBFEF112EB010B43F115
:10DD5800000C0021614500F1020008BF584538BF9A
:10DD680083465A46A149022010F026F8032801F2FA
:10DD7800668201A353F820F0F9BC000891DD000881
:10DD8800F9BC000891DD00086268A3682669991A41
:10DD9800B14284BFE260216103283FF475AF0133CB
:10DDA800B3FBF8F208FB12320AB143449B1A002273
:10DDB800636022753A684946023200200FF0FCFF82
:10DDC800032801F23C8201A353F820F0F9BC0008B3
:10DDD80065DE0008F9BC000891DC000841F2701308
:10DDE800E35C002B3DF484AF7D4812F09DFEFDF707
:10DDF8007FBF00230AAE3146184609220FF032FDD4
:10DE080001287DF475AF0A9B93F8FE21552A01F08D
:10DE1800198241F2B41202210123A1546370FDF763
:10DE280067BF0AAE41F2FC173146E05900230922C8
:10DE38000FF018FD01287DF45BAF00230A9A2370C8
:10DE4800B2F80B30B3F5007F01F0D48341F2B4127D
:10DE580003210123A1546370FDF74ABF636884F866
:10DE680014A00133A36065E7614A624CD2ED006AF1
:10DE7800614A94ED006A1278C9ED646A89ED656AB1
:10DE8800002A00F0F18276EE665A99F99821C9EDD8
:10DE9800615A0132C9ED626A00F09486049BC9F8A0
:10DEA8009C31002437EE677AFCEEE77A534D89ED12
:10DEB800687A17EE902AA9F88C21FF2295ED005A6E
:10DEC80089F89821FEF7BEB9DFED4D7A4D4B99EDF3
:10DED800687AC3ED007AC3ED017AC3ED027A4A4B42
:10DEE800B0EE676AF0EE673A1968FDF7EDB8F9F732
:10DEF80041FD029B03901F78142F05BF434BD9F8AF
:10DF08001441D9F814411C80FCF716BE404B1C780C
:10DF180004F0010EFDF773BC3E49DFED3F7A096856
:10DF2800C9ED4C7A11F0805C40F05E84DBF800109B
:10DF380011F4800C00F0F5824FF0000CB6EE007A78
:10DF480067EE877AF4EEE57AF1EE10FAC8BFF0EEE4
:10DF5800675A40F34984C9ED685AFDF7FEBA244A66
:10DF6800244CD2ED007A244A94ED007A1278C9ED57
:10DF7800647A89ED657A002A00F0228477EE676A70
:10DF880099F99821C9ED616A0132C9ED627A00F008
:10DF98006987049BC9F89C3100249FED197A174DB5
:10DFA80089ED687AFF2295ED005A89F89821FEF7E5
:10DFB80049B973EEC67AB7EE007AF4EEC77AF1EE95
:10DFC80010FAC9ED4C7A41F3328184EEA77A8DEDCF
:10DFD8000A7AFDF7B8BA00BFA468002014570020D9
:10DFE8008068002018690020206900201857002048
:10DFF80034360020DC4600203C520020F046002049
:10E00800000000005C3C002024410020D03D00209E
:10E018002F560020A437002000000080002E00F0BA
:10E02800D58725EE866ACE48A5EE076AB0EE675A10
:10E03800A6EE265ABDEEC56A16EE10EA16EE106A6E
:10E04800BE45A8BF3E467145C8BF0E4606EE106ADB
:10E05800B8EEC66A012A80ED006A3DF4D4AB94EDAF
:10E06800046A9DED0B5A25EE866AA5EE076AB0EEA6
:10E07800675AA6EE265ABDEEC56A16EE10EA16EEE7
:10E08800106ABE45A8BF3E467145C8BF0E4606EE9B
:10E09800106AB8EEC66A022A80ED016A3DF4B3AB95
:10E0A80094ED086A9DED0C5A25EE866AA5EE076A7E
:10E0B800B0EE675AA6EE265ABDEEC56A16EE10EA0D
:10E0C80016EE106ABE45A8BF3E467145C8BF0E464B
:10E0D80006EE106AB8EEC66A032A80ED026A3DF4BD
:10E0E80092AB94ED0C6A9DED0D5A25EE866AA5EE6D
:10E0F800076AB0EE675AA6EE265ABDEEC56A16EE56
:10E1080010EA16EE106ABE45A8BF3E467145C8BF64
:10E118000E4606EE106AB8EEC66A042A80ED036A57
:10E128003DF471AB94ED106A9DED0E5A25EE866AAA
:10E13800A5EE076AB0EE675AA6EE265ABDEEC56A86
:10E1480016EE10EA16EE106ABE45A8BF3E467145A7
:10E15800C8BF0E4606EE106AB8EEC66A052A80EDFC
:10E16800046A3DF450AB94ED146A9DED0F5A25EE08
:10E17800866AA5EE076AB0EE675AA6EE265ABDEE85
:10E18800C56A16EE10EA16EE106ABE45A8BF3E46EE
:10E198007145C8BF0E4606EE106AB8EEC66A062A72
:10E1A80080ED056A3DF42FAB94ED186A9DED105A89
:10E1B80025EE866AA5EE076AB0EE675AA6EE265ADD
:10E1C800BDEEC56A16EE10EA16EE106ABE45A8BF87
:10E1D8003E467145C8BF0E4606EE106AB8EEC66ADE
:10E1E800072A80ED066A3DF40EAB94ED1C6A9DED9E
:10E1F800115A65EE865AE5EE075AE6EEA57AFDEE67
:10E20800E77A17EE902A9742A8BF17469142D8BFDF
:10E21800394607EE901AF8EEE77AC0ED077AFDF76F
:10E22800F2BA8222FDF732BEDFED4E7AFDF7FABD73
:10E23800BAF93830CAF8202007EE903A0122F8EEF1
:10E24800E77ACAF86030CAF87C200023012DCAEDAD
:10E258001C7ACAED1B7ACAF8743001F01881B542ED
:10E268007EF4CBA8BAF93A30CAF8643007EE903A8F
:10E2780000220123F8EEE77ACAF82420CAF8903081
:10E288000023012DCAED217ACAED207ACAF8883018
:10E2980001F0F980B5427EF4E3A8BAF93C30CAF837
:10E2A800683007EE903A00220123F8EEE77ACAF8C0
:10E2B8002820CAF8A4300023012DCAED267ACAED19
:10E2C800257ACAF89C307EF4FEA89FED278A032C95
:10E2D80038D04FB107EE907AF8EEE77AF4EEC87AC4
:10E2E800F1EE10FA01F17E81204ADFF89090039B4D
:10E2F8001168DAF86820D88099F8200102EB5602F4
:10E3080092FBF6F60022CAF828608A620A63CA629B
:10E3180028B1174A126832F480637EF4D8A8154AE7
:10E32800126812F4003241F05580134C1146A35C78
:10E33800012B02F10C0200F07D8501311829F6D17C
:10E34800FEF7C5B8B0EE480A26F00EFE00B2C0E7E8
:10E35800F7EE006AFDF72ABCF7EE006AFDF79FBCEE
:10E36800C03C002000000243000000003C7A00206E
:10E378001C410020F42F0020DC7503081C2000201D
:10E388006D4C6E4E94ED004A94ED057AD4ED014A39
:10E3980094ED066AD4ED046A94ED035AD4ED025A5A
:10E3A80067EE897A06EB8502A4EE277AA4EEA76ABF
:10E3B80066EEC76AA5EE476AE5EEA76A20EE070A89
:10E3C80084ED056AC4ED066A82ED007A29EE088AB2
:10E3D80026F0CAFD69EE288AD4ED0E5AD4ED176AE4
:10E3E80094ED091AD4ED121A94ED0F5A94ED187A97
:10E3F80094ED0A2AD4ED132A94ED0D6AD4ED167A19
:10E4080094ED0C3AD4ED0B3A94ED154AD4ED144A38
:10E41800E1EE085A002206EB8501E8EEA16A00B297
:10E42800C9F80021A2EE085AC9F80421C9F8082140
:10E43800A8EEA27A26EE656A67EEE67AA3EE655A3A
:10E44800A3EE886AA6EEC47AE8EEA47A84ED0E5AA2
:10E45800C1ED205A84ED0F6AC1ED406A84ED177A48
:10E46800C4ED187AFEF76DBE76EEC65AF0EE466A2F
:10E478000BE59E00314B03EBC8185FEA9E0300EBE7
:10E48800060C4E4401F0598001331B0108EB0305CB
:10E4980008F110020CF1100006F1100112ED024A09
:10E4A80012ED035A12ED016A12ED047A50ED024A98
:10E4B80050ED035A50ED016A50ED047A64EE244A97
:10E4C80065EE255A66EE266A67EE277A103295427F
:10E4D80041ED024A41ED035A41ED016A41ED047AEA
:10E4E80000F1100001F11001D8D1103B98440CEB59
:10E4F80003001E441EF0030E3FF467A8B8EC017A2F
:10E50800F0EC017A67EE277ABEF1010EE6EC017AAB
:10E51800F4D1FFF75AB80A4B1F68B7F93260FEF713
:10E5280032BAB6EE007AF4EEC75AF1EE10FA3FF7B7
:10E5380005ADFDF712B800BF283B0020BC3800200D
:10E548002441002094ED006A9DED0A4ABA4825EE60
:10E55800866AFDEEE43AA4EE076AB0EE674AA6EED4
:10E56800264A13EE901AB4EEC45AF1EE10FAB0EE41
:10E57800446A88BFB0EE646ABDEEC66A16EE10CA79
:10E5880016EE106ABC45A8BF3E466145C8BF0E4698
:10E5980006EE106AB8EEC66A012A80ED006A3DF4FC
:10E5A8002EA994ED046A9DED0B4A25EE866AA4EE29
:10E5B800076AB0EE674AA6EE264AB4EEC45AF1EEF0
:10E5C80010FAB0EE446A88BFB0EE646ABDEEC66A5F
:10E5D80016EE10CA16EE106ABC45A8BF3E468C451A
:10E5E800B8BF0E4606EE106AB8EEC66A022A80ED7B
:10E5F800016A3DF404A994ED086A9DED0C4A25EEE4
:10E60800866AA4EE076AB0EE674AA6EE264AB4EE1A
:10E61800C45AF1EE10FAB0EE446A88BFB0EE646AEC
:10E62800BDEEC66A16EE10CA16EE106ABC45A8BF43
:10E638003E468C45B8BF0E4606EE106AB8EEC66A6E
:10E64800032A80ED026A3DF4DAA894ED0C6A9DED88
:10E658000D4A25EE866AA4EE076AB0EE674AA6EE72
:10E66800264AB4EEC45AF1EE10FAB0EE446A88BFF6
:10E67800B0EE646ABDEEC66A16EE10CA16EE106AEF
:10E68800BC45A8BF3E468C45B8BF0E4606EE106A8C
:10E69800B8EEC66A042A80ED036A3DF4B0A894ED8A
:10E6A800106A9DED0E4A25EE866AA4EE076AB0EE62
:10E6B800674AA6EE264AB4EEC45AF1EE10FAB0EE56
:10E6C800446A88BFB0EE646ABDEEC66A16EE10CA28
:10E6D80016EE106ABC45A8BF3E468C45B8BF0E462C
:10E6E80006EE106AB8EEC66A052A80ED046A3DF4A3
:10E6F80086A894ED146A9DED0F4A25EE866AA4EE6D
:10E70800076AB0EE674AA6EE264AB4EEC45AF1EE9E
:10E7180010FAB0EE446A88BFB0EE646ABDEEC66A0D
:10E7280016EE10CA16EE106ABC45A8BF3E468C45C8
:10E73800B8BF0E4606EE106AB8EEC66A062A80ED25
:10E74800056A3DF45CA894ED186A9DED104A25EE23
:10E75800866AA4EE076AB0EE674AA6EE264AB4EEC9
:10E76800C45AF1EE10FAB0EE446A88BFB0EE646A9B
:10E77800BDEEC66A16EE10CA16EE106ABC45A8BFF2
:10E788003E468C45B8BF0E4606EE106AB8EEC66A1D
:10E79800072A80ED066A3DF432A894ED1C6A9DEDC7
:10E7A800114A65EE865AE7EE045AE6EEA57AB4EE0B
:10E7B800E75AF1EE10FAC8BFF0EE647AFDF70FB829
:10E7C80077EEC76AF0EE477AFFF7DABBBB8E9FEDAC
:10E7D8001B7A07EE903AF8EEE77A194B67EE877ADC
:10E7E800C3ED007AFDF760B8B7EE007A77EE677A86
:10E7F800F4EEE75AF1EE10FA88BFF0EE675AFFF729
:10E80800AABB07EE904ADFED0F6AF8EEE77A66EEEC
:10E81800A65A9FED0D5A9FED0D6A9FED0D7AA5EE54
:10E82800856A26EEA55AA5EE867AE5EE076A26EEF3
:10E83800A70AFFF7B2B900BFC03C00206F12833AA5
:10E848000400002084F9223F92E741B99730083C40
:10E8580015A82ABE94ED006A9DED0A4ADC4825EE0B
:10E86800866AFDEEE43AA4EE076AB0EE674AA6EEC1
:10E87800264A13EE906AB4EEC45AF1EE10FAB0EEDE
:10E88800446A88BFB0EE646ABDEEC66A16EE10EA46
:10E8980016EE101ABE45A8BF39467645C8BF3146A0
:10E8A80006EE101AB8EEC66A012A80ED006A3DF439
:10E8B800AFAF94ED046A9DED0B4A25EE866AA4EE8F
:10E8C800076AB0EE674AA6EE264AB4EEC45AF1EEDD
:10E8D80010FAB0EE446A88BFB0EE646ABDEEC66A4C
:10E8E80016EE10EA16EE101ABE45A8BF3946B64510
:10E8F800B8BF314606EE101AB8EEC66A022A80ED95
:10E90800016A3DF485AF94ED086A9DED0C4A25EE49
:10E91800866AA4EE076AB0EE674AA6EE264AB4EE07
:10E92800C45AF1EE10FAB0EE446A88BFB0EE646AD9
:10E93800BDEEC66A16EE10EA16EE101ABE45A8BF5E
:10E948003946B645B8BF314606EE101AB8EEC66A63
:10E95800032A80ED026A3DF45BAF94ED0C6A9DEDED
:10E968000D4A25EE866AA4EE076AB0EE674AA6EE5F
:10E97800264AB4EEC45AF1EE10FAB0EE446A88BFE3
:10E98800B0EE646ABDEEC66A16EE10EA16EE101A0C
:10E99800BE45A8BF3946B645B8BF314606EE101A7F
:10E9A800B8EEC66A042A80ED036A3DF431AF94EDEF
:10E9B800106A9DED0E4A25EE866AA4EE076AB0EE4F
:10E9C800674AA6EE264AB4EEC45AF1EE10FAB0EE43
:10E9D800446A88BFB0EE646ABDEEC66A16EE10EAF5
:10E9E80016EE101ABE45A8BF3946B645B8BF31461F
:10E9F80006EE101AB8EEC66A052A80ED046A3DF4E0
:10EA080007AF94ED146A9DED0F4A25EE866AA4EED1
:10EA1800076AB0EE674AA6EE264AB4EEC45AF1EE8B
:10EA280010FAB0EE446A88BFB0EE646ABDEEC66AFA
:10EA380016EE10EA16EE101ABE45A8BF3946B645BE
:10EA4800B8BF314606EE101AB8EEC66A062A80ED3F
:10EA5800056A3DF4DDAE94ED186A9DED104A25EE89
:10EA6800866AA4EE076AB0EE674AA6EE264AB4EEB6
:10EA7800C45AF1EE10FAB0EE446A88BFB0EE646A88
:10EA8800BDEEC66A16EE10EA16EE101ABE45A8BF0D
:10EA98003946B645B8BF314606EE101AB8EEC66A12
:10EAA800072A80ED066A3DF4B3AE94ED1C6A9DED2D
:10EAB800114A65EE865AE7EE045AE6EEA57AB4EEF8
:10EAC800E75AF1EE10FAC8BFF0EE647AFDEEE77A85
:10EAD80017EE901A8F42A8BF0F468E42D8BF3E4607
:10EAE80007EE906AF8EEE77AC0ED077AFDF78DBE7B
:10EAF80001297FF7EAAB07EE10EAB8EEC77AC7EE4E
:10EB0800876AB1EEE68AFFF7E2BB012940F3BF84CA
:10EB180007EE10EAB8EEC77AC7EE876AB1EEE68A62
:10EB2800032C14D04FB107EE907AF8EEE77AF4EEA2
:10EB3800C87AF1EE10FA00F15585DAF8603003EB87
:10EB4800560393FBF6F3CAF82030FFF788BBB0EE04
:10EB5800480A26F009FA00B2E4E7012940F3938451
:10EB680007EE10EAB8EEC77AC7EE876AB1EEE68A12
:10EB7800032C14D04FB107EE907AF8EEE77AF4EE52
:10EB8800C87AF1EE10FA00F12D85DAF8643003EB5B
:10EB9800560393FBF6F3CAF82430FFF77BBBB0EEBD
:10EBA800480A26F0E1F900B2E4E70A494A69002A6E
:10EBB8003CF478A90A6813604B74FCF773B9064CE7
:10EBC800FCF7ECBED9F89C41049B1C1BFFF76AB903
:10EBD800C03C0020A0760020EC3E0020002E00F073
:10EBE800A483E94C9DED0A4A94ED006A25EE866AF5
:10EBF800A4EE076AB0EE674AA6EE264AB0EE446A6B
:10EC080033B1B4EE445AF1EE10FAC8BFB0EE646AFC
:10EC1800FDEEE44ABDEEC66A14EE906A16EE101ACE
:10EC28008E4214EE90EA00F3D984B942A8BF39465F
:10EC380006EE101AD548B8EEC66A012A80ED006AB9
:10EC48003CF4E1AD94ED046ADDED0B4A25EE866AED
:10EC5800A4EE876AF0EE674AE6EE264AB0EE646AEA
:10EC6800002B00F0B184B4EEE45AF1EE10FA40F350
:10EC7800AB843146B942A8BF394606EE101AB8EE41
:10EC8800C66A022A80ED016A3CF4BDAD94ED086ABB
:10EC9800DDED0C4A25EE866AA4EE876AF0EE674A37
:10ECA800E6EE264AB0EE646A002B00F08384B4EEE8
:10ECB800E45AF1EE10FA40F37D843146B942A8BF18
:10ECC800394606EE101AB8EEC66A032A80ED026AC3
:10ECD8003CF499AD94ED0C6ADDED0D4A25EE866A9B
:10ECE800A4EE876AF0EE674AE6EE264AB0EE646A5A
:10ECF800002B00F05584B4EEE45AF1EE10FA40F31C
:10ED08004F843146B942A8BF394606EE101AB8EE0C
:10ED1800C66A042A80ED036A3CF475AD94ED106A66
:10ED2800DDED0E4A25EE866AA4EE876AF0EE674AA4
:10ED3800E6EE264AB0EE646A002B00F02784B4EEB3
:10ED4800E45AF1EE10FA40F321843146B942A8BFE3
:10ED5800394606EE101AB8EEC66A052A80ED046A2E
:10ED68003CF451AD94ED146ADDED0F4A25EE866A48
:10ED7800A4EE876AF0EE674AE6EE264AB0EE646AC9
:10ED8800002B00F0FA83B4EEE45AF1EE10FA40F3E7
:10ED9800F4833146B942A8BF394606EE101AB8EED8
:10EDA800C66A062A80ED056A3CF42DAD94ED186A12
:10EDB800DDED104A25EE866AA4EE876AF0EE674A12
:10EDC800E6EE264AB0EE646A002B00F0CD83B4EE7E
:10EDD800E45AF1EE10FA40F3C7833146B942A8BFAE
:10EDE800394606EE101AB8EEC66A072A80ED066A9A
:10EDF8003CF409AD94ED1C6ADDED114A65EE865AC6
:10EE0800E4EE875AE5EEA67A002B00F0A583F4EE2F
:10EE1800C57AF1EE10FA40F19F833246BA42A8BF94
:10EE28003A46964607EE90EAF8EEE77AC0ED077A9A
:10EE3800FCF7E9BCD9F8245148003DB1421804EB6D
:10EE480082026D785278AA42BDF441AB014404EBCA
:10EE580081040021C9F82441A9F80C12C9F810123C
:10EE6800FDF735BBD9F89C41049B1C1BFFF795B8EF
:10EE780094ED000A039226F077F84549DFF848E157
:10EE8800D1F8EC10434B8EFB012EC917C1EBAE1124
:10EE980007EE901AF8EEE77A1880FDEEE77A039A03
:10EEA80017EE901A5980FCF77EBD07EE904ADFED09
:10EEB8003A6A9FED3A7A89F80442F8EEE77A67EE03
:10EEC800A67A77EE876ABDEEE66A16EE102A203239
:10EED800402A40F29282DFED326A324BBDEEE77A89
:10EEE800C3ED016A17EE102A2032402A00F282820E
:10EEF8009FED2D7AF4EEC77AF1EE10FA40F3FD8318
:10EF0800DFED2A5A9FED2A6A01E0F0EE477AF4EE27
:10EF1800C67AF1EE10FA37EEE57AF6DCDFED257AFF
:10EF2800B4EEE77AF1EE10FA40F1DA83DFED1F5A1A
:10EF38009FED216A01E0B0EE677AB4EEC67AF1EE91
:10EF480010FA77EE257AF6D49FED147AF4EEC77AA4
:10EF5800F1EE10FA40F39F829FED137A77EE677A0D
:10EF680067EEA75A9FED155A9FED156A9FED157A22
:10EF7800A5EE856A27EEA55AA5EE867AE5EE077A0C
:10EF8800C9ED827AFDF751BD58460020C03C0020EB
:10EF980020030020D03D002035FA8E3CDB0FC93F0E
:10EFA8000000000004000020DB0F4940DB0FC940CF
:10EFB800E4CB1641DB0F49C0E4CB16C192E741B957
:10EFC8009730083C15A82ABED34D621025EE866AF4
:10EFD800A5EE076AB0EE675AA6EE265ABDEEC56AD8
:10EFE80016EE100A814200F39E81B842A8BF384647
:10EFF80006EE100AB8EEC66ABCF1000F00F0BC833A
:10F00800D148012A80ED006A3CF4FDAB94ED046A16
:10F018009DED0B5A25EE866AA5EE076AB0EE675A93
:10F02800A6EE265ABDEEC56A16EE106AB14200F386
:10F038007881BE42A8BF3E4606EE106AB8EEC66AA0
:10F04800BCF1000F00F06D83022A80ED016A3CF4E8
:10F05800DAAB94ED086A9DED0C5A25EE866AA5EEAA
:10F06800076AB0EE675AA6EE265ABDEEC56A16EED6
:10F07800106AB14200F35381BE42A8BF3E4606EE75
:10F08800106AB8EEC66ABCF1000F00F0A183032A2B
:10F0980080ED026A3CF4B7AB94ED0C6A9DED0D5A15
:10F0A80025EE866AA5EE076AB0EE675AA6EE265ADE
:10F0B800BDEEC56A16EE106AB14200F32E81BE425B
:10F0C800A8BF3E4606EE106AB8EEC66ABCF1000F4D
:10F0D80000F07383042A80ED036A3CF494AB94ED4A
:10F0E800106A9DED0E5A25EE866AA5EE076AB0EE07
:10F0F800675AA6EE265ABDEEC56A16EE106AB142E8
:10F1080000F30981BE42A8BF3E4606EE106AB8EE7B
:10F11800C66ABCF1000F00F04583052A80ED046A39
:10F128003CF471AB94ED146A9DED0F5A25EE866A96
:10F13800A5EE076AB0EE675AA6EE265ABDEEC56A76
:10F1480016EE106AB14200F3E480BE42A8BF3E4604
:10F1580006EE106AB8EEC66ABCF1000F00F017831D
:10F16800062A80ED056A3CF44EAB94ED186A9DEDD5
:10F17800105A25EE866AA5EE076AB0EE675AA6EE23
:10F18800265ABDEEC56A16EE106AB14200F3BF807A
:10F19800BE42A8BF3E4606EE106AB8EEC66ABCF18B
:10F1A800000F00F07E83072A80ED066A3CF42BAB43
:10F1B80094ED1C6A9DED115A65EE865AE7EE055AE4
:10F1C800E6EEA57AFDEEE77A17EE902A914203DC87
:10F1D800BA42A8BF3A46114607EE901AF8EEE77A07
:10F1E800BCF1000F7FF422AE089B002B7FF41EAE0B
:10F1F800039B079A9342B8BFF0EE647A16E69FED38
:10F20800530A534B25EE800A1C4625F0ADFEE080DC
:10F21800D9F81441FCF74ABE4E484F498446FEF7D8
:10F22800C3B9D9F89C41049B1C1BFEF709B84B498C
:10F23800096811F0805C7EF481AEFEF777BE237D0D
:10F24800FEF774BD93F8FF21AA2A7EF4E2ADD3F845
:10F25800C61149B193F8C221A2F10B0001282DD99A
:10F2680002F0F702062A29D0D3F8D61149B193F84B
:10F27800D221A2F10B00012820D902F0F702062AB8
:10F288001CD0D3F8E61149B193F8E221A2F10B00A2
:10F29800012813D902F0F702062A0FD0D3F8F61185
:10F2A80000293EF4B6AD93F8F231A3F10B02012A1E
:10F2B80004D903F0F703062B7EF4ABAD41F2FC1240
:10F2C8000123A150A370FEF7ADBDF8F753FB029AD6
:10F2D8001F4B1778039A98F80010D9F81441801A30
:10F2E8009880FEF71FBBF8F745FB029A184B177872
:10F2F800039A801A5880FEF780B9F8F73BFB029A08
:10F30800134B1778039A801A5880FEF7B7B90E4640
:10F3180041E70E461CE70E46F7E60E46D2E60E46D5
:10F32800ADE60E4688E6084662E60AA9BDEEE46A3E
:10F3380001EB820296460A48034C09951A4616EED6
:10F34800106A634614E000BFC03C00200000C842B9
:10F35800D03D00203C3A00201C200020A43700208B
:10F36800584600207145A4EC016A00F1100039D01C
:10F3780090ED006AB1EC014A25EE866AA7EE046AB0
:10F38800B0EE674AA6EE864AB0EE446A32B1B4EEF1
:10F39800445AF1EE10FAC8BFB0EE646ABDEEC66A10
:10F3A80016EE10CA664506EE106A04DCBC45A8BF16
:10F3B800BC4606EE10CAB8EEC66A002BD2D1089D2C
:10F3C800002DCFD1039DAC46079DAC45B8BFB0EE2C
:10F3D800646AC7E7D84A1278032A00F07D810022C0
:10F3E800FEF7A3BF099DFCF70EBAD44E06F18002C2
:10F3F800FEF780BADFEDD27AC2E5F4EEC77AF1EE15
:10F4080010FA40F37D81DFEDCF5A9FEDCF6A01E01E
:10F41800F0EE476AF4EEC66AF1EE10FA36EEE57AD7
:10F42800F6DCDFEDCA6AB4EEE67AF1EE10FA40F1E6
:10F438005A81DFEDC45A9FEDC66A01E0B0EE667AE4
:10F44800B4EEC67AF1EE10FA77EE256AF6D49FED9F
:10F45800C17AF4EEC76AF1EE10FA71DD9FEDBE7A5B
:10F4680077EE666A66EEA65A9FEDBC5A9FEDBC6AB7
:10F478009FEDBC7AA5EE856A26EEA55AA5EE867A9A
:10F48800E5EE076A29E59FEDAE8AFFF771BB9FEDB0
:10F49800AC8AFFF745BB9FEDB47AF4EEC77AF1EE7C
:10F4A80010FA44BF9FEDA97A77EE677A58E59FED89
:10F4B800AA7AF4EEC76AF1EE10FA40F32781DFED7D
:10F4C800A15A9FEDA16A01E0F0EE476AF4EEC66A20
:10F4D800F1EE10FA36EEE57AF6DCDFED9C6AB4EE72
:10F4E800E67AF1EE10FA40F10E81DFED965A9FEDC3
:10F4F800986A01E0B0EE667AB4EEC67AF1EE10FAD8
:10F5080077EE256AF6D49FED937AF4EEC76AF1EEAA
:10F5180010FA05DD9FED907A77EE666AFFF777B906
:10F528009FED917AF4EEC76AF1EE10FA44BF9FEDB1
:10F53800877A77EE666AFFF76AB96046FEF7DABF40
:10F548009FED897AF4EEC76AF1EE10FA44BF9FED99
:10F558007F7A77EE666A85E7FDEEE77A17EE902AFE
:10F56800B242FFF65FAC59E4BDEEC66A16EE101A59
:10F57800B142BFF633AC314633E4BDEEC66A16EE8F
:10F58800101AB142BFF606AC314606E4BDEEC66AB3
:10F5980016EE101AB142BFF6D9AB3146FFF7D9BB08
:10F5A800BDEEC66A16EE101AB142BFF6ABAB3146D5
:10F5B800FFF7ABBBBDEEC66A16EE101AB142BFF636
:10F5C8007DAB3146FFF77DBBBDEEC66A16EE101A5D
:10F5D800B142BFF64FAB3146FFF74FBB14EE901A5E
:10F5E800FFF726BB039BAAF8A860D880DFF84C91E8
:10F5F800FCF774BF137C022B7EF428AC92F8FE3122
:10F60800552B7EF423AC92F8FF31AA2B7EF41EAC66
:10F61800D689E759554B37441F6092F80DE041F2FF
:10F6280010210EF1FF337F2B44F801E03EF60EACBB
:10F63800CEF100033EEA03037EF408AC4FEA4E2302
:10F6480041F21821013B6350D08A00B9506A4849F9
:10F6580041F20423E050B2F811305B0103F2FF13CA
:10F668005B120B60B2F8131001B9116A40001E4416
:10F678000644891B41F2082C40F6F476B1FBFEF1F2
:10F68800B14244F80C1048D94FF6F476B14240D94B
:10F6980003212170D26A37493B44184441F20C26B1
:10F6A80041F21C230978A051E25009B925F0C6F9A6
:10F6B800A3780133A370FCF71BBB02287CF418ABBA
:10F6C80041F2B4120123A3546370FCF711BB10F08C
:10F6D8007BFE2369FEF7F9BA22F0C4F9FCF7F7BEFE
:10F6E800F0EE477A30E4F0EE476AB0E699F8783100
:10F6F800002B7BF4A5ACFBF790BCB0EE677A0DE469
:10F70800B0EE667A8DE6F0EE476AFCE6B0EE667A11
:10F71800E3E6022222700022BDE701232370FEF7F0
:10F7280095BB089B002B7FF48FAC039B079EB342CD
:10F73800B8BFB0EE646A87E4507800201C2000202F
:10F7480000000000DB0FC940E4CB1641DB0F49C0C5
:10F75800E4CB16C1DB0FC93FDB0F494092E741B943
:10F768009730083C15A82ABEDB0FC9BF10690020D6
:10F7780030690020F0680020089B002B7FF440AC23
:10F78800039B07988342B8BFB0EE646A38E4089BCD
:10F79800002B7FF4E5AC039B079EB342B8BFB0EEE5
:10F7A800646ADDE4089B002B7FF4B7AC039B079EDB
:10F7B800B342B8BFB0EE646AAFE4089B002B7FF495
:10F7C80089AC039B079EB342B8BFB0EE646A81E47C
:10F7D800089B002B7FF45BAC039B079EB342B8BF2A
:10F7E800B0EE646A53E4132B05D1B0EE480A25F055
:10F7F800BBFB039B1880B0EE480ADAF8083245488C
:10F808009847029B1B78132BB0EE408A7CF472ACAD
:10F8180025F0AAFB039B5880FCF76CBC3E4A3F4B83
:10F8280010681B6898473E4BD6ED006A93ED007A46
:10F838003C4BD3ED007A3C4B83ED020A3B4B67EE21
:10F84800277A234427EEAC7AD3ED007A384B67EE5B
:10F85800277AF0EE665AEDEEA75A93ED006AB1EEFC
:10F86800467AB4EEE57AF1EE10FA08DCB4EEE56A11
:10F87800F1EE10FA8CBFB0EE657AB0EE467A2D4BF9
:10F888001B78012B02D0192B7BF444ABDFED2A7ACD
:10F89800F4EEE7DAF1EE10FACCBF01230023FBF710
:10F8A80044BB089B002B7FF47EAC039B079EB342AE
:10F8B800B8BFB0EE646A76E4DFED207AB4EEE7EA2A
:10F8C800F1EE10FA20DCDFED1E7AB4EEE7EAF1EE95
:10F8D80010FA19D41B4BD3ED007AB1EE677AF4EE27
:10F8E800C7DAF1EE10FA12D4F4EEE7DAF1EE10FA14
:10F8F80088BFF0EE67DA144B86ED00CA1B689342A6
:10F90800BBF612AAFBF73ABADFED10DAF3E7F0EE2E
:10F9180047DAF0E7884F0020A4750020B87500206A
:10F92800F874002004000020503C0020C875002016
:10F93800307600205C7400200000964200C0F84435
:10F9480000C0F8C42C7600201076002000000000CB
:10F95800436A8269D154436A0169826B01338B42DD
:10F9680028BF00234362002A2FD0EFF311815023D0
:10F9780083F31288836B1A68D2072CD470B45E683C
:10F988006EB9456A826A954217D084691444DC606E
:10F998000ED9AA1A5A608562002280F854201A6883
:10F9A80042F00102C9B21A6081F3118870BC704735
:10F9B8000469A21A5A608662EEE7012380F854307F
:10F9C800C9B281F3118870BC7047026D136843F0A7
:10F9D800800313607047C9B281F31188704700BF74
:10F9E800426B10B462B1436CC2684469D11A013BDE
:10F9F800615C5DF8044B08BF13464364C8B27047A6
:10FA0800016A4369C4685B5C0131A14228BF1146A1
:10FA180001625DF8044BD8B2704700BF836B13B125
:10FA280090F854007047836A406A181AB0FA80F058
:10FA380040097047416A836A99420AD3CB1A816B9D
:10FA4800026961B14968501E0B4483420AD2C01A48
:10FA5800704702691144CB1A816B0029F2D1501EFC
:10FA6800C01A704700207047436B43B1426C5B6813
:10FA780093422FBF981AC0689B1AC0187047C26972
:10FA8800036A9A422FBFD01AC0688018C01A7047FC
:10FA98000A4B30B503F10C0493F900205D78072A6E
:10FAA800C8BF143A811804338D7213F8025C855468
:10FAB80013F8012C0A75A342EED130BD7861030812
:10FAC80003682DE9F041DF691FB13B46BDE8F0410D
:10FAD8001847002A164611DD04460D460E4400E07C
:10FAE80023689B68204698470028F9D0236815F8B2
:10FAF800011B1B6820469847AE42F1D1BDE8F08152
:10FB080000232822027043708370C3707047232338
:10FB180003702423C370252383712D2343702E2360
:10FB280003712F23C371704730B50446006D6171AE
:10FB38000368A26823F00103036087B0A3790092E9
:10FB480013F004023DD04FF4805213F002030192E7
:10FB580044D102934FF480630022039311F0010310
:10FB6800059237D1049308238D07694648BF04934B
:10FB78001AF062FA6079236DA17900F00202002A76
:10FB880015BF4FF440324FF480324FF40034002454
:10FB980010F0010F586808BF2246CC074CBF02433B
:10FBA80020EA02025A609A6809074CBF42F008022C
:10FBB80022F008029A601A6842F001021A6007B03F
:10FBC80030BD13F0020301920BD04FF400551346D9
:10FBD8000295C1E7042304930C23C5E74FF40053AF
:10FBE800B7E70293B8E700BF10B50446006DA160FF
:10FBF800036823F001030360A37986B013F00402BD
:10FC0800009141D04FF4805213F00203019244D185
:10FC180002934FF4806362790393D1074FF0000396
:10FC28000493059345BF0423049308230C236946D2
:10FC3800920748BF04931AF0FFF96079236DA17900
:10FC480000F00202002A15BF4FF440324FF4803210
:10FC58004FF40034002410F0010F586808BF224602
:10FC6800CC074CBF024320EA02025A609A6809078F
:10FC78004CBF42F0080222F008029A601A6842F06B
:10FC880001021A6006B010BD13F00203019207D0FA
:10FC98004FF4005113460291BDE74FF40053B7E704
:10FCA8000293B8E70023262203600270272282709D
:10FCB8000122436002718371704700BF1D4B70B50C
:10FCC8001C68236D626BDD69C2B1A36B2BB12B0776
:10FCD80002D5236D08221A6270BD2A06F7D5A26ADA
:10FCE800616A8A4220D0511CA069A162825C2069A5
:10FCF800266D81423285EAD3A362E8E7A906E4D5F6
:10FD0800E26A22B1988C216B80B29047DDE7E16905
:10FD18009B8C6069DBB24E1CE6614354E169E36881
:10FD2800994228BFE261D0E7226D136823F080036F
:10FD38001360CCE7F42A002070B4EFF31186502347
:10FD480083F31288836B1A68D20720D45D686DB973
:10FD5800446A826A944217D081691144D9600ED9E5
:10FD6800A21A5A608462002280F854201A6842F06D
:10FD78000102F1B21A6081F3118870BC7047016901
:10FD88008A1A5A608562EEE7012380F85430F1B28E
:10FD980081F3118870BC704703685B6A03B1184728
:10FDA800704700BF03681B6A03B11847704700BF5C
:10FDB80003682DE9F041DF691FB13B46BDE8F0411A
:10FDC8001847002A164611DD04460D460E4400E089
:10FDD80023689B68204698470028F9D0236815F8BF
:10FDE800011B1B6820469847AE42F1D1BDE8F0815F
:10FDF80003689B69184700BF0368DB68184700BFA2
:10FE080003689B68184700BF03685B68184700BF12
:10FE180003681B68184700BF054B53F8203033B1FF
:10FE28001A689B88918A0B4218BF1B04936170471C
:10FE38008C76002003682DE9F04F03F13845644EB5
:10FE4800AD0A0124755D05F01F066D09022D04FA3F
:10FE580006F400F0A280032D00F0A480012D52D0FA
:10FE68008088B0FA80F4C4F11F04A4B2E50803EB5B
:10FE7800850504F007042E6AA4000F27A74026EA88
:10FE880007062E622E6A01F0030702FA04F47A1EAE
:10FE98003443012AC1F3810CC1F300182C62C1F369
:10FEA800411135D9C60700F19780850700F1A38075
:10FEB800440700F1B180020700F1BF80C60600F1D7
:10FEC800CD80850600F1DB80440600F1E98002065A
:10FED80000F1F780C60500F10581850500F1138161
:10FEE800440500F12181020500F12F81C60400F1CB
:10FEF8003D81850400F14B81440400F159810204DD
:10FF080055D4BDE8F08F334D6E6934436C61A7E773
:10FF1800002422464FF0010E4FF0030904E001329D
:10FF2800102A04F10204ECD00EFA02F636EA0005B3
:10FF3800F5D1D3F808A009FA04F5ED430AEA050A51
:10FF4800C3F808A0D3F808B00CFA04FA4AEA0B0A76
:10FF5800C3F808A0B3F804A01FFA8AFA2AEA06062A
:10FF68009E80B3F804A008FA02F646EA0A06B6B27A
:10FF78009E801E682E401E60D3F800A007FA04F683
:10FF880046EA0A061E60D3F80CA001FA04F605EA50
:10FF98000A0A46EA0A05DD60C1E70E4DAE69344338
:10FFA800AC615DE70B4DEE693443EC6158E71A68C4
:10FFB80022F040421A601A6842EA87771F60DA68BE
:10FFC80022F0404242EA8171D960BDE8F08F00BF5B
:10FFD8005C880308001002401A6822F003021A60C5
:10FFE8001A683A431A60DA6822F003020A4385075E
:08FFF800DA607FF55DAF1A68C5
:020000040801F1
:1000000022F00C021A601A6842EA87021A60DA6863
:1000100022F00C0242EA81024407DA607FF54FAF1A
:100020001A6822F030021A601A6842EA07121A604F
:10003000DA6822F0300242EA0112DA6002077FF544
:1000400041AF1A6822F0C0021A601A6842EA8712A9
:100050001A60DA6822F0C00242EA8112C606DA604B
:100060007FF533AF1A6822F440721A601A6842EAC8
:1000700007221A60DA6822F4407242EA01228506F9
:10008000DA607FF525AF1A6822F440621A601A68B8
:1000900042EA87221A60DA6822F4406242EA812248
:1000A0004406DA607FF517AF1A6822F440521A60EE
:1000B0001A6842EA07321A60DA6822F4405242EAC9
:1000C0000132DA6002067FF509AF1A6822F4404275
:1000D0001A601A6842EA87321A60DA6822F44042EB
:1000E00042EA8132C605DA607FF5FBAE1A6822F477
:1000F00040321A601A6842EA07421A60DA6822F44B
:10010000403242EA01428505DA607FF5EDAE1A68B9
:1001100022F440221A601A6842EA87421A60DA68BA
:1001200022F4402242EA81424405DA607FF5DFAEE4
:100130001A6822F440121A601A6842EA07521A60DA
:10014000DA6822F4401242EA0152DA6002057FF5D1
:10015000D1AE1A6822F440021A601A6842EA875245
:100160001A60DA6822F4400242EA8152C604DA6078
:100170007FF5C3AE1A6822F040721A601A6842EA2C
:1001800007621A60DA6822F0407242EA016285046E
:10019000DA607FF5B5AE1A6822F040621A601A681C
:1001A00042EA87621A60DA6822F0406242EA8162BB
:1001B0004404DA607FF5A7AE1A6822F040521A6054
:1001C0001A6842EA07721A60DA6822F0405242EA7C
:1001D0000172DA6097E600BF036803F138422DE947
:1001E000F04F920A584DAA5C02F01F0552090124F3
:1001F000022A04FA05F400F08C80032A00F08E80B5
:10020000012A3CD001F003077A1E012AC1F3810CB8
:10021000C1F300188088C1F3411135D9C60700F138
:100220009780850700F1A380440700F1B1800207A1
:1002300000F1BF80C60600F1CD80850600F1DB80AD
:10024000440600F1E980020600F1F780C60500F1DE
:100250000581850500F11381440500F12181020526
:1002600000F12F81C60400F13D81850400F14B812E
:10027000440400F15981020455D4BDE8F08F334A9B
:1002800055692C435461BDE7002422464FF0010E0E
:100290004FF0030904E00132102A04F10204ECD00B
:1002A0000EFA02F636EA0005F5D1D3F808A009FAED
:1002B00004F5ED430AEA050AC3F808A0D3F808B02C
:1002C0000CFA04FA4AEA0B0AC3F808A0B3F804A02F
:1002D0001FFA8AFA2AEA06069E80B3F804A008FAF2
:1002E00002F646EA0A06B6B29E801E682E401E60DE
:1002F000D3F800A007FA04F646EA0A061E60D3F80F
:100300000CA001FA04F605EA0A0A46EA0A05DD60CD
:10031000C1E70E4A95692C43946173E70B4AD5698E
:100320002C43D4616EE71A6822F040421A601A68C2
:1003300042EA87771F60DA6822F0404242EA817120
:10034000D960BDE8F08F00BF5C8803080010024050
:100350001A6822F003021A601A683A431A60DA68CF
:1003600022F003020A438507DA607FF55DAF1A6861
:1003700022F00C021A601A6842EA87021A60DA68F0
:1003800022F00C0242EA81024407DA607FF54FAFA7
:100390001A6822F030021A601A6842EA07121A60DC
:1003A000DA6822F0300242EA0112DA6002077FF5D1
:1003B00041AF1A6822F0C0021A601A6842EA871236
:1003C0001A60DA6822F0C00242EA8112C606DA60D8
:1003D0007FF533AF1A6822F440721A601A6842EA55
:1003E00007221A60DA6822F4407242EA0122850686
:1003F000DA607FF525AF1A6822F440621A601A6845
:1004000042EA87221A60DA6822F4406242EA8122D4
:100410004406DA607FF517AF1A6822F440521A607A
:100420001A6842EA07321A60DA6822F4405242EA55
:100430000132DA6002067FF509AF1A6822F4404201
:100440001A601A6842EA87321A60DA6822F4404277
:1004500042EA8132C605DA607FF5FBAE1A6822F403
:1004600040321A601A6842EA07421A60DA6822F4D7
:10047000403242EA01428505DA607FF5EDAE1A6846
:1004800022F440221A601A6842EA87421A60DA6847
:1004900022F4402242EA81424405DA607FF5DFAE71
:1004A0001A6822F440121A601A6842EA07521A6067
:1004B000DA6822F4401242EA0152DA6002057FF55E
:1004C000D1AE1A6822F440021A601A6842EA8752D2
:1004D0001A60DA6822F4400242EA8152C604DA6005
:1004E0007FF5C3AE1A6822F040721A601A6842EAB9
:1004F00007621A60DA6822F0407242EA01628504FB
:10050000DA607FF5B5AE1A6822F040621A601A68A8
:1005100042EA87621A60DA6822F0406242EA816247
:100520004404DA607FF5A7AE1A6822F040521A60E0
:100530001A6842EA07721A60DA6822F0405242EA08
:100540000172DA6097E600BF10B50409013C052C82
:1005500017D80D4B33F8142000F00F0042FA00F3C7
:1005600013F001030DD0012303FA00F0013810400D
:1005700024F0A8F8054A064B125D104403EBC000B6
:1005800010BD002010BD00BF488803085488030830
:10059000F87E00202DE9F04F4A484B4B4B4C4FF072
:1005A00090414FF0010A4FF002094FF004084FF05C
:1005B000080C4FF0100E20274026802530F8022B23
:1005C00012F0010F03D01960A3F804A0083312F051
:1005D000020F03D01960A3F80490083312F0040F3F
:1005E00003D01960A3F80480083312F0080F03D079
:1005F0001960A3F804C0083312F0100F03D019607B
:10060000A3F804E0083312F0200F02D019609F8095
:10061000083312F0400F02D019609E80083312F0A8
:10062000800F02D019609D80083312F4807F05D0BE
:100630004FF4807B1960A3F804B0083312F4007FF4
:1006400005D04FF4007B1960A3F804B0083312F40E
:10065000806F05D04FF4806B1960A3F804B00833A5
:1006600012F4006F05D04FF4006B1960A3F804B0CA
:10067000083312F4805F05D04FF4805B1960A3F853
:1006800004B0083312F4005F05D04FF4005B19602A
:10069000A3F804B0083312F4804F05D04FF4804B18
:1006A0001960A3F804B00833D20B04D04FF4004211
:1006B00019609A80083301F58061A1427FF47EAF12
:1006C000BDE8F08F48880308F87E00200018004835
:1006D000002867D003682DE9F04F03F138445C4EE1
:1006E000A40A0125345D04F01F066409022C05FAF2
:1006F00006F558D0032C00F0A580012C58D0808836
:10070000B0FA80F4C4F11F04A4B2E50803EB850538
:1007100004F007042E6AA4000F27A74026EA070664
:100720002E622E6A01F00307A2407C1E3243012C88
:10073000C1F3810CC1F300182A62C1F341113CD905
:10074000C60700F18980850700F19580440700F114
:10075000A380020700F1B180C60600F1BF808506C4
:1007600000F1CD80440600F1DB80020600F1E98053
:10077000C60500F1F780850500F10581440500F10B
:100780001381020500F12181C60400F12F81850447
:1007900000F13D81440400F14B81020400F15981D4
:1007A000BDE8F08F70472B4CA6693543A561A6E7DD
:1007B000284C666935436561A1E7002422464FF065
:1007C000010E4FF0030904E00132102A04F1020483
:1007D000E6D00EFA02F636EA0005F5D1D3F808A005
:1007E00009FA04F5ED430AEA050AC3F808A0D3F8AC
:1007F00008B00CFA04FA4AEA0B0AC3F808A0B3F8E6
:1008000004A01FFA8AFA2AEA06069E80B3F804A01A
:1008100008FA02F646EA0A06B6B29E801E682E4024
:100820001E60D3F800A007FA04F646EA0A061E6026
:10083000D3F80CA001FA04F605EA0A0A46EA0A050A
:10084000DD60C1E7034CE6693543E56157E700BF6A
:100850005C880308001002401A6822F003021A6044
:100860001A683A431A60DA6822F003020A438507DD
:10087000DA607FF56BAF1A6822F00C021A601A6812
:1008800042EA87021A60DA6822F00C0242EA810228
:100890004407DA607FF55DAF1A6822F030021A6013
:1008A0001A6842EA07121A60DA6822F0300242EA55
:1008B0000112DA6002077FF54FAF1A6822F0C0021A
:1008C0001A601A6842EA87121A60DA6822F0C002D7
:1008D00042EA8112C606DA607FF541AF1A6822F457
:1008E00040721A601A6842EA07221A60DA6822F433
:1008F000407242EA01228506DA607FF533AF1A685A
:1009000022F440621A601A6842EA87221A60DA68A2
:1009100022F4406242EA81224406DA607FF525AF84
:100920001A6822F440521A601A6842EA07321A60C2
:10093000DA6822F4405242EA0132DA6002067FF5B8
:1009400017AF1A6822F440421A601A6842EA8732E6
:100950001A60DA6822F4404242EA8132C605DA605F
:100960007FF509AF1A6822F440321A601A6842EA29
:1009700007421A60DA6822F4403242EA01428505F1
:10098000DA607FF5FBAE1A6822F440221A601A681A
:1009900042EA87421A60DA6822F4402242EA81423F
:1009A0004405DA607FF5EDAE1A6822F440121A6051
:1009B0001A6842EA07521A60DA6822F4401242EAE0
:1009C0000152DA6002057FF5DFAE1A6822F44002B8
:1009D0001A601A6842EA87521A60DA6822F4400202
:1009E00042EA8152C604DA607FF5D1AE1A6822F07D
:1009F00040721A601A6842EA07621A60DA6822F0E6
:100A0000407242EA01628504DA607FF5C3AE1A687B
:100A100022F040621A601A6842EA87621A60DA6855
:100A200022F0406242EA81624404DA607FF5B5AEAA
:100A30001A6822F040521A601A6842EA07721A6075
:100A4000DA6822F0405242EA0172DA6002047FF56D
:100A5000A7AE1A6822F040421A601A6842EA877705
:100A60001F60DA6822F0404242EA8171D960BDE835
:100A7000F08F00BF002852D0036803F138422DE9FF
:100A8000F04F920A504DAA5C02F01F055209012452
:100A9000022A04FA05F443D0032A00F09080012AC8
:100AA00043D001F003077A1E012AC1F3810CC1F380
:100AB00000188088C1F341113CD9C60700F1888035
:100AC000850700F19480440700F1A280020700F13D
:100AD000B080C60600F1BE80850600F1CC804406D9
:100AE00000F1DA80020600F1E880C60500F1F68028
:100AF000850500F10481440500F11281020500F131
:100B00002081C60400F12E81850400F13C8144045B
:100B100000F14A81020400F15881BDE8F08F70476E
:100B20002A4A95692C439461BBE7284A55692C43AE
:100B30005461B6E7002422464FF0010E4FF003093E
:100B400004E00132102A04F10204E6D00EFA02F6A3
:100B500036EA0005F5D1D3F808A009FA04F5ED430B
:100B60000AEA050AC3F808A0D3F808B00CFA04FA98
:100B70004AEA0B0AC3F808A0B3F804A01FFA8AFADD
:100B80002AEA06069E80B3F804A008FA02F646EAAE
:100B90000A06B6B29E801E682E401E60D3F800A0E2
:100BA00007FA04F646EA0A061E60D3F80CA001FA1A
:100BB00004F605EA0A0A46EA0A05DD60C1E7034AC7
:100BC000D5692C43D4616CE75C88030800100240AF
:100BD0001A6822F003021A601A683A431A60DA6847
:100BE00022F003020A438507DA607FF56CAF1A68CA
:100BF00022F00C021A601A6842EA87021A60DA6868
:100C000022F00C0242EA81024407DA607FF55EAF0F
:100C10001A6822F030021A601A6842EA07121A6053
:100C2000DA6822F0300242EA0112DA6002077FF548
:100C300050AF1A6822F0C0021A601A6842EA87129E
:100C40001A60DA6822F0C00242EA8112C606DA604F
:100C50007FF542AF1A6822F440721A601A6842EABD
:100C600007221A60DA6822F4407242EA01228506FD
:100C7000DA607FF534AF1A6822F440621A601A68AD
:100C800042EA87221A60DA6822F4406242EA81224C
:100C90004406DA607FF526AF1A6822F440521A60E3
:100CA0001A6842EA07321A60DA6822F4405242EACD
:100CB0000132DA6002067FF518AF1A6822F440426A
:100CC0001A601A6842EA87321A60DA6822F44042EF
:100CD00042EA8132C605DA607FF50AAF1A6822F46B
:100CE00040321A601A6842EA07421A60DA6822F44F
:100CF000403242EA01428505DA607FF5FCAE1A68AF
:100D000022F440221A601A6842EA87421A60DA68BE
:100D100022F4402242EA81424405DA607FF5EEAED9
:100D20001A6822F440121A601A6842EA07521A60DE
:100D3000DA6822F4401242EA0152DA6002057FF5D5
:100D4000E0AE1A6822F440021A601A6842EA87523A
:100D50001A60DA6822F4400242EA8152C604DA607C
:100D60007FF5D2AE1A6822F040721A601A6842EA21
:100D700007621A60DA6822F0407242EA0162850472
:100D8000DA607FF5C4AE1A6822F040621A601A6811
:100D900042EA87621A60DA6822F0406242EA8162BF
:100DA0004404DA607FF5B6AE1A6822F040521A6049
:100DB0001A6842EA07721A60DA6822F0405242EA80
:100DC0000172DA6002047FF5A8AE1A6822F0404290
:100DD0001A601A6842EA87771F60DA6822F0404298
:100DE00042EA8171D960BDE8F08F00BF10B103689D
:100DF00082881A85704700BF10B1036882889A61A3
:100E0000704700BF38B100298388026814BF0021F1
:100E100010218B409361704710B40A4B0A4A1C782A
:100E200001238340234052F8200029B9B3FA83F10B
:100E300049095DF8044BE5E7191C18BF01215DF86D
:100E4000044BDFE7887600208C76002030B1036801
:100E500082881B8A1A4214BF01200020704700BFFD
:100E60002DE9F0410B4E346873691C400FD0DFF858
:100E700028800127B4FA84F3C3F11F0307FA03F5AE
:100E800058F8230003689847AC437561F2D1BDE878
:100E9000F08100BF00040140342200202DE9F04120
:100EA0000B4E346873691C400FD0DFF8288001278F
:100EB000B4FA84F3C3F11F0307FA03F558F82300CB
:100EC00003689847AC437561F2D1BDE8F08100BF7B
:100ED00000040140342200202DE9F0410B4E34681B
:100EE00073691C400FD0DFF828800127B4FA84F31F
:100EF000C3F11F0307FA03F558F823000368984766
:100F0000AC437561F2D1BDE8F08100BF000401403F
:100F1000342200202DE9F0410B4E346873691C40E7
:100F20000FD0DFF828800127B4FA84F3C3F11F0340
:100F300007FA03F558F8230003689847AC43756136
:100F4000F2D1BDE8F08100BF00040140342200204E
:100F50002DE9F0410B4E346873691C400FD0DFF867
:100F600028800127B4FA84F3C3F11F0307FA03F5BD
:100F700058F8230003689847AC437561F2D1BDE887
:100F8000F08100BF00040140342200202DE9F0412F
:100F90000B4E346873691C400FD0DFF8288001279E
:100FA000B4FA84F3C3F11F0307FA03F558F82300DA
:100FB00003689847AC437561F2D1BDE8F08100BF8A
:100FC00000040140342200202DE9F0410B4E34682A
:100FD00073691C400FD0DFF828800127B4FA84F32E
:100FE000C3F11F0307FA03F558F823000368984775
:100FF000AC437561F2D1BDE8F08100BF000401404F
:1010000034220020084A936910B5084C43F00103CC
:10101000936120464022002124F067FF4FF0FF3308
:101020002364C4F8433010BD001002403422002075
:1010300003681B6A184700BF70B44E1C0568C27273
:101040008672AC69A44670BC604700BF2DE9F041D0
:10105000044618460D461646984622F019FE2768A3
:10106000E6722844A07229467D69434632462046EE
:10107000AC46BDE8F0416047036810B504461B6804
:101080009847236820469B689847A37B0133A37346
:1010900010BD00BF03681B69184700BF10B5036887
:1010A00004469B689847FF2301226373227310BD97
:1010B00008B5FFF749FA38B12D2282710022C271BA
:1010C0002021BDE80840D5E408BD00BF0B4B984285
:1010D00006D0A3F5784398420DD04FF0FF3070470B
:1010E0000022074B03EB02135A89013292B25A8154
:1010F000588980B270470122F3E700BF00300140F9
:10110000283D0020F8B50546806816461F4610B1F8
:10111000036882881A8541F08001686840F2E934EA
:1011200001E0002C44D00389013C13F0020FA4B26B
:10113000F7D0017340F2E93101E0002938D003898A
:10114000013913F0010F89B2F7D0037B68688389F6
:101150004FF0000C4FF47A714FF6FF724FF0FF0E14
:10116000674502D11DE0914219D0038901399C07DE
:1011700089B2F8D580F80CE04FF47A7102E0A1B2A0
:1011800091420CD00389DB0701F1FF34F7D5037BD3
:10119000DBB20EB1337001360CF1010CE0E7FFF762
:1011A00095FFAB6813B11A689B8893610120F8BD65
:1011B000FFF78CFFCAE700BF38B5836804461546C1
:1011C00013B11A689B881385606840F2E93300E028
:1011D0007BB30289013B12F0020F9BB2F8D001737E
:1011E00040F2E93300E023B30289013B12F0010F22
:1011F0009BB2F8D0037B606840F2E93300E0DBB1DA
:101200000189013B11F0020F9BB2F8D0057340F247
:10121000E93300E083B10289013B12F0010F9BB278
:10122000F8D0037BA36813B11A689B8893610120EF
:1012300038BDFFF74BFFDEE7FFF748FFF2E700BFDF
:10124000F0B50E460178012985B004464BD002293D
:101250004FD11D46836846F0800113B118689B8802
:101260000385606840F2E93301E0002B55D0068920
:10127000013B16F0020F9BB2F7D0017340F2E93345
:1012800001E0002B49D00189013B11F0010F9BB215
:10129000F7D0037B60684FF0000C83894FF6FF7630
:1012A0004FF47A734FF0FF0E654502D126E0B3424A
:1012B00022D00189013B8F079BB2F8D580F80CE062
:1012C0004FF47A7302E0BBB2B34215D00189C9076B
:1012D00003F1FF37F7D5017BC9B20AB111700132B2
:1012E0000CF1010CE0E790F90400411C01D0022848
:1012F0000CDD002005B0F0BDFFF7E8FEA3688BB160
:101300001A689B889361012005B0F0BD6179009255
:101310003246F1F7CBFF05B0F0BD0392FFF7D6FEE2
:10132000039AB7E70120E5E7F8B50378012B49D028
:10133000022B4DD1836801F07F0113B11C689B889B
:10134000238504461546406840F2E93302E0002B4D
:1013500000F0B1800289013B12F0020F9BB2F6D07F
:10136000017340F2E93302E0002B00F0A48002890F
:10137000013B12F0010F9BB2F6D0037B606840F294
:10138000E93302E0002B00F093800189013B11F06A
:10139000020F9BB2F6D0057340F2E93302E0002B56
:1013A00000F086800289013B12F0010F9BB2F6D05B
:1013B000037BA368002B00F088801A689B889361E8
:1013C0000120F8BD90F904305C1C01D0022B01DD36
:1013D0000020F8BD464C03EB830304EB83035E68F7
:1013E000002EF5D04579434C4FF420436D00A364A3
:1013F000EDB249F6FF73B06907044CD470683E4FF4
:1014000045F0807343F49033384018434FF4204341
:101410007060A36401E05F1C50D0B06910F002005E
:1014200003F1FF33F7D04FF42043A364B16249F6D0
:10143000FF7301E09F1C4AD0B06910F0800003F1F7
:10144000FF33F7D073682C4945F000750B4045F425
:1014500080351D434FF42043A364756049F6FF7344
:1014600001E0991C33D0B06910F0020003F1FF33A2
:10147000F7D04FF42043B262A3641A4602E012F19F
:10148000FF322DD3B36913F02003F8D02023A264D8
:10149000F3610120F8BD013B981CACD1174A1388B9
:1014A00001339BB24FF0FF311380A1640020F8BDDF
:1014B000FFF70CFE7DE7FFF709FE5FE70F4AA36425
:1014C000138801339BB21380F8BD0120F8BD0B4A8D
:1014D000138801339BB24FF0FF311380A164F8BD34
:1014E0000649A2640A88013292B218460A80F8BD01
:1014F0006076002034220020009800FC142D00208B
:10150000427A02B9704710B504460368406804F196
:101510000A0198470023637210BD00BF437A5A1C2A
:101520000344D2B242729972037A934200D802B94C
:10153000704710B504460368406804F10A019847F3
:101540000023637210BD00BF98B10B4B012210B491
:1015500002FA01F103F1750402E00333A34209D05A
:101560001A788242F9D15A780A42F6D001205DF801
:10157000044B70470020FAE78461030830B40A4D39
:10158000002305F10C0401E0272B09D003EB4302F3
:101590000133A15C8142F7D12A4430BC907B704773
:1015A000002030BC704700BF786103082DE9F3418B
:1015B000056906460F467DBBD0F80080C8F30A03D4
:1015C00023B30023D6F8008001931FF0BFFC04284A
:1015D00019D1224C236943F001032361BBB2A8F85F
:1015E00000301FF0B3FC04282ED108F10203019350
:1015F000019B3F0C1F801FF0A9FC2369042823F0E6
:101600000103236125D06FF0010505E01FF09EFC6A
:10161000042805D04FF0FF35284602B0BDE8F08120
:101620000E4C236943F002032361C4F8148023693C
:1016300043F0400323611FF089FC2369042823F051
:1016400002032361BDD0E5E7236923F00103236191
:10165000D9E7336804333360DEE700BF002002407F
:10166000F8B504460D468E180027B54201D1206911
:10167000F8BDE368591CE160234415F8012B1A7288
:101680000429F2D1A1682046FFF790FFE7602061AE
:10169000EBE770B5448806460D46C4F30B042246BA
:1016A0000021284624F021FC33690A4A934209D3D9
:1016B000094A934206D2224628461946BDE87040A0
:1016C00023F082BA23B121462846BDE8704018476E
:1016D00070BD00BF34C603081CC70308064B07498A
:1016E0008B4202D30023184670471A88C2F30B02BC
:1016F0009042F8D01433F3E7C0C1030834C603089E
:10170000024A136823EA0000106070475C820020E0
:1017100030B4034600F12405064C07CC0C3343F8E3
:101720000C0C43F8081C43F8042CAB42F4D130BC39
:10173000704700BFFC610308034B33F80C2F028095
:101740009B788370704700BFFC610308084B1968E1
:1017500061B130B45D68074C642202FB05F2B2FB54
:10176000F1F2228030BC002018605860704700BF42
:1017700080220020182D00200B4A13680360536854
:10178000436030B59368094C83601421002301FB4A
:1017900003429579AD0602D51379C37230BD01338A
:1017A0000C2BF4D130BD00BF0B6203083886030850
:1017B000704700BFF0B53B4B5B79012B83B03AD04B
:1017C000022B0FD0384B00221A805A80374B1B78DF
:1017D000022B05D1344A364B5188128819805A8021
:1017E00003B0F0BD334B1B681B01EFD5FF200DF09C
:1017F0000BFE03780A2B51D8B0F902202E49D317DB
:1018000081FB0212C3EBA2039BB207EE903AB8EE43
:10181000670A2A4C04F10C006381EEF745FEFCEEEA
:10182000C07A214A6389CDED017A5380BDF8043036
:1018300023811380CAE7224A224B92781F4D33F846
:101840001240A4B207EE904A05F13400B8EE670AE0
:10185000EEF72AFE1C4A1449107896785378FCEE6D
:10186000C07A00EB4010CDED017ABDF8042044F6BB
:10187000FB77C3EB033300FB027200FB0474B2FB83
:10188000F3F2B4FBF3F3B2FBF6F2B3FBF6F392B26E
:101890009BB22A866B860A804B8097E79FED0B0AE6
:1018A0000023B6E7A8400020D43E0020CC3D002015
:1018B000D03D002018500020676666668022002018
:1018C0003876002058760020F580002000000000C7
:1018D000F8B5314D31496879314C324B324E0422E2
:1018E00064270A7001284FF0000184F8582084F81A
:1018F0006170A4F85A10A4F85C1084F86010616656
:101900003170198059802DD002280ED0A979274A2C
:1019100000230229136084F868305360936034D048
:1019200004292DD001290ED0F8BD282204F1080089
:1019300024F0DBFA4CF250319FED1D0A04F10C004B
:10194000F0F782FDE2E71B4AE36653609360D360E1
:101950009FED190A02F110004CF25031BDE8F84039
:10196000F0F772BD282204F1300024F0BEFA4CF2E8
:1019700050319FED0F0A04F13400F0F765FDC5E723
:101980000E4AC4F8AC305360F8BD0D4AC4F8A0301C
:1019900053609360F8BD00BFA8400020507800203D
:1019A00080220020D43E0020EA3E0020B8400020E3
:1019B000CDCCCC3DEC220020CDCCCC3E2C23002045
:1019C00020230020F8B5264C94F8B430002B46D0E4
:1019D00094F8B530002B42D094F8B63003F0FF07EE
:1019E000002B3CD1D4F8B830C31A002B37DB1D4B89
:1019F0001D491B780625013B05FB03120A26128CA4
:101A0000B2FBF6F2D4F8BC6006F1010E0E4405FB01
:101A1000031196F82E60CB8BC4F8BCE072431844D7
:101A20001044BEF10E0F88BFC4F8BC70C4F8B800F3
:101A3000F5F777FA012384F8B6300C4BD4F8C020C0
:101A40001B8AD4F8C410536000234B620B889BB2EE
:101A500043F001030B80136843F001031360F8BDEA
:101A600080220020307B0020FC6103083C7B0020AA
:101A7000044B587920B1044B1878003018BF01206E
:101A8000704700BFA8400020EA3E00201F4B187896
:101A9000002839D01E4A1389FBB11E4A9FED1E6AE9
:101AA000D2ED026A07EE903AF8EEE66AF8EE677A4F
:101AB00007EE103A77EEE66AB8EEC77A66EE866A07
:101AC000C6EE877AFDEEE77A17EE900A6428A8BF83
:101AD000642020EAE070C0B2704710B40F4B547815
:101AE0001B88117804FB1032091B642300FB01F0F2
:101AF00003FB02F3B3FBF0F06428A8BF64205DF899
:101B0000044B20EAE070C0B2704700BFEA3E0020FC
:101B1000A8400020B84000200000C842D43E002069
:101B20002DE9F04F794D81B0F5F728FFD5F8CC407D
:101B30000022C5F8C820002C00F0A580237D052BCD
:101B4000074617D9216A23690B44C31A9342B8BFC9
:101B500005F1CC010ADBD5E0137D052B0AD9136A08
:101B600012691344FB1A002B80F2CC8051F8042F29
:101B7000002AF1D14FF0010B0023B9461E46C5F8EB
:101B8000C83098469A46274623E07A6A39693B7DF1
:101B9000A9EB0204B4FBF1F40134A4B213FB04F387
:101BA000013301369BB2B6B23C83FB82984506D224
:101BB000BBF1000F01D1012C5FD99846BA46D5F888
:101BC000C830013305EB8302C5F8C830D2F8CC70B9
:101BD00047B3BB68C3B1FC8A002CD6D1396A4846EA
:101BE000A9EB01019847D0B195F82C31002B52D1C7
:101BF0003B7DC7F82490013601334FF00102B6B2A5
